:020000040000FA
:080000000002040000000000F2
:04000C00A43B000011
:10001000A43B0000A43B0000A43B0000A43B000064
:10002000A43B0000A43B0000A43B0000A43B000054
:10003000A43B0000A43B0000A43B0000A43B000044
:10004000A43B0000A43B0000A43B0000A43B000034
:10005000A43B0000A43B0000A43B0000A43B000024
:10006000A43B0000A43B0000A43B0000A43B000014
:10007000A43B0000A43B0000A43B0000A43B000004
:10008000A43B0000A43B0000A43B0000A43B0000F4
:10009000A43B0000A43B0000A43B0000A43B0000E4
:1000A000E43B0000A43B0000A43B0000A43B000094
:1000B000A43B0000A43B0000A43B0000A43B0000C4
:1000C000A43B0000A43B0000A43B0000A43B0000B4
:1000D000A43B0000A43B0000A43B0000A43B0000A4
:1000E000A43B0000A43B0000A43B0000A43B000094
:1000F000A43B0000A43B0000A43B0000A43B000084
:10010000A43B0000A43B0000A43B0000A43B000073
:10011000A43B0000A43B0000A43B0000A43B000063
:10012000A43B0000A43B0000A43B0000A43B000053
:10013000A43B0000A43B0000A43B0000A43B000043
:10014000A43B0000A43B0000A43B0000A43B000033
:10015000A43B0000A43B0000A43B0000A43B000023
:10016000A43B0000A43B0000A43B0000A43B000013
:10017000A43B0000A43B0000A43B0000A43B000003
:10018000A43B0000A43B0000A43B0000A43B0000F3
:10019000A43B0000A43B0000A43B0000A43B0000E3
:1001A000A43B0000A43B0000A43B0000A43B0000D3
:1001B000A43B0000A43B0000A43B0000A43B0000C3
:1001C000A43B0000A43B0000A43B0000A43B0000B3
:1001D000A43B0000A43B0000A43B0000A43B0000A3
:1001E000A43B0000A43B0000A43B0000A43B000093
:1001F000A43B0000A43B0000A43B0000A43B000083
:1004000000802000E1FF2100018009000018EB00BE
:100410002060EF00040028008411880004402000C0
:1004200094118800A4002000C41188002C23EF0040
:100430002A23EF000FF82100F0FF210020A0B700D1
:10044000000000000028EF000628EF002868EF00F9
:100450002968EF0097C0A900040E2000140288004C
:100460002CA3EF002AA3EF002400240034168800F8
:10047000CA62A800C662A900CA82A800C682A900F2
:10048000A00020008C3B02000000000004082400B3
:10049000641688000470200094168800440520002B
:1004A000F41688000428210024178800CA02A90035
:1004B000C602A90040A7A900283C020000000000D5
:1004C0002D28A8002D48A9002D68A800CA02A9005F
:1004D000C602A90001002000010078004E3602008B
:1004E000000000008100E8003322AF00FEFF37006B
:1004F000A0118800500120000008E600F6FF370038
:10050000783D020000000000A4E0270014B388003A
:10051000423F020000000000903F02000000000087
:100520000CEBB700645880006A24E10003003E0031
:10053000A0C0B3000CEBB700060037006458800081
:1005400003042000041CE10002003E0000C4B300CC
:100550000CEBB700BE3F02000000000008400200A4
:10056000000000008441020000000000D762A800E3
:1005700060C0B30068F6B70010C0B30069F6B700FA
:10058000C63F02000000000010C0B3000AEBB70035
:1005900010C0B3000BEBB7005F76EF006076EF00A2
:1005A0000442020000000000F4FF200044588800CC
:1005B000062BEF00050020000500780072360200CF
:1005C000000000000040B3004220AF0005003700EB
:1005D0008502E80062F6B700BA450200000000009C
:1005E000F5FF370040C1B3005FF6B700A0C0B3000D
:1005F00060F6B7000442020000000000082BEF0084
:1006000004FF200034588800050020000500780011
:100610009A360200000000000040B3004220AF0004
:10062000050037008502E80062F6B700BA4502000F
:1006300000000000F5FF3700A0C5B3005FF6B7006B
:10064000A0C0B30060F6B700044202000000000042
:10065000082BEF0004F0200034588800050020002B
:1006600005007800B2360200000000000040B30030
:100670004220AF00050037008502E80062F6B700AF
:10068000BA45020000000000F5FF370020C3B300A8
:100690005FF6B70040C1B30060F6B7000442020045
:1006A00000000000082BEF00F40020003458880000
:1006B0000500200005007800CA3602000000000096
:1006C0000040B3004220AF00050037008502E8007B
:1006D00062F6B700BA45020000000000F5FF3700DF
:1006E00010C0B30062F2B7001C4702000000000017
:1006F00004E0270014B38800423F0200000000001D
:10070000903F020000000000C5EAB700BE3F0200B3
:1007100000000000245680004822DE00F4CFB20022
:1007200002003A0010C0B300C5EAB70014E0270089
:1007300014B38800423F0200000000009E47020000
:1007400000000000B0568800C1568800BE3F02007D
:1007500000000000C45680006020E10005003E005B
:100760000C003900B45680006520E10001003E0015
:1007700008003700C45680006020E10008003900FE
:1007800004003E00B4568000430620000418E10037
:1007900003003E0024032000B4568800D82AEF004E
:1007A00054E0270014B38800423F0200000000001C
:1007B000903F020000000000BFEAB700BE3F020009
:1007C00000000000BF4AE20004003200F45580003F
:1007D0004822DE00F4CFB20002003A0020C0B3008D
:1007E000BFEAB70084E0270014B38800423F02004C
:1007F00000000000D04702000000000050598800AF
:10080000BE3F02000000000054598000C31F2200B8
:100810000418E10004003E005459800003A32200A4
:100820000418E10002003100C41F2200545988005E
:100830000100200001007800E03602000000000006
:100840008100E8003322AF00FEFF3700A0118800CE
:10085000C00020000008E600F6FF37005059800075
:1008600004002000FA470200000000003322AF001D
:10087000FEFF370004022000A411880054598000B4
:10088000610052005059880054598000F40FB200A2
:10089000745988002BCBBF002AEBB7002B6BEF00FD
:1008A00054598000F40FB2006459880000C2B300AC
:1008B00079F2B7007A72EF002CCBBF007BF2B70061
:1008C0002ECBBF007CF2B7007D72EF007E72EF008E
:1008D0007F72EF008072EF00703C020000000000A9
:1008E0002E3D020000000000804278000040EB0036
:1008F0000AE0AF000000E8000004E00002003A0057
:1009000000000000F6FF370010C0B30052EEB70041
:1009100010C0B3009CEAB7002D08A900684A020085
:10092000000000006104E10002003E0010C0B300BE
:100930009DEAB7002D28AE000B0037000100200013
:1009400001007800FE360200000000008100E8008F
:100950003322AF00FEFF3700A011880020012000E5
:100960000008E600F6FF3700E45480004822DE006D
:100970006124E1000F003A002C500200000000004A
:100980002D28AE000B003700010020000100780088
:100990001E370200000000008100E8003322AF0093
:1009A000FEFF3700A0118800700120000008E6005B
:1009B000F6FF37002D88A9006028EF006228EF00BD
:1009C00014002000444388006A28EF005B68EF00B1
:1009D0005D68EF005F68EF008441020000000000E6
:1009E0002E3D020000000000804278000040EB0035
:1009F0000AE0AF000000E8000004E00002003A0056
:100A000000000000F6FF3700505E0200000000000A
:100A1000F05F020000000000E45480004822DE0085
:100A20006124E10002003A006E7E02000000000036
:100A30002D28AE008D0037004E6EEF0074728000DE
:100A40007B24E10089003200757280000B60EF00AA
:100A50000600200001002000010078004437020059
:100A6000000000008100E8003322AF00FEFF3700E5
:100A7000A0118800900020000008E600F6FF370073
:100A8000050078008600780044002000526B0200C8
:100A9000000000004ECEBF000160EF004200DD000C
:100AA00024C9200004004000900278001003900048
:100AB0000100200001007800603702000000000003
:100AC0008100E8003322AF00FEFF3700A01188004C
:100AD000400020000008E600F6FF3700050078001F
:100AE0008600780084002000526B020000000000A5
:100AF0003322AF00FEFF370004022000A41188005B
:100B00004ECEBF000160EF004200DD00E4CF2000C8
:100B100004004000900278001003900001002000C3
:100B20000100780078370200000000008100E80032
:100B30003322AF00FEFF3700A011880040002000E4
:100B40000008E600F6FF3700050078008600780010
:100B500084002000526B0200000000003322AF002E
:100B6000FEFF370004022000A41188004ECEBF0013
:100B70000160EF004200DD00A4D620000400400028
:100B8000900278001003900001002000010078001E
:100B900090370200000000008100E8003322AF001F
:100BA000FEFF3700A0118800400020000008E6008A
:100BB000F6FF3700050078008600780084002000EA
:100BC000526B0200000000003322AF00FEFF37002E
:100BD00004022000A41188004ECEBF000160EF0087
:100BE0004200DD0064DD2000040040009002780037
:100BF000100390000100200001007800A8370200D7
:100C0000000000008100E8003322AF00FEFF370043
:100C1000A0118800500020000008E600F6FF370011
:100C2000050078008600780004002000526B020066
:100C3000000000003322AF00FEFF37000402200056
:100C4000A41188003322AF00FEFF3700A40020006B
:100C5000A41188003322AF00FEFF3700D40020002B
:100C6000A41188004E6EEC0074FF3700BE2EAE005B
:100C700010003700F45580004822DE006124E100B6
:100C80000C003A00E45480004822DE006124E100B8
:100C900008003A0010C0B30062F2B70054A202008C
:100CA000000000002475EF003EA1020000000000DB
:100CB0000200370020C0B300BFEAB70097C0A80009
:100CC0004220EF0028C8BF002948E300030032009B
:100CD000C4AC020000000000FAFF37000200200050
:100CE000E1822000020078000428020000000000D9
:100CF000805878000201E8000004E0004220AE00C5
:100D0000F8FF37002C68EF002868EF002968EF0033
:100D1000A6E40200000000000500200005007800A5
:100D2000C0370200000000000040B3004220AF00C6
:100D3000060037008502E8003322AF00FEFF3700CF
:100D400034E2B7003562EF00F4FF37005628EC00BC
:100D50004220AF005828EC0097C0A8004220EF00C6
:100D600028C8BF002948E30003003200C4AC0200D9
:100D700000000000FAFF370066E5020000000000F6
:100D8000947280006224E1000C003A00F455800067
:100D90004822DE006324E1000800320020C0B300D6
:100DA00024F5B7008CB6020000000000534EE200AC
:100DB00002003200F2C00200000000002E3D0200DE
:100DC00000000000804278000040EB000A40AF00C5
:100DD0000000E8006104E10006003A00F4558000DC
:100DE0004822DE006324E10002003200A6E4020093
:100DF0000000000097C0A900040E20001402880023
:100E0000C44280006020E1000F03390003003E006F
:100E1000B44280006A20E1000B033900F4558000E1
:100E20004822DE006124E10002003A00040337009A
:100E300005003700F45580004822DE006324E100FD
:100E400001003A00FE023700505E02000000000080
:100E5000F0C7B3005FF6B700A0C0B30060F6B700FC
:100E60000442020000000000082BEF00F4FF200005
:100E700034588800C48080004822DE006124E100EC
:100E80000D003A000500200005007800D837020068
:100E9000000000000040B3004220AF000500370012
:100EA0008502E80062F6B700BA45020000000000C3
:100EB000F5FF37002D003700248080004822DE0037
:100EC0006124E1001D003A00C48080006124E1003B
:100ED0000D003A000500200005007800E837020008
:100EE000000000000040B3004220AF0005003700C2
:100EF0008502E80062F6B700BA4502000000000073
:100F0000F5FF37000C0037000500200005007800D1
:100F1000F8370200000000000040B3004220AF009C
:100F2000050037008502E80062F6B700BA45020006
:100F300000000000F5FF37000C003700050020001E
:100F40000500780008380200000000000040B300EF
:100F50004220AF00050037008502E80062F6B700C6
:100F6000BA45020000000000F5FF370020C0B300C2
:100F70000AEBB70020C0B3000BEBB7005F76EF00C1
:100F800020C0B30060F6B700044202000000000079
:100F900004C0200044588800F4FF20003458880022
:100FA000E10121001104E00008003200811F7800F7
:100FB0001140780062F6B700BA4502000000000058
:100FC000CF0078008100E800F6FF370010C0B300C2
:100FD0000AEBB70010C0B3000BEBB70040C9B30079
:100FE0005FF6B700A0C0B30060F6B700044202008D
:100FF00000000000082BEF00444420003458880013
:10100000F9CFBF00800278000B60EF0006002000DF
:10101000050078008600780014002800729E020007
:101020000000000040C6B3005FF6B700A0C0B300E8
:1010300060F6B7000442020000000000082BEF0039
:10104000F4FF200034588800908080004170220016
:101050006464020000000000849280004822DE00E8
:101060006124E1005C003A002D08AF005A0037000F
:101070005F76EF0030C1B30060F6B70004420200B3
:1010800000000000082BEF0004882000345888007E
:10109000759280008502FB000003EB0005F0A700BD
:1010A0000083EB000500780086007800140028001B
:1010B000729E020000000000A0C3B30062F6B700F9
:1010C000BA450200000000004FD2BF008002780045
:1010D0008502FB000003EB0005F0A7000083EB0096
:1010E000050078008600780014002800729E020037
:1010F0000000000000C2B30062F6B700BA4502006B
:101100000000000000C2B30062F6B700BA4502005A
:1011100000000000212521001104E0000800320039
:10112000811F78001140780062F6B700BA450200CE
:1011300000000000CF0078008100E800F6FF3700D3
:1011400000C2B30062F6B700BA450200000000001A
:10115000612521001104E00008003200811F7800A1
:101160001140780062F6B700BA45020000000000A6
:10117000CF0078008100E800F6FF370000C2B3001E
:1011800062F6B700BA45020000000000F09180004E
:101190000192800014002800729E020000000000EE
:1011A000C0C2B30062F6B700BA45020000000000FA
:1011B00090918000A191800044002000729E020066
:1011C0000000000000C2B30062F6B700BA4502009A
:1011D000000000005172EF001950E20002003200DE
:1011E0009D4AE20016023A008402210004B38800FE
:1011F000989D0200000000006204E10007003E002C
:10120000A40A210004B38800989D02000000000099
:101210006204E10001003E0006023700AA2AEF0046
:10122000545580000484B20016003200840221006C
:10123000535580000480410010407800004FB200F8
:101240000004E0000D003A00AA0AF800AC0AF90018
:10125000645580000484B20007003200840221003B
:10126000635580008482410000C2B300804A780048
:10127000AC2AEC00F6FF37006870EF00AA2AEC00F9
:10128000E7FF3700AA2AEF00545580000484B2001B
:1012900016003200A40A210053558000048041004A
:1012A00010407800004FB2000004E0000D003A004A
:1012B000AA0AF800AC0AF900645580000484B20060
:1012C00007003200A40A2100635580008482410097
:1012D00000C2B300804A7800AC2AEC00F6FF370069
:1012E000EA70EF00AA2AEC00E7FF37002C71EF004C
:1012F0006871EF00A471EF00E071EF004A71EF0038
:101300008671EF00C271EF00FE71EF00082BEF0055
:1013100004FF200034588800A401200034558800C0
:10132000A60AE20013003200840221003355800037
:10133000048041001042780004C2B2000B003A0061
:10134000A6CABF002BF5B700C412210064A988000B
:101350008402210074A98800609D02000000000042
:10136000A60AF8009E0AF90002003700A62AED003E
:10137000EBFF37009E0AF800A80AF90044558000E8
:101380007A20E10007003200C4122100435580009A
:101390008482410000C2B300804A7800A82AEC0091
:1013A000F6FF37004671EF005F76EF0020C3B30011
:1013B00060F6B7000442020000000000C1122100E4
:1013C0001104E00008003200811F7800114078000D
:1013D00062F6B700BA45020000000000CF007800B6
:1013E0008100E800F6FF3700F45480007A024200E2
:1013F00034558800305580009E0AE3001500320005
:10140000840221003355800004804100104278009E
:1014100004C2B2000D003A00800221009E0AB4000E
:1014200080027800A6CABF002BF5B7008416210001
:1014300064A9880075A98800609D02000000000072
:10144000A60AF800A00AF90002003700A62AED005B
:10145000E8FF370004558000F35480000300520079
:1014600040558800445580007A20E1000700320092
:1014700084162100435580008482410000C2B300DD
:10148000804A7800A82AEC00F6FF37008271EF004E
:101490005F76EF00C0C3B30060F6B70004420200FD
:1014A00000000000811621001104E0000800320055
:1014B000811F78001140780062F6B700BA4502003B
:1014C00000000000CF0078008100E800F6FF370040
:1014D000045580007A02420034558800305580005F
:1014E000A00AE30015003200840221003355800079
:1014F000048041001042780004C2B2000D003A009E
:1015000080022100A00AB40080027800A6CABF00B1
:101510002BF5B700441A210064A9880075A988003A
:10152000609D020000000000A60AF800A20AF9006F
:1015300002003700A62AED00E8FF370014558000AE
:101540000355800003005200405588004455800038
:101550007A20E10007003200441A21004355800040
:101560008482410000C2B300804A7800A82AEC00BF
:10157000F6FF3700BE71EF005F76EF0060C4B30086
:1015800060F6B7000442020000000000411A21008A
:101590001104E00008003200811F7800114078003B
:1015A00062F6B700BA45020000000000CF007800E4
:1015B0008100E800F6FF3700145580007A024200EF
:1015C0003455880030558000A20AE300150032002F
:1015D00084022100335580000480410010427800CD
:1015E00004C2B2000D003A0080022100A20AB40039
:1015F00080027800A6CABF002BF5B700041E2100A8
:1016000064A9880075A98800609D020000000000A0
:10161000A60AF800A40AF90002003700A62AED0085
:10162000E8FF370024558000135580000300520066
:1016300040558800445580007A20E10007003200C0
:10164000041E2100435580008482410000C2B30083
:10165000804A7800A82AEC00F6FF3700FA71EF0004
:101660005F76EF0000C5B30060F6B70004420200E9
:1016700000000000011E21001104E00008003200FB
:10168000811F78001140780062F6B700BA45020069
:1016900000000000CF0078008100E800F6FF37006E
:1016A000082BEF00F400200034588800A40120002B
:1016B00034558800A60AE20013003200A40A210073
:1016C00033558000048041001042780004C2B2000B
:1016D0000B003A00A6CABF002BF5B700A4142100E6
:1016E00064A98800A40A210074A98800609D0200F2
:1016F00000000000A60AF8009E0AF9000200370068
:10170000A62AED00EBFF37009E0AF800A80AF900B0
:10171000445580007A20E10007003200A414210023
:10172000435580008482410000C2B300804A7800A3
:10173000A82AEC00F6FF37006471EF005F76EF0037
:10174000A0C5B30060F6B70004420200000000002C
:10175000A11421001104E00008003200811F78006C
:101760001140780062F6B700BA45020000000000A0
:10177000CF0078008100E800F6FF3700F4548000C5
:101780007A02420034558800305580009E0AE300FA
:1017900015003200A40A2100335580000480410066
:1017A0001042780004C2B2000D003A00A00A2100E5
:1017B0009E0AB40080027800A6CABF002BF5B700CD
:1017C0006418210064A9880075A98800609D020042
:1017D00000000000A60AF800A00AF9000200370085
:1017E000A62AED00E8FF370004558000F35480007E
:1017F0000300520040558800445580007A20E100E3
:1018000007003200641821004355800084824100A3
:1018100000C2B300804A7800A82AEC00F6FF370027
:10182000A071EF005F76EF0040C6B30060F6B7002E
:101830000442020000000000611821001104E000D1
:1018400008003200811F78001140780062F6B7006E
:10185000BA45020000000000CF0078008100E800D7
:10186000F6FF3700045580007A02420034558800A4
:1018700030558000A00AE30015003200A40A2100C0
:1018800033558000048041001042780004C2B20049
:101890000D003A00A00A2100A00AB40080027800DE
:1018A000A6CABF002BF5B700241C210064A988003C
:1018B00075A98800609D020000000000A60AF800DB
:1018C000A20AF90002003700A62AED00E8FF37005F
:1018D00014558000035580000300520040558800D5
:1018E000445580007A20E10007003200241C2100CA
:1018F000435580008482410000C2B300804A7800D2
:10190000A82AEC00F6FF3700DC71EF005F76EF00ED
:10191000E0C6B30060F6B700044202000000000019
:10192000211C21001104E00008003200811F780012
:101930001140780062F6B700BA45020000000000CE
:10194000CF0078008100E800F6FF370014558000D2
:101950007A0242003455880030558000A20AE30024
:1019600015003200A40A2100335580000480410094
:101970001042780004C2B2000D003A00A00A210013
:10198000A20AB40080027800A6CABF002BF5B700F7
:10199000E41F210064A9880075A98800609D0200E9
:1019A00000000000A60AF800A40AF90002003700AF
:1019B000A62AED00E8FF370024558000135580006B
:1019C0000300520040558800445580007A20E10011
:1019D00007003200E41F210043558000848241004B
:1019E00000C2B300804A7800A82AEC00F6FF370056
:1019F0001872EF005F76EF0080C7B30060F6B700A3
:101A00000442020000000000E11F21001104E00078
:101A100008003200811F78001140780062F6B7009C
:101A2000BA45020000000000CF0078008100E80005
:101A3000F6FF3700082BEF00F4FF20003458880031
:101A40005628EF005828EF00C48080004822DE00AE
:101A50006124E100BC003A00E45480004822DE002A
:101A60006124E100B8003A00F45580004822DE000D
:101A70006324E10002003200B6EB02000000000027
:101A8000F45580004822DE006124E10002003A00A3
:101A9000AC00370005003700F45580004822DE0016
:101AA0006324E10001003A00A6003700D45580000D
:101AB000431F20000418E10005003900D4558000C0
:101AC00061024200D45588009000370001003700C1
:101AD000BA2AEF00FEEC020000000000B4EAB700F2
:101AE000B56AEF00B40AE2004B003A00C0C1B3008F
:101AF0005DF6B700D05F02000000000040C2B300F6
:101B00005DF6B700D05F020000000000A0C2B30085
:101B10005DF6B700D05F02000000000020C3B300F4
:101B20005DF6B700D05F020000000000A0C3B30064
:101B30005DF6B700D05F02000000000020C4B300D3
:101B40005DF6B700D05F020000000000A0C4B30043
:101B50005DF6B700D05F02000000000020C5B300B2
:101B60005DF6B700D05F020000000000A0C5B30022
:101B70005DF6B700D05F02000000000020C6B30091
:101B80005DF6B700D05F020000000000A0C6B30001
:101B90005DF6B700D05F02000000000020C7B30070
:101BA0005DF6B700D05F020000000000A0C7B300E0
:101BB0005DF6B700D05F0200000000005F76EF0026
:101BC000C0C1B30060F6B70004420200000000008C
:101BD000082BEF008488200034588800534EE20020
:101BE0000C003A00050020000500780018380200BB
:101BF000000000000040B3004220AF0005003700A5
:101C00008502E80062F6B700BA4502000000000055
:101C1000F5FF37003D003700A0558000C455800017
:101C20000020E10001003900B82AEF005F76EF00E4
:101C3000C0C1B30060F6B70004420200000000001B
:101C40000500200005007800343802000000000084
:101C50000040B3004220AF00050037008502E800D5
:101C600062F6B700BA45020000000000F5FF370039
:101C70005F76EF00C0C1B30060F6B7000442020017
:101C800000000000082BEF008488200034588800F2
:101C9000C555800006002000E182420085037800DF
:101CA00060034B0006047800070078008800780085
:101CB00004002000729E020000000000A555800074
:101CC00006002000F0C2B30062F6B700BA45020079
:101CD0000000000005007800860078000400200065
:101CE000729E020000000000B8CABF0024F5B700D1
:101CF00010C0B30025F5B700CEB802000000000008
:101D0000C455800061024200C455880010C0B30071
:101D100050F5B700F40A200094AA88005435EF006B
:101D20005635EF00040A2000C4AA8800640220008F
:101D3000D4AA880064022000E4AA88008C8B0200E8
:101D4000000000000000000000FC37000040FE0022
:0C4004003220EF00030A2000830150006E
:1040100005003100E3012200008041001040BA0099
:104020000160EF0000000600F001220083814100E2
:10403000808141001380BA000000060000003200B9
:104040000000490000007900005F410000003E00D0
:1040500000077E0000071100001411007F141100FA
:104060007F147E00242A7F007F2A49001223490002
:10407000130849006462360036493E00552241006B
:10408000500041000503410000002200001C7F0099
:104090002241410000004100412222001C001C007E
:1040A00014087F003E08490014084900083E4900F2
:1040B0000808410000507F00300009000008090096
:1040C000080809000808010000603E006000410087
:1040D000002049001008490004027A003E517F0088
:1040E000494508003E000800427F080040007F006C
:1040F000426100005149410046217F004145410095
:104100004B31000018142000127F4000102741009E
:1041100045453F00453901003C4A7F0049490800B8
:1041200030011400710922000503410036497F0067
:10413000494940003606400049494000291E4000D8
:1041400000367F003600020000000C0056360200E8
:1041500000007F0008147F002241040000140800C2
:104160001414100014147F0000413E00221441007A
:10417000080241000151410009063E003220EF00D3
:10418000030A20008301500005003100A30D220026
:10419000008041001040BA000160EF0000000600FE
:1041A000B00D220083814100808141001380BA005C
:1041B000000006007F097C0009091400063E140077
:1041C00041511400215E08007F09080019291400DC
:1041D000464614004949180049317C0001017C0021
:1041E0007F010800013F040040400400403F0800F8
:1041F0001F204800402054001F3F54004038540006
:10420000403F20006314040008143F00630744008B
:10421000087040000807200061513C0049454000FB
:10422000430040007F41200041007C0002041C004C
:104230000810200020004000414120007F001C00A9
:1042400004023C00010240000440300040404000B5
:1042500040403C00000144000204280000201000FF
:1042600054542800547844007F480C0044445000C3
:10427000383850004444500044203C003844440046
:10428000444864007F38540054544C00541844008F
:10429000087E000009010800020C3600525241005D
:1042A000523E00007F0800000404000078007F00F8
:1042B000447D00004000000020400000443D4100DB
:1042C000007F360010280800440000000041100064
:1042D0007F400800007C08000418100004780800E3
:1042E0007C087800040446007838410044444600C5
:1042F000443878003220EF0023082000830150006A
:104300000500310063192200008041001040BA000E
:104310000160EF0000000600701922008381410057
:10432000808141001380BA00000006001E213C007D
:1043300061214100123C400041404100217C3C0091
:104340003854000056550000182000005555000054
:1043500055780000205520005455480078203E0034
:10436000555649005478620020540000555400000E
:10437000781C000022620000221000003855000066
:10438000555500001838000055540000551800001D
:10439000385440005556680018003E00457C09001E
:1043A00041000200004520007D41540000005600FD
:1043B000457E550040007800781500001415440033
:1043C00078787E0014154100147800007C54380081
:1043D000565544004424460054784500544838005B
:1043E0007E093C007E494000493842004545210095
:1043F00045387C0038457C004445090038380500C4
:1044000045460500443878003C417C0041210900C4
:104410007C3C110041422100207C7C000C517E003C
:10442000505125003C3825004544260045381800E9
:104430003220EF00630320008301500004003100AC
:1044400083232200008041001000BA000000060013
:104450009023220083814100808141003380BA0093
:104460009381BA00C819DD000080710000000600C9
:104470000F0000000F0000000F000F000F000000F1
:104480000F000F000F0000000F000F000F000000D2
:104490000F000F000000000000000F0000000000EF
:1044A0000F000F000F0000000F000F000F000000B2
:1044B0000F000F0000000000000000000F000000CF
:1044C0000F000F000F0000000F000F000F00000092
:1044D0000F000F00000000000F0000003220EF006E
:1044E000630320008301500004003100E328220010
:1044F000008041001000BA0000000600F0282200F1
:1045000083814100808141003380BA009381BA00E9
:10451000C819DD000080710000000600F0000000F6
:10452000F0000000F000000000000000F000F000CB
:10453000F0000000F000F000F0000000F000F000DB
:10454000F00000000000F000F0000000F000F000BB
:10455000F0000000F000F000F0000000F000F000BB
:10456000000000000000F000F0000000F00000007B
:10457000F0000000F0000000F0000000F000F0008B
:10458000F0000000F00000003220EF006303200084
:104590008301500004003100432E220000804100BE
:1045A0001000BA0000000600502E22008381410056
:1045B000808141003380BA009381BA00C819DD00C0
:1045C0000080710000000600FF0FFF00000F0F00C9
:1045D000FF0F0000000F0F00FF0FFF00000F0F0084
:1045E000FF0F0000000F0F00000FFF00FF0F0F0074
:1045F000000FFF00FF0F0F00000F0000FF0F0F0064
:10460000000FFF00FF0F0F00FF0F0000000F0F0053
:10461000FF0FFF00000F0F00FF0F0000000F0F0043
:10462000FF0FFF00000F0F00000F0000FF0F0F0033
:10463000000F00003220EF006303200083015000D0
:1046400004003100A3332200008041001000BA00B2
:1046500000000600B03322008381410080814100C8
:104660003380BA009381BA00C819DD000080710060
:1046700000000600000F0000000F0F00000F0000F8
:10468000000F0F00000F0000000F0F00000F0000D0
:10469000000F0F00000F0000000F0F00000F0000C0
:1046A000000F0F00000F0000000F0F00000F0000B0
:1046B000000F0F00000F0000000F0F00FF0F0000A1
:1046C000000F0F00FF0F0000FF0F0F00FF0F000093
:1046D000000F0F00000F0000000F0F00000F000080
:1046E0003220EF00C3372200008041001040BA00A2
:1046F0000160EF0000000600202A00002A7300007D
:1047000069200000706F00007765000072200000D3
:10471000757000002A2A0000200000003220EF00FF
:10472000A3392200008041001040BA000160EF0070
:10473000000006002A0000003220EF00833A220029
:10474000008041001040BA000160EF000000060048
:10475000202A00002A730000692000007475000000
:104760006E6500002A2A0000200000003220EF00C1
:10477000233C2200008041001040BA000160EF009D
:104780000000060073740000000000003220EF00FB
:10479000233D2200008041001040BA000160EF007C
:1047A000000006006D6F0000000000003220EF00E6
:1047B000233E2200008041001040BA000160EF005B
:1047C000000006004E6F00002043000061720000F0
:1047D00064200000466F0000756E00006421000038
:1047E000200000003220EF00E33F22000080410063
:1047F0001040BA000160EF000000060020630000D6
:1048000061720000643F0000200000003220EF00D1
:1048100023412200008041001040BA000160EF00F7
:10482000000006004361000072640000203F0000A9
:104830002020000020200000202000002000000098
:104840003220EF00C3422200008041001040BA0035
:104850000160EF0000000600616300006D6400006D
:10486000383D000025780000200000003220EF00D5
:1048700023442200008041001040BA000160EF0094
:104880000000060043610000726400002042000046
:104890006F6F0000742E00002E2E0000000000003C
:1048A0003220EF00C3452200008041001040BA00D2
:1048B0000160EF00000006007374000061740000E6
:1048C000313D0000202500004C7800002000000051
:1048D0003220EF0043472200008041001040BA0020
:1048E0000160EF00000006007374000061740000B6
:1048F000323D0000202500004C7800002000000020
:104900003220EF00C3482200008041001040BA006E
:104910000160EF000000060053440000484300001F
:104920003D20000025780000200000003220EF002C
:10493000234A2200008041001040BA000160EF00CD
:104940000000060020200000534400002042000028
:104950006F6F0000742E00002E2E0000000000007B
:104960003220EF00C34B2200008041001040BA000B
:104970000160EF00000006005344000048430000BF
:10498000204200006F6F0000742E00002E2E0000E9
:10499000000000003220EF00634D22000080410043
:1049A0001040BA000160EF000000060073740000C0
:1049B00061740000333D0000202500006C78000089
:1049C000200000003220EF00E34E22000080410072
:1049D0001040BA000160EF000000060061630000B3
:1049E0006D640000343100003D2000002578000097
:1049F000200000003220EF006350220000804100C0
:104A00001040BA000160EF00000006004D4D0000AC
:104A1000432000004D4F00004445000020000000EE
:104A20003220EF00C3512200008041001040BA0044
:104A30000160EF0000000600204D00004D43000023
:104A4000204200006F6F0000740000003220EF0071
:104A500023532200008041001040BA000160EF00A3
:104A6000000006000A0D00002072000065610000D1
:104A7000645F0000626F00006F740000207300002C
:104A80007461000072740000696E0000672000000D
:104A90000A0D0000000000003220EF0083552200C4
:104AA000008041001040BA000160EF0000000600E5
:104AB0005365000063560000423D0000254C000095
:104AC000782000000A0D0000000000003220EF00F6
:104AD00023572200008041001040BA000160EF001F
:104AE000000006004270000053650000633D0000B6
:104AF000202500004C780000200A00000D00000076
:104B00003220EF00C3582200008041001040BA005C
:104B10000160EF00000006005365000063700000B4
:104B2000436C0000753D0000202500004C7800001B
:104B3000200A00000D0000003220EF00835A2200FE
:104B4000008041001040BA000160EF000000060044
:104B500052530000656300003D200000254C00001A
:104B6000782000000A0D0000000000003220EF0055
:104B7000235C2200008041001040BA000160EF0079
:104B80000000060046610000744E00003D20000059
:104B9000254C0000782000000A0D000000000000F5
:104BA0003220EF00C35D2200008041001040BA00B7
:104BB0000160EF000000060053650000634600003E
:104BC00061740000313D0000202500004C78000099
:104BD000200A00000D0000003220EF00835F220059
:104BE000008041001040BA000160EF0000000600A4
:104BF00046410000543100005F6C0000626100001B
:104C00005F73000074610000727400003D200000BA
:104C1000254C0000782000000A0D00000000000074
:104C20003220EF00C3612200008041001040BA0032
:104C30000160EF00000006005370000046610000B4
:104C4000743D0000202500004C780000200A000080
:104C50000D0000003220EF0063632200008041005D
:104C60001040BA000160EF0000000600524400004E
:104C700069720000456E0000744E00003D20000087
:104C8000254C0000782000000A0D00000000000004
:104C90003220EF0043652200008041001040BA003E
:104CA0000160EF00000006002046000041540000B3
:104CB000313600002C200000000000003220EF0000
:104CC000A3662200008041001040BA000160EF009E
:104CD0000000060053650000635200006F6F000083
:104CE00074440000697200003D2500004C7800000B
:104CF000200A00000D0000003220EF00836822002F
:104D0000008041001040BA000160EF000000060082
:104D1000456E00006453000065630000526F0000A0
:104D20006F74000044690000723D0000254C0000D3
:104D3000782000000A0D0000000000003220EF0083
:104D4000A36A2200008041001040BA000160EF0019
:104D5000000006005365000063700000464100003B
:104D600054330000323D0000254C00007820000044
:104D70000A0D0000000000003220EF00836C2200CA
:104D8000008041001040BA000160EF000000060002
:104D9000436C0000755200006F6F00007444000007
:104DA000697200005F460000415400003332000089
:104DB0003D2500004C780000200A00000D00000096
:104DC0003220EF00C36E2200008041001040BA0084
:104DD0000160EF00000006006C62000061520000FC
:104DE0006F6F000074440000697200003D250000F0
:104DF0004C780000200A00000D0000003220EF0077
:104E0000A3702200008041001040BA000160EF0052
:104E10000000060021210000204200007053000025
:104E20006563000020690000732000006E6F0000C1
:104E300074200000353100003220000021210000E4
:104E4000200A00000D0000003220EF000373220052
:104E5000008041001040BA000160EF000000060031
:104E60006363000073300000310000003220EF0067
:104E700023742200008041001040BA000160EF005E
:104E800000000600202A000043430000462A0000DC
:104E9000200000003220EF006375220000804100F6
:104EA0001040BA000160EF000000060053630000EC
:104EB000616E00006E6900006E6700002E2E00001B
:104EC0002E0000003220EF00E37622000080410037
:104ED0001040BA000160EF000000060063630000AC
:104EE00073300000320000003220EF00037822000F
:104EF000008041001040BA000160EF000000060091
:104F00002A2A0000736500006373000063610000DB
:104F10006E3D0000254C00007820000000000000DD
:104F20003220EF00C3792200008041001040BA0017
:104F30000160EF0000000600726F00007773000050
:104F4000636100006E3D0000254C000078200000E9
:104F5000000000003220EF00637B2200008041004F
:104F60001040BA000160EF0000000600726F000000
:104F700077730000636100006E3100003D25000082
:104F80004C780000200000003220EF00037D22005A
:104F9000008041001040BA000160EF0000000600F0
:104FA000726F000077730000636100006E320000D2
:104FB0003D2500004C7800000A0D000000000000B4
:104FC0003220EF00C37E2200008041001040BA0072
:104FD0000160EF0000000600444500004C20000086
:104FE000000000003220EF00E37F2200008041003B
:104FF0001040BA000160EF00000006004C460000BF
:105000004E200000000000003220EF00038122004B
:10501000008041001040BA000160EF00000006006F
:10502000000000003220EF00E381220000804100F8
:105030001040BA000160EF0000000600202A0000C6
:105040002A2A00002A250000732A00002A2A0000CC
:105050002A2000000A0D0000000000003220EF00AE
:10506000A3832200008041001040BA000160EF00DD
:105070000000060064690000725F0000703D0000DF
:105080002575000020200000000000003220EF0005
:1050900023852200008041001040BA000160EF002B
:1050A00000000600202A0000303100002A20000005
:1050B000000000003220EF006386220000804100E3
:1050C0001040BA000160EF0000000600202A000036
:1050D000303300002A200000000000003220EF00E2
:1050E000A3872200008041001040BA000160EF0059
:1050F00000000600726F00006F74000020000000C6
:105100003220EF00C3882200008041001040BA0026
:105110000160EF0000000600202A0000303400008B
:105120002A200000000000003220EF00038A220045
:10513000008041001040BA000160EF00000006004E
:10514000202A0000303500002A2000000000000066
:105150003220EF00438B2200008041001040BA0053
:105160000160EF0000000600636300007330000080
:10517000330000003220EF00638C220000804100E9
:105180001040BA000160EF00000006004469000012
:10519000724300006C750000733D0000253800006C
:1051A0006C780000200A00000D0000003220EF00A3
:1051B000238E2200008041001040BA000160EF0001
:1051C00000000600454E00004431000020000000B1
:1051D0003220EF00438F2200008041001040BA00CF
:1051E0000160EF0000000600454E00004432000060
:1051F000200000003220EF00639022000080410078
:105200001040BA000160EF00000006006E6500006B
:1052100078740000436C0000757300007465000032
:10522000723D0000254C0000782000000A0D0000AF
:10523000000000003220EF00639222000080410055
:105240001040BA000160EF00000006002046000098
:1052500041540000333200002C2000000000000008
:105260003220EF00C3932200008041001040BA00BA
:105270000160EF000000060063630000323D0000A3
:10528000256C0000782000000A0D000000000000DE
:105290003220EF0043952200008041001040BA0008
:1052A0000160EF0000000600202A00006672000086
:1052B000616700003D200000257800002A200000E2
:1052C0000A0D0000000000003220EF0003972200CA
:1052D000008041001040BA000160EF0000000600AD
:1052E0000A0D0000000000003220EF0003982200A9
:1052F000008041001040BA000160EF00000006008D
:105300007374000061720000742000006672000077
:10531000616D00005F6200006C6100006E6B000058
:1053200020300000000000003220EF00039A22002D
:10533000008041001040BA000160EF00000006004C
:105340007374000061720000742000006672000037
:10535000616D00005F6200006C6100006E6B000018
:1053600020310000000000003220EF00039C2200EA
:10537000008041001040BA000160EF00000006000C
:105380002021000031200000000000003220EF004A
:10539000239D2200008041001040BA000160EF0010
:1053A0000000060020210000322000000000000064
:1053B0003220EF00439E2200008041001040BA00DE
:1053C0000160EF00000006000A0D0000200A000046
:1053D0000D0000003220EF00639F2200008041009A
:1053E0001040BA000160EF00000006000A0D000046
:1053F0002A2A00002070000061670000653D00005F
:1054000025750000200000003220EF0003A12200DB
:10541000008041001040BA000160EF00000006006B
:1054200061630000743D000025750000200000004D
:105430003220EF0043A22200008041001040BA0059
:105440000160EF00000006006C6F0000633D00008B
:10545000254C000075200000000000003220EF0005
:10546000A3A32200008041001040BA000160EF00B9
:105470000000060064690000723D00002575000010
:10548000200000003220EF00E3A422000080410051
:105490001040BA000160EF000000060065780000CF
:1054A000743D000025750000200000003220EF0050
:1054B00023A62200008041001040BA000160EF00E6
:1054C0000000060065760000743D0000254C0000D9
:1054D00075200000000000003220EF0083A72200AA
:1054E000008041001040BA000160EF00000006009B
:1054F00065760000746300006C7200003D000000DF
:105500003220EF00C3A82200008041001040BA0002
:105510000160EF0000000600202A00002A2A000097
:10552000200000003220EF00E3A9220000804100AB
:105530001040BA000160EF000000060020000000EB
:105540003220EF00C3AA2200008041001040BA00C0
:105550000160EF0000000600202D00003E2000004A
:10556000000000003220EF00E3AB22000080410089
:105570001040BA000160EF0000000600202A000081
:1055800065760000745F0000636F00006C6F0000C0
:10559000757200003D25000075200000000000002D
:1055A0003220EF00C3AD2200008041001040BA005D
:1055B0000160EF00000006004C3D0000000000000C
:1055C0003220EF00C3AE2200008041001040BA003C
:1055D0000160EF0000000600443D000000000000F4
:1055E0003220EF00C3AF2200008041001040BA001B
:1055F0000160EF000000060045580000543D000027
:10560000000000003220EF00E3B0220000804100E3
:105610001040BA000160EF0000000600455600008F
:10562000543D0000000000003220EF0003B22200D1
:10563000008041001040BA000160EF000000060049
:10564000203F0000544900004D4500003F2000006D
:10565000000000003220EF0063B322000080410010
:105660001040BA000160EF0000000600206A000050
:10567000257500003A7400006D3D0000257500009E
:10568000200000003220EF00E3B42200008041003F
:105690001040BA000160EF00000006002021000069
:1056A0002121000021200000544900004D45000048
:1056B0004F550000542000002575000020210000F7
:1056C0002121000021200000000000003220EF0016
:1056D00023B72200008041001040BA000160EF00B3
:1056E00000000600202000002020000020200000F4
:1056F000200000003220EF0063B82200008041004B
:105700001040BA000160EF000000060020520000C7
:1057100045430000200000003220EF0083B9220042
:10572000008041001040BA000160EF000000060058
:10573000202A00002A660000726100006D3000001F
:10574000312A00002A200000000000003220EF0073
:1057500023BB2200008041001040BA000160EF002E
:10576000000006000A0D0000205400004D43000018
:10577000206900006E690000743A000020430000B8
:10578000433D000025780000204C0000544E0000EE
:105790003D250000782000000A0D000000000000F8
:1057A0003220EF00C3BD2200008041001040BA004B
:1057B0000160EF0000000600546F000074610000FB
:1057C0006C200000466900006C650000733D00001D
:1057D00020250000346C0000752000000A0D000038
:1057E000000000003220EF00E3BF220000804100F3
:1057F0001040BA000160EF0000000600646900007C
:10580000725F00006E7500006D620000657200003E
:10581000202500004C7800003D2000000000000022
:105820003220EF00C3C12200008041001040BA00C6
:105830000160EF0000000600746F0000746100005A
:105840006C64000069720000733D000020250000B8
:105850004C780000200A00000D0000003220EF000C
:10586000A3C32200008041001040BA000160EF0095
:1058700000000600202A00002A7400006D6300006A
:105880005F630000635F00006C7400006E20000026
:10589000303100002A2A0000000000003220EF0012
:1058A000A3C52200008041001040BA000160EF0053
:1058B000000006000A0D000020430000433D0000E8
:1058C00025780000204C0000544E00003D250000CB
:1058D000782000000A0D0000000000003220EF00D8
:1058E000A3C72200008041001040BA000160EF0011
:1058F000000006000A0D000020430000435F000086
:10590000766100006C3D000025780000204C00000E
:10591000544E00005F760000616C00003D250000E1
:10592000782000000A0D0000000000003220EF0087
:1059300023CA2200008041001040BA000160EF003D
:1059400000000600434300003D0000003220EF004D
:1059500023CB2200008041001040BA000160EF001C
:10596000000006004C5400004E3D00000000000006
:105970003220EF0043CC2200008041001040BA00EA
:105980000160EF0000000600202A00002A740000D9
:105990006D6300005F630000635F00006C740000D3
:1059A0006E200000303200002A2A000000000000B3
:1059B0003220EF0043CE2200008041001040BA00A8
:1059C0000160EF0000000600202A00002A74000099
:1059D0006D6300005F6300006F7500006E7400006F
:1059E000727900002A2A0000000000003220EF0037
:1059F00023D02200008041001040BA000160EF0077
:105A00000000060041540000000000003220EF00BA
:105A100023D12200008041001040BA000160EF0055
:105A20000000060042450000000000003220EF00A8
:105A300023D22200008041001040BA000160EF0034
:105A400000000600434E0000000000003220EF007E
:105A500023D32200008041001040BA000160EF0013
:105A600000000600435A0000000000003220EF0052
:105A700023D42200008041001040BA000160EF00F2
:105A80000000060044550000000000003220EF0036
:105A900023D52200008041001040BA000160EF00D1
:105AA00000000600444B0000000000003220EF0020
:105AB00023D62200008041001040BA000160EF00B0
:105AC0000000060046490000000000003220EF0000
:105AD00023D72200008041001040BA000160EF008F
:105AE0000000060046520000000000003220EF00D7
:105AF00023D82200008041001040BA000160EF006E
:105B00000000060044450000000000003220EF00C5
:105B100023D92200008041001040BA000160EF004C
:105B20000000060049540000000000003220EF0091
:105B300023DA2200008041001040BA000160EF002B
:105B4000000006004E4C0000000000003220EF0074
:105B500023DB2200008041001040BA000160EF000A
:105B6000000006004E4F0000000000003220EF0051
:105B700023DC2200008041001040BA000160EF00E9
:105B80000000060045530000000000003220EF0036
:105B900023DD2200008041001040BA000160EF00C8
:105BA0000000060053450000000000003220EF0016
:105BB00023DE2200008041001040BA000160EF00A7
:105BC0000000060043480000000000003220EF0003
:105BD00023DF2200008041001040BA000160EF0086
:105BE00000000600554B0000000000003220EF00CE
:105BF00023E02200008041001040BA000160EF0065
:105C000000000600202A00002A2A0000415400005B
:105C10002D4100005553000054520000494100003E
:105C20002A2A00002A200000000000003220EF0095
:105C300023E22200008041001040BA000160EF0022
:105C400000000600202A00002A2A00004245000029
:105C50002D420000454C000047490000554D000012
:105C60002A2A00002A200000000000003220EF0055
:105C700023E42200008041001040BA000160EF00E0
:105C800000000600202A00002A2A0000434E0000DF
:105C90002D430000484900004E4100002A2A000020
:105CA0002A200000000000003220EF0003E622005E
:105CB000008041001040BA000160EF0000000600C3
:105CC000202A00002A2A0000435A00002D43000029
:105CD0005A45000043480000494100002A2A0000BC
:105CE0002A200000000000003220EF0003E822001C
:105CF000008041001040BA000160EF000000060083
:105D0000202A00002A2A0000445500002D440000EB
:105D100055420000414900002A2A00002A200000C4
:105D2000000000003220EF00E3E922000080410083
:105D30001040BA000160EF0000000600202A0000B9
:105D40002A2A0000444B00002D440000454E00006C
:105D50004D410000524B00002A2A00002A2000007A
:105D6000000000003220EF00E3EB22000080410041
:105D70001040BA000160EF0000000600202A000079
:105D80002A2A0000464900002D460000494E000026
:105D90004C4100004E4400002A2A00002A20000046
:105DA000000000003220EF00E3ED220000804100FF
:105DB0001040BA000160EF0000000600202A000039
:105DC0002A2A0000465200002D46000052410000E1
:105DD0004E430000452A00002A2A0000200000004F
:105DE0003220EF00C3EF2200008041001040BA00D3
:105DF0000160EF0000000600202A00002A2A0000AF
:105E0000444500002D470000455200004D41000070
:105E10004E5900002A2A00002A200000000000003D
:105E20003220EF00C3F12200008041001040BA0090
:105E30000160EF0000000600202A00002A2A00006E
:105E4000495400002D490000544100004C59000005
:105E50002A2A00002A200000000000003220EF0063
:105E6000A3F32200008041001040BA000160EF005F
:105E700000000600202A00002A2A00004E4C0000E4
:105E80002D4E00004554000048450000524C0000D3
:105E9000414E0000445300002A2A00002A2000003E
:105EA000000000003220EF00E3F5220000804100F6
:105EB0001040BA000160EF0000000600202A000038
:105EC0002A2A00004E4F00002D4E00004F520000C5
:105ED00057410000592A00002A2A00002000000033
:105EE0003220EF00C3F72200008041001040BA00CA
:105EF0000160EF0000000600202A00002A2A0000AE
:105F0000455300002D53000050410000494E000051
:105F10002A2A00002A200000000000003220EF00A2
:105F2000A3F92200008041001040BA000160EF0098
:105F300000000600202A00002A2A00005345000025
:105F40002D53000057450000444500004E2A000034
:105F50002A2A0000200000003220EF0083FB2200EC
:105F6000008041001040BA000160EF000000060010
:105F7000202A00002A2A0000434800002D53000078
:105F800057490000545A0000455200004C4100009F
:105F90004E4400002A2A00002A20000000000000D1
:105FA0003220EF00C3FD2200008041001040BA0003
:105FB0000160EF0000000600202A00002A2A0000ED
:105FC000554B00002D49000054490000532A0000A1
:105FD0002A2A0000200000003220EF0083FF220068
:105FE000008041001040BA000160EF000000060090
:105FF000202A00002A2A0000554B00002D540000E2
:106000004D2A00002A2A0000200000003220EF0064
:1060100023012300008041001040BA000160EF001E
:10602000000006000A0D00002A200000543D000078
:1060300025750000204600003D2500007520000069
:10604000445000003D250000750000003220EF00A4
:1060500023032300008041001040BA000160EF00DC
:1060600000000600204400003D25000075200000CF
:1060700064690000723D00002575000020450000A5
:10608000585400003D250000750000003220EF004C
:1060900023052300008041001040BA000160EF009A
:1060A0000000060020450000565400003D25000079
:1060B0004C750000204C00004F4300003D250000BF
:1060C0004C750000200000003220EF000307230081
:1060D000008041001040BA000160EF00000006009F
:1060E00020540000554E0000204900004E4600009C
:1060F0000A0D0000000000003220EF00830823009A
:10610000008041001040BA000160EF00000006006E
:1061100020530000414D0000452000004D53000079
:1061200047200000696E0000204600005241000038
:106130004D200000000000003220EF00830A230001
:10614000008041001040BA000160EF00000006002E
:10615000204F000054480000204D0000534700002D
:10616000206900006E20000046520000414D0000F2
:10617000200000003220EF00630C2300008041006B
:106180001040BA000160EF0000000600207400001B
:106190006D6300005F63000075720000725F0000B5
:1061A0006D6500007373000061670000653D0000CD
:1061B00020250000750000003220EF00830E230030
:1061C000008041001040BA000160EF0000000600AE
:1061D000202A00002A2A0000200A00000D200000CA
:1061E0000A0D0000000000003220EF000310230021
:1061F000008041001040BA000160EF00000006007E
:106200002021000021200000746D0000635F000069
:1062100065760000745F000073740000726900000E
:106220006E6700003D250000732000000A0D00008D
:10623000000000003220EF006312230000804100C4
:106240001040BA000160EF0000000600207400005A
:106250006D6300005F65000076740000636C0000F1
:10626000725F000073740000726900006E670000C6
:10627000323D000025730000200A00000D000000E0
:106280003220EF00C3142300008041001040BA0008
:106290000160EF0000000600206D00006174000046
:1062A00063680000206900003D25000075200000A3
:1062B0002A2A00002A2A00002A2A00002A2A00008E
:1062C000000000003220EF00E316230000804100B0
:1062D0001040BA000160EF0000000600204D0000F1
:1062E00053470000204300004E4C0000440A0000C9
:1062F0000D0000003220EF006318230000804100F1
:106300001040BA000160EF0000000600206E00009F
:106310006F740000206900006E2000005A5A0000CF
:106320002D6100006C650000727400002D63000098
:1063300021200000000000003220EF00831A23001B
:10634000008041001040BA000160EF00000006002C
:106350000A0D0000202B00002B2B00002043000022
:10636000433D000025780000204C0000544E000002
:106370003D250000782000000A0D0000000000000C
:106380003220EF00C31C2300008041001040BA00FF
:106390000160EF00000006006E6F00007420000036
:1063A000696E0000204C00004F4300000A0D000001
:1063B000000000003220EF00631E23000080410037
:1063C0001040BA000160EF0000000600310000003C
:1063D0003220EF00431F2300008041001040BA002C
:1063E0000160EF0000000600206E00006F740000E6
:1063F000206900006E200000504F0000494E000050
:10640000545300000A0D0000000000003220EF008D
:1064100023212300008041001040BA000160EF00FA
:1064200000000600320000003220EF0003222300AB
:10643000008041001040BA000160EF00000006003B
:10644000582E0000000000003220EF00032323003C
:10645000008041001040BA000160EF00000006001B
:10646000502E0000000000003220EF000324230023
:10647000008041001040BA000160EF0000000600FB
:10648000546E00006C0000003220EF000325230052
:10649000008041001040BA000160EF0000000600DB
:1064A000427200006964000067650000000000009F
:1064B0003220EF0043262300008041001040BA0044
:1064C0000160EF0000000600436100007220000040
:1064D00050610000726B0000000000003220EF00ED
:1064E000A3272300008041001040BA000160EF00A4
:1064F00000000600467200006F6E00007469000024
:1065000065720000000000003220EF000329230024
:10651000008041001040BA000160EF00000006005A
:1065200054650000726D0000696E0000616C00002F
:10653000000000003220EF00632A230000804100A9
:106540001040BA000160EF00000006004861000042
:10655000726200006F750000720000003220EF00D0
:10656000A32B2300008041001040BA000160EF001F
:106570000000060041690000727000006F720000A8
:10658000740000003220EF00E32C23000080410063
:106590001040BA000160EF000000060053740000D4
:1065A00061740000696F00006E0000003220EF008F
:1065B000232E2300008041001040BA000160EF004C
:1065C0000000060056690000616400007563000069
:1065D000740000003220EF00632F23000080410090
:1065E0001040BA000160EF00000006003300000018
:1065F0003220EF0043302300008041001040BA00F9
:106600000160EF0000000600340000003220EF00BF
:1066100023312300008041001040BA000160EF00E8
:1066200000000600350000003220EF000332230096
:10663000008041001040BA000160EF000000060039
:10664000202A00002A2A00004D53000047200000A5
:10665000746F000020460000524100004D2A0000E7
:106660002A2A0000200000003220EF00033423001B
:10667000008041001040BA000160EF0000000600F9
:10668000202A00002A2A0000202500007320000094
:10669000000000003220EF0063352300008041003D
:1066A0001040BA000160EF00000006007C200000EE
:1066B00025730000202D00002D3E0000200000006A
:1066C0003220EF00C3362300008041001040BA00A2
:1066D0000160EF000000060020610000742000004F
:1066E0002573000020250000730000003220EF0019
:1066F00023382300008041001040BA000160EF0001
:106700000000060020660000726F00006D2000008F
:106710002573000020250000730000003220EF00E8
:10672000A3392300008041001040BA000160EF004F
:1067300000000600207400006F2000002573000098
:1067400020250000730000003220EF00033B2300EF
:10675000008041001040BA000160EF000000060018
:10676000202000002020000020200000204E0000FB
:1067700045570000202000002020000020200000BD
:1067800020200000200000003220EF00033D230005
:10679000008041001040BA000160EF0000000600D8
:1067A0002020000020200000202000005550000084
:1067B000444100005445000020200000202000003B
:1067C00020200000200000003220EF00033F2300C3
:1067D000008041001040BA000160EF000000060098
:1067E00061640000643000003120000000000000FF
:1067F0003220EF0043402300008041001040BA00E7
:106800000160EF000000060077300000312000003A
:10681000000000003220EF006341230000804100AF
:106820001040BA000160EF00000006002070000078
:106830007265000030330000200000003220EF00BD
:10684000A3422300008041001040BA000160EF0025
:106850000000060020730000746F0000703000001C
:1068600031200000000000003220EF00034423002C
:10687000008041001040BA000160EF0000000600F7
:106880006164000064320000200000003220EF004C
:1068900023452300008041001040BA000160EF0052
:1068A00000000600773000003220000000000000E9
:1068B0003220EF0043462300008041001040BA0020
:1068C0000160EF00000006002D2D00002D2D0000BE
:1068D0002D2D00002D2D0000000000003220EF00C3
:1068E000C30120008301500005003100A3482300AC
:1068F000008041001040BA000160EF000000060077
:10690000B048230083814100808141001380BA0098
:106910000000060020202000202020002020200051
:1069200020202000202020002020200020202000E7
:1069300020202000202020002020200020202000D7
:106940002020200020202000202000003220EF0006
:10695000234B2300008041001040BA000160EF008B
:106960000000060020200000202000002020000061
:106970002020000020200000202000002020000017
:106980002020000020200000202000002020000007
:10699000200000003220EF00634D23000080410002
:1069A0001040BA000160EF00000006002043000024
:1069B000545F00004D4A0000443D0000256C00007B
:1069C00075200000000000003220EF00034F23007C
:1069D000008041001040BA000160EF000000060096
:1069E0004D6F00006E0000003220EF0003502300C6
:1069F000008041001040BA000160EF000000060076
:106A000054750000650000003220EF0003512300A0
:106A1000008041001040BA000160EF000000060055
:106A200057650000640000003220EF00035223008D
:106A3000008041001040BA000160EF000000060035
:106A400054680000750000003220EF00035323005B
:106A5000008041001040BA000160EF000000060015
:106A600046720000690000003220EF00035423004A
:106A7000008041001040BA000160EF0000000600F5
:106A800053610000740000003220EF000355230022
:106A9000008041001040BA000160EF0000000600D5
:106AA000537500006E0000003220EF0003562300F3
:106AB000008041001040BA000160EF0000000600B5
:106AC0004A6100006E0000003220EF0003572300EF
:106AD000008041001040BA000160EF000000060095
:106AE00046650000620000003220EF0003582300DA
:106AF000008041001040BA000160EF000000060075
:106B00004D610000720000003220EF0003592300A5
:106B1000008041001040BA000160EF000000060054
:106B200041700000720000003220EF00035A230081
:106B3000008041001040BA000160EF000000060034
:106B40004D610000790000003220EF00035B23005C
:106B5000008041001040BA000160EF000000060014
:106B60004A7500006E0000003220EF00035C230035
:106B7000008041001040BA000160EF0000000600F4
:106B80004A7500006C0000003220EF00035D230016
:106B9000008041001040BA000160EF0000000600D4
:106BA00041750000670000003220EF00035E230003
:106BB000008041001040BA000160EF0000000600B4
:106BC00053650000700000003220EF00035F2300D7
:106BD000008041001040BA000160EF000000060094
:106BE0004F630000740000003220EF0003602300B8
:106BF000008041001040BA000160EF000000060074
:106C00004E6F0000760000003220EF000361230089
:106C1000008041001040BA000160EF000000060053
:106C200044650000630000003220EF00036223008F
:106C3000008041001040BA000160EF000000060033
:106C40000A0D000020530000494400003D250000CB
:106C5000782000000A0D0000000000003220EF0044
:106C6000A3632300008041001040BA000160EF00E0
:106C7000000006004465000066610000756C0000BD
:106C800074200000696E00007465000072720000DC
:106C900075700000740D00000A0000003220EF0043
:106CA000A3652300008041001040BA000160EF009E
:106CB000000006000A0D00002030000035340000FE
:106CC000202D0000204C0000697600006551000076
:106CD000205400004D430000202000000A0D000059
:106CE000000000003220EF00E36723000080410035
:106CF0001040BA000160EF0000000600204F0000C5
:106D00004C450000442000003136000030200000D7
:106D1000782000003132000038200000646F00004D
:106D20007473000020520000474200002021000040
:106D3000200000003220EF00636A23000080410041
:106D40001040BA000160EF0000000600546500002A
:106D5000636800004465000073690000676E00000E
:106D6000200000003220EF00E36B23000080410090
:106D70001040BA000160EF0000000600456C000002
:106D800065630000747200006F6E000069630000AC
:106D9000730000003220EF00636D2300008041008B
:106DA0001040BA000160EF00000006004C690000CE
:106DB0007665000051200000544D000043000000A3
:106DC0003220EF00C36E2300008041001040BA0063
:106DD0000160EF00000006002070000072650000F6
:106DE00073650000745F000066720000657100004A
:106DF0003D2500004C750000200000003220EF000F
:106E0000A3702300008041001040BA000160EF0031
:106E1000000006004D4D0000432F000053440000C9
:106E2000206900006E69000074200000646F00009B
:106E30006E650000200A00000D0000003220EF0007
:106E4000A3722300008041001040BA000160EF00EF
:106E5000000006004D4D0000432F00005344000089
:106E6000207200006561000064200000626F000075
:106E70006F740000206400006F6E0000650A00005F
:106E80000D200000000000003220EF0003752300F9
:106E9000008041001040BA000160EF0000000600D1
:106EA0000A0D0000202A00002A200000666E000063
:106EB0006E3D0000253400006C75000000000000ED
:106EC0003220EF00C3762300008041001040BA005A
:106ED0000160EF0000000600206600007363000000
:106EE0003D250000386C0000752000000000000007
:106EF0003220EF0043782300008041001040BA00A8
:106F00000160EF00000006002066000073730000BF
:106F10003D250000386C00007520000000000000D6
:106F20003220EF00C3792300008041001040BA00F6
:106F30000160EF0000000600206600006C6C00009D
:106F40003D250000386C00007520000000000000A6
:106F50003220EF00437B2300008041001040BA0044
:106F60000160EF0000000600206600007261000072
:106F7000673D000025750000200A00000D0000009C
:106F80003220EF00C37C2300008041001040BA0093
:106F90000160EF0000000600206500006E64000044
:106FA0005F6200006F6F0000740A00000D000000B7
:106FB0003220EF00437E2300008041001040BA00E1
:106FC0000160EF0000000600746D00006300000027
:106FD0003220EF00437F2300008041001040BA00C0
:106FE0000160EF0000000600544100002000000096
:106FF0003220EF0043802300008041001040BA009F
:107000000160EF0000000600545000002000000066
:107010003220EF0043812300008041001040BA007D
:107020000160EF00000006002020000020000000AA
:107030003220EF0043822300008041001040BA005C
:107040000160EF00000006004E6F000020540000B9
:107050004D4300002D6D000065730000736100005A
:1070600067650000730000003220EF0003842300F6
:10707000008041001040BA000160EF0000000600EF
:107080002020000020200000202000002020000000
:1070900020200000202000002020000020200000F0
:1070A0002020000020200000200000003220EF00FF
:1070B00023862300008041001040BA000160EF00E9
:1070C00000000600202A00002A6500006E740000FF
:1070D000657200002A2A0000200000003220EF0024
:1070E000A3872300008041001040BA000160EF0038
:1070F00000000600202A00002A70000072650000CF
:107100007365000074200000736100007665000064
:10711000642A00002A200000000000003220EF0056
:10712000A3892300008041001040BA000160EF00F5
:107130000000060073610000766500006400000036
:107140003220EF00C38A2300008041001040BA00C3
:107150000160EF0000000600202A000054550000E6
:107160004E2A0000200000003220EF00038C230094
:10717000008041001040BA000160EF0000000600EE
:10718000202A000053450000542A0000200000007F
:107190003220EF00438D2300008041001040BA00F0
:1071A0000160EF000000060020530000657400003D
:1071B000746900006E67000073200000200000006A
:1071C0003220EF00C38E2300008041001040BA003F
:1071D0000160EF000000060052490000474800002F
:1071E000543A00002066000061630000746F0000E4
:1071F0007279000020720000657300006574000061
:10720000000000003220EF00E390230000804100E6
:107210001040BA000160EF00000006004C4500007D
:10722000465400003A2000007265000073650000BB
:107230007276000065640000000000003220EF005C
:10724000A3922300008041001040BA000160EF00CB
:1072500000000600555000003A2000004F4C00008E
:1072600045440000206900006E740000656E000057
:107270007369000074790000207500007000000040
:107280003220EF00C3942300008041001040BA0078
:107290000160EF0000000600444F0000574E000060
:1072A0003A2000004F4C00004544000020690000D7
:1072B0006E740000656E0000736900007479000050
:1072C000206400006F7700006E0000003220EF00A5
:1072D00023972300008041001040BA000160EF00B6
:1072E00000000600454E000054450000523A0000E0
:1072F000206C00006561000076650000206D0000D4
:10730000656E0000750000003220EF000399230035
:10731000008041001040BA000160EF00000006004C
:10732000202A00004E410000562A000020000000E4
:107330003220EF00439A2300008041001040BA0041
:107340000160EF0000000600202A00002A72000001
:1073500069670000687400002A2A0000200000000D
:107360003220EF00C39B2300008041001040BA0090
:107370000160EF0000000600202A00002A6C0000D7
:1073800065660000742A00002A200000000000004A
:107390003220EF00439D2300008041001040BA00DE
:1073A0000160EF0000000600202A00002A7500009E
:1073B000702A00002A200000000000003220EF00A8
:1073C000A39E2300008041001040BA000160EF003E
:1073D000000006004F4C00004544000020690000FA
:1073E0006E740000656E000073690000747900001F
:1073F0003D200000000000003220EF0083A02300A9
:10740000008041001040BA000160EF00000006005B
:10741000202A00002A6400006F7700006E2A000016
:107420002A200000000000003220EF0003A2230009
:10743000008041001040BA000160EF00000006002B
:107440002073000074610000727400005F6300002C
:1074500069740000794E00003D25000064000000C2
:107460003220EF00C3A32300008041001040BA0087
:107470000160EF0000000600202A00002A2A000018
:107480002A4300004C300000326100002000000060
:107490003220EF0043A52300008041001040BA00D5
:1074A0000160EF00000006003C6500006E64000013
:1074B000206F0000662000006C69000073740000FB
:1074C0003E0000003220EF00E3A6230000804100D0
:1074D0001040BA000160EF0000000600202000000C
:1074E000202000002020000020200000202000009C
:1074F0002020000020200000000000003220EF00CB
:10750000A3A82300008041001040BA000160EF00F2
:1075100000000600206D0000617000005F7A00002E
:107520006F6F00006D3D0000256C000075200000AD
:10753000000000003220EF0063AA23000080410019
:107540001040BA000160EF00000006002047000074
:107550006F7400006F2000007A6F00006F6D0000F4
:107560002076000069650000773A000020000000E6
:107570003220EF0043AC2300008041001040BA00ED
:107580000160EF0000000600206B00006D2000008D
:10759000200000003220EF0063AD23000080410096
:1075A0001040BA000160EF000000060066720000A3
:1075B000640000003220EF0063AE23000080410031
:1075C0001040BA000160EF00000006006672000083
:1075D000750000003220EF0063AF230000804100FF
:1075E0001040BA000160EF00000006006366000072
:1075F000720000003220EF0063B0230000804100E1
:107600001040BA000160EF00000006007366000041
:10761000720000003220EF0063B1230000804100BF
:107620001040BA000160EF00000006007264000024
:10763000730000003220EF0063B22300008041009D
:107640001040BA000160EF00000006006366000011
:10765000723D0000253300002E310000672000003D
:107660000A0D0000200000003220EF0003B42300C8
:10767000008041001040BA000160EF0000000600E9
:1076800063660000723D0000253300002E310000CB
:1076900067200000000000003220EF0083B52300C7
:1076A000008041001040BA000160EF0000000600B9
:1076B00020500000533D0000257300002000000012
:1076C0003220EF00C3B62300008041001040BA0012
:1076D0000160EF000000060052540000613D000010
:1076E000257300000A0D0000000000003220EF00AA
:1076F00023B82300008041001040BA000160EF0071
:107700000000060052540000623D00002573000096
:107710000A0D0000000000000000E0004220AF0061
:1077200008003700190E09000000000005000900DC
:1077300000000000FF3F0900000000000000E90019
:10774000F5FF3700000006003600F800801F7800C3
:10775000200020000C000900B01F7800010020006C
:10776000010078002E360200000000008100E800D1
:107770003322AF00FEFF3700A01188002001200057
:107780000008E600F6FF3700803E20008C3B020038
:1077900000000000A00120000C0009004F1078003C
:1077A0004F0078003600F900004006003202AE00BB
:1077B000FEFF37003202F8000608F900B011800021
:1077C0003222A900000006003600F800801F780071
:1077D000200020000C000900B01F78004441800008
:1077E0000960EF008380200083024200467F800012
:1077F000D63B020000000000467F8800804A7800E7
:1078000028C8BF002AE8B700444180006142420016
:107810000440780000E0B7007F40600028E8B7002F
:1078200028C8BF002948E30002003A002AC8BF0068
:1078300028E8B70087C0A900A00120000C000900BB
:107840004F1078004F0078003600F9000040060025
:10785000CAC2A800C6C2A90000000000E8C2A90070
:10786000E902A9000000060070C0B30082F2B70070
:1078700014948000F4CFB2001800320081D2BF000F
:107880008000780082D2BF000100A5000200310014
:10789000E862A90001003700E862A80000000000CB
:1078A000000000000000000000000000E842A80006
:1078B00000000000000000000000000000000000C8
:1078C000E842A900000000000000000000000000E5
:1078D000000000008272ED00E5FF370000000600A6
:1078E0000428210024178800E842A900E862A900C2
:1078F0000000000000000000E9C2A9000000000034
:1079000000000000000000000000000080C4B30080
:1079100081F2B700343C02000000000079D2BF00C1
:1079200081F2B700343C0200000000007AD2BF00B0
:1079300081F2B700343C0200000000007BD2BF009F
:1079400081F2B700343C0200000000007CD2BF008E
:1079500081F2B700343C0200000000007DD2BF007D
:1079600081F2B700343C0200000000007ED2BF006C
:1079700081F2B700343C0200000000007FD2BF005B
:1079800081F2B700343C02000000000080D2BF004A
:1079900081F2B700343C020000000000000000004B
:1079A000000000000000000000000000E9C2A80084
:1079B00000000600E70160004300DE000100400017
:1079C0000000A700E88141000000A1000204E000DF
:1079D0001098AD0000000600851F78006372EF006C
:1079E00070C0B30064F2B70024938000F4CFB200FB
:1079F00016003200E842A80000000000000000006D
:107A00000000000000000000E842A900E662AE00AD
:107A1000080037003126210064D2BF000160EF006A
:107A200012002000821F78004F017800DA3C02002B
:107A30000000000000000000000000000000000046
:107A4000000000006472ED00E7FF370063D2BF0062
:107A500000E0B700CF027800000006006072EF007F
:107A60000428210024178800E842A900E862A90040
:107A7000E9C2A900000000000000000000000000B2
:107A80000000000000C8B30081F2B700343C0200DF
:107A900000000000000000000000000000000000E6
:107AA0000000000084282100241788000000000046
:107AB000000000000000000000000000EC3C02009C
:107AC0000000000060F2B7000000000000000000AD
:107AD0000000000000000000E9C2A8000428210006
:107AE0002417880060D2BF0000E0B7000000060045
:107AF000851F7800861F7800E9C2A80004282100AD
:107B000024178800E842A900E862A900E9A2A800B9
:107B10001E0E090000000000FF3F090000000000E9
:107B2000E9A2A9001E0E090000000000FF3F0900A5
:107B300000000000E9A2A8001E0E090000000000DD
:107B4000FF3F090000000000010020000100780054
:107B500070230200000000008100E8003322AF0023
:107B6000FEFF3700A0118800000120000008E60099
:107B7000F6FF370010C0B30079F2B70000C1B300C0
:107B80007AF2B70050C0B3007BF2B7007C72EF000E
:107B90007D72EF007E72EF007F72EF008072EF0067
:107BA000703C0200000000002E3D020000000000BA
:107BB000804278000040EB000AE0AF000000E800DF
:107BC0000004E00006003A00000000003322AF008D
:107BD000FEFF3700A4022000A4118800F2FF370046
:107BE00020C1B30079F2B7007A72EF0010C1B30080
:107BF0007BF2B7007C72EF007D72EF0010C0B30023
:107C00007EF2B7007F72EF008072EF00703C0200DE
:107C1000000000002E3D02000000000080427800BD
:107C20000040EB000AE0AF000000E8000004E000C4
:107C300002003A0000000000F6FF370020C1B30048
:107C400079F2B7007A72EF0050C1B3007BF2B7004F
:107C50007C72EF007D72EF0010C0B3007EF2B700BF
:107C60007F72EF008072EF00703C020000000000A5
:107C70002E3D020000000000804278000040EB0032
:107C80000AE0AF000000E8000004E00002003A0053
:107C900000000000F6FF370020C1B30079F2B70002
:107CA0007A72EF0050C1B3007BF2B70010C0B3008E
:107CB0007CF2B7007D72EF0010C0B3007EF2B70017
:107CC0007F72EF008072EF00703C02000000000045
:107CD0002E3D020000000000804278000040EB00D2
:107CE0000AE0AF000000E8000004E00002003A00F3
:107CF00000000000F6FF370020C1B30079F2B700A2
:107D00007A72EF0050C1B3007BF2B70020C0B3001D
:107D10007CF2B70050C5B3007DF2B70010C0B300CD
:107D20007EF2B7007F72EF008072EF00703C0200BD
:107D3000000000002E3D020000000000804278009C
:107D40000040EB000AE0AF000000E8000004E000A3
:107D500002003A0000000000F6FF3700F0C3B30055
:107D60000EEBB70020C1B30079F2B7007A72EF00D2
:107D700000C4B3007BF2B7007C72EF007D72EF00AD
:107D80000ECBBF007EF2B7007F72EF008072EF0073
:107D9000703C0200000000002E3D020000000000C8
:107DA000804278000040EB000AE0AF000000E800ED
:107DB0000004E00002003A0000000000F6FF370077
:107DC00001002000010078009C2302000000000058
:107DD0008100E8003322AF00FEFF3700A0118800C9
:107DE000C00020000008E600F6FF370000C2B30024
:107DF00079F2B7007A72EF0010C2B3007BF2B700DD
:107E0000C0CFB3007CF2B7007D72EF007E72EF004E
:107E10007F72EF008072EF00703C020000000000F3
:107E20002E3D020000000000804278000040EB0080
:107E30000AE0AF000000E8000004E00002003A00A1
:107E400000000000F6FF370010C2B30079F2B7005F
:107E5000C0C0B3007AF2B7007B72EF007C72EF0013
:107E60007D72EF007E72EF007F72EF008072EF0094
:107E7000703C0200000000004F037800CF02780041
:107E8000000006003400200024B38800CAC2A90004
:107E9000C6C2A90070C0B30066F6B70034B3800054
:107EA000F4CFB2000B00320021B3800066D6BF00D1
:107EB0000100A50002003100E902A900010037001D
:107EC000E902A800E8C2A900E8C2A8006676ED00B1
:107ED000F2FF37006216F8006416F900F0C0B30034
:107EE00066F6B70034B38000F4CFB2000B00320066
:107EF00021B3800066D6BF000100A500020031005A
:107F0000E902A90001003700E902A800E8C2A900BF
:107F1000E8C2A8006676ED00F2FF37000000060018
:107F20005D76EF0070C0B3005EF6B700F4B280007B
:107F3000F4CFB2000E003200E8C2A900E8C2A800E7
:107F4000E6E2AE0008003700D16521005ED6BF0032
:107F50000160EF0012002000821F78004F017800BE
:107F6000DA3C0200000000005E76ED00EFFF370013
:107F70005DD6BF0000E0B70000000600E8C2A9001F
:107F8000CAC2A800C6C2A90000000600851F78006A
:107F9000E822A900CB62A900C762A900CB82A80091
:107FA000C782A900CBA2A900C7A2A90044B3800040
:107FB0000960EF000380200083024200B5168800AC
:107FC000CBA2A800C7A2A900E822A800E822A90025
:107FD000CB62A800C762A900CB82A800C782A90013
:107FE000CBA2A900C7A2A90044B380004822DE00AA
:107FF0000380200083024200B5168800CBA2A800AF
:10800000C7A2A900E822A800CF027800000006005D
:10801000E822A800E9E2A900A00020008C3B0200B1
:1080200000000000E9E2A8001E0E090000000000A8
:10803000FF3F090000000000400620008C3B0200CA
:108040000000000040C0B30068F6B70010C0B300E5
:1080500069F6B700C63F0200000000001E0E0900CE
:1080600000000000FF3F09000000000040C0B30016
:1080700068F6B70040C0B30069F6B700C63F02001B
:10808000000000001E0E090000000000FF3F090074
:108090000000000060C1B30068F6B70050C4B30030
:1080A00069F6B700C63F02000000000020C0B30020
:1080B00068F6B70010C4B30069F6B700C63F020007
:1080C0000000000080C0B30068F6B70030C0B30005
:1080D00069F6B700C63F02000000000090C0B30080
:1080E00068F6B70050C0B30069F6B700C63F02009B
:1080F00000000000A0C0B30068F6B70050C0B30095
:1081000069F6B700C63F020000000000B0C0B3002F
:1081100068F6B70080C4B30069F6B700C63F020036
:1081200000000000C0C0B30068F6B700D0C4B300C0
:1081300069F6B700C63F020000000000D0C0B300DF
:1081400068F6B70060C4B30069F6B700C63F020026
:108150000000000000C1B30068F6B7000CCBBF0000
:1081600069F6B700C63F02000000000010C1B3006E
:1081700068F6B7000CCBBF0069F6B700C63F020037
:108180000000000020C1B30068F6B7000CCBBF00B0
:1081900069F6B700C63F02000000000040C0B3000F
:1081A00068F6B7006976EF00C63F020000000000E5
:1081B0001E0E090000000000FF3F09000000000043
:1081C0001E0E090000000000FF3F09000000000033
:1081D000B0C3B30068F6B7006976EF00C63F02008F
:1081E0000000000000000600851F780065B38000D5
:1081F000C22ADD006DD6BF000160EF004400DE0042
:108200006FF6B700054078006F76B7007106A900D9
:108210006D66AF007106A80065B38000C82ADE0055
:10822000C52ADD006ED6BF000160EF004100DE0010
:1082300070F6B700054078007076B7007126A90087
:108240006E06AF007126A800E822A900CB62A80044
:10825000C762A900CB82A800C782A900CBA2A9004F
:10826000C7A2A90074B380004822DE00038020006A
:1082700083024200B51688007106AF000200370085
:10828000CB02A90001003700CB02A800C702A90059
:10829000CBA2A800C7A2A900CB62A900C762A9000F
:1082A000E822A800E822A900CB62A800C762A900C2
:1082B000CB82A800C782A900CBA2A900C7A2A900AF
:1082C00084B380000960EF00038020008302420035
:1082D000B51688007126AF0002003700CB02A90056
:1082E00001003700CB02A800C702A900CBA2A8005A
:1082F000C7A2A900CB62A900C762A900E822A80012
:10830000CF02780000000600047020009416880058
:1083100070C1B30068F6B7006976EF00C63F02008F
:108320000000000080C1B30068F6B700F0C9B300D8
:1083300069F6B700C63F02000000000090C1B3001C
:1083400068F6B7006976EF00C63F02000000000043
:10835000A0C1B30068F6B700F0C7B30069F6B70074
:10836000C63F02000000000000C2B30068F6B7007C
:108370006976EF00C63F02000000000010C2B300A3
:1083800068F6B700F0C7B30069F6B700C63F020051
:10839000000000000470200094168800E822A90064
:1083A000CB62A900C762A900CB82A800C782A9003E
:1083B000CBA2A900C7A2A90024822000B41688007D
:1083C000CBA2A800C7A2A900CB62A800C762A900DF
:1083D000E822A8002635EF0034A98000030025001C
:1083E0000418E100070032006C76EF006D76EF00B4
:1083F0006E76EF00F4400200000000002635EC002D
:10840000F5FF37000000060070C1B30068F6B70042
:108410006976EF00C63F02000000000080C1B30093
:1084200068F6B700F0C9B30069F6B700C63F0200AE
:108430000000000090C1B30068F6B7006976EF0055
:10844000C63F020000000000A0C1B30068F6B700FC
:10845000F0C7B30069F6B700C63F02000000000095
:1084600000C2B30068F6B7005FD6BF0069F6B70078
:10847000C63F02000000000010C2B30068F6B7005B
:1084800060D6BF0069F6B700C63F020000000000DA
:108490005FD6BF0002EBB700036BEF0060D6BF00F2
:1084A00004EBB700056BEF00047020009416880001
:1084B000E822A900CB62A900C762A900CB82A8006C
:1084C000C782A900CBA2A900C7A2A90024822000CC
:1084D000B4168800CBA2A800C7A2A900CB62A8004E
:1084E000C762A900E822A80000000600F457800037
:1084F00074CCB20003003A0000C8B300FEEAB70033
:10850000E3003700F4578000C4CFB20003003A0004
:1085100010C8B300FEEAB700DD003700F457800052
:1085200094CEB20003003A0020C8B300FEEAB700C0
:10853000D7003700F457800024CEB20003003A0081
:1085400030C8B300FEEAB700D1003700F45780000E
:1085500044CEB20003003A0040C8B300FEEAB700C0
:10856000CB003700F457800004CEB20003003A007D
:1085700050C8B300FEEAB700C5003700F4578000CA
:1085800054CEB20003003A0060C8B300FEEAB70060
:10859000BF003700F457800074CEB20003003A00E9
:1085A00070C8B300FEEAB700B9003700F457800086
:1085B000A4CEB20003003A0080C8B300FEEAB700C0
:1085C000B3003700F4578000B4CEB20003003A0085
:1085D00090C8B300FEEAB700AD003700F457800042
:1085E00084CEB20003003A00A0C8B300FEEAB70090
:1085F000A7003700F4578000F4CEB20003003A0021
:10860000B0C8B300FEEAB700A1003700F4578000FD
:10861000E4CEB20003003A00C0C8B300FEEAB700DF
:108620009B003700F4578000C4CEB20003003A002C
:10863000D0C8B300FEEAB70095003700F4578000B9
:1086400044CCB20003003A00E0C8B300FEEAB70031
:108650008F003700F457800054CCB20003003A007A
:10866000F0C8B300FEEAB70089003700F457800075
:1086700094CCB20003003A0000C9B300FEEAB70090
:1086800083003700F457800064CEB20003003A0044
:1086900010C9B300FEEAB7007D003700F457800030
:1086A00064CCB20003003A0020C9B300FEEAB70070
:1086B00077003700F457800044CFB20003003A003F
:1086C00030C9B300FEEAB70071003700F4578000EC
:1086D00064CFB20003003A0040C9B300FEEAB7001D
:1086E0006B003700F457800024CFB20003003A003B
:1086F00050C9B300FEEAB70065003700F4578000A8
:10870000B4CFB20003003A0060C9B300FEEAB7007C
:108710005F003700F457800094CFB20003003A00A6
:1087200070C9B300FEEAB70059003700F457800063
:10873000F4CFB20003003A0080C9B300FEEAB700EC
:1087400053003700F457800064CDB20003003A00B4
:1087500090C9B300FEEAB7004D003700F45780001F
:10876000C4CDB20003003A00A0C9B300FEEAB700CE
:1087700047003700F457800084CFB20003003A006E
:10878000B0C9B300FEEAB70041003700F4578000DB
:1087900034CAB20003003A00C0C9B300FEEAB70011
:1087A0003B003700F457800084CDB20003003A004C
:1087B000D0C9B300FEEAB70035003700F457800097
:1087C00074CDB20003003A00E0C9B300FEEAB7007E
:1087D0002F003700F457800034C8B20003003A007D
:1087E000F0C9B300FEEAB70029003700F457800053
:1087F00014CEB20003003A0000CAB300FEEAB7008C
:1088000023003700F4578000D4CEB20003003A00B2
:1088100010CAB300FEEAB7001D003700F45780000D
:1088200034CFB20003003A0020CAB300FEEAB7001A
:1088300017003700F4578000A4CFB20003003A00BD
:1088400030CAB300FEEAB70011003700F4578000C9
:1088500014CFB20003003A0040CAB300FEEAB700EA
:108860000B003700F457800014CDB20003003A002B
:1088700050CAB300FEEAB70005003700F457800085
:10888000F4CDB20002003A0060CAB300FEEAB700BD
:1088900000000600851F7800861F7800F4578000CE
:1088A00003022000041CE10002003600AE00370085
:1088B00006003700F4578000F3072000041CE10095
:1088C000020031007642020000000000F4578000F0
:1088D000630A2000041CE10001003100A2003700FF
:1088E000FF6AEF00F45780004822DE006524E100B3
:1088F00073003100F457800003052000041CE100E0
:108900000C003600FECABF000042B10000427800F1
:108910000960EF006520B80000EBB70000CBBF0096
:10892000FF4AB400022002000000000001EBB70083
:108930001F003700F457800003082000041CE100EA
:108940000C003600FECABF000045B10000427800AE
:108950000960EF006520B80000EBB70000CBBF0056
:10896000FF4AB400BE2002000000000001EBB70087
:108970000F003700F4578000730A2000041CE10048
:108980000B003600FECABF000048B100004278006C
:108990000960EF006520B80000EBB70000CBBF0016
:1089A000FF4AB4007A2102000000000001EBB7008A
:1089B0006476EF0064D6BF000A4BE3003E0032004D
:1089C00070C0B30063F6B70014B380004822DE0025
:1089D000F4CFB2003600320000F02000080BB600E1
:1089E000800278004628DE0030B3880045588000B9
:1089F000050FB20045B388006836D5006836D5004B
:108A000040588000EF02600055B388006A36D400F9
:108A10006A36D40001CBBF008000780063D6BF0067
:108A20000100A5000F00390000F02000060BB60081
:108A3000800278004628DE0030B388003558800078
:108A4000050FB20045B388006836D5006836D500FA
:108A500030588000EF02600055B388006A36D400B9
:108A60006A36D4006576EF0065D6BF000B4BE30095
:108A70000A00320066D6BF006CF6B70068D6BF00A9
:108A80006DF6B7006AD6BF006EF6B700F44002007C
:108A9000000000006576EC00F3FF370014B380009F
:108AA0004822DE006140520063F6B700C6FF37007F
:108AB0006476EC00BFFF3700FF6AEC0089FF3700E7
:108AC00000F02000080BB600800278004628DE0087
:108AD00030B3880045588000050FB20045B38800C8
:108AE0006836D5006836D50040588000EF02600037
:108AF00055B388006A36D4006A36D4006476EF0035
:108B000064D6BF000A4BE300170032006376EF0023
:108B100014B380004822DE006824E1001000320017
:108B20006576EF0065D6BF000B4BE3000A0032000C
:108B300066D6BF006CF6B70068D6BF006DF6B7000A
:108B40006AD6BF006EF6B700F440020000000000D5
:108B50006576EC00F3FF37006376EC00ECFF37003E
:108B60006476EC00E6FF37004F037800CF02780010
:108B700000000600851F7800861F780070C1B300D2
:108B800068F6B70002CBBF0069F6B700C63F020027
:108B900000000000545880000960EF006620B80013
:108BA0000080FB001458800084024000801F780081
:108BB00080C1B30068F6B7004F007800801F7800CE
:108BC0000540780069F6B7004F007800C63F020004
:108BD0000000000090C1B30068F6B70004CBBF00EE
:108BE00069F6B700C63F0200000000000BCBBF00D3
:108BF0004300DD000080FB00245880008402400018
:108C000061835200A0C1B30068F6B7000640780047
:108C100069F6B700C63F02000000000000C2B300C2
:108C200068F6B70002CBBF0069F6B700C63F020086
:108C3000000000000BCBBF004300DD000080FB0004
:108C400024588000840240006183520010C2B300A7
:108C500068F6B7000640780069F6B700C63F020024
:108C6000000000000470200094168800E822A9008B
:108C7000CB62A900C762A900CB82A800C782A90065
:108C8000CBA2A900C7A2A90024822000B4168800A4
:108C9000CBA2A800C7A2A900CB62A800C762A90006
:108CA000E822A80062D6BF00FEEAB7004A440200EC
:108CB00000000000545880000960EF006620B800F2
:108CC0000080FB00022BB4004F037800CF02780035
:108CD000000006006400200074A98800CAC2A90030
:108CE000C6C2A90070C0B3002BF5B70054A980001C
:108CF0004822DE00F4CFB2000B00320071A98000E0
:108D00002BD5BF000100A50002003100E902A90037
:108D100001003700E902A800E8C2A900E8C2A800E3
:108D20002B75ED00F1FF3700E8C2A900CAC2A80008
:108D3000C6C2A900E8C2A900CAC2A900C6C2A90049
:108D40002400200074A9880070C0B3002BF5B70080
:108D500054A980004822DE00F4CFB2000B0032009C
:108D600071A980002BD5BF000100A50002003100D1
:108D7000E902A90001003700E902A800E8C2A90041
:108D8000E8C2A8002B75ED00F1FF3700E8C2A9008A
:108D90002C15F8002E15F900F0C0B3002BF5B70024
:108DA00054A980004822DE00F4CFB2000B0032004C
:108DB00071A980002BD5BF000100A5000200310081
:108DC000E902A90001003700E902A800E8C2A900F1
:108DD000E8C2A8002B75ED00F1FF3700E8C2A9003A
:108DE0000000060027D5BF0028F5B70070C0B3000B
:108DF00029F5B70044A980004822DE00F4CFB20074
:108E00000B00320041A9800029D5BF000100A50058
:108E100002003100E902A90001003700E902A800C0
:108E2000E8C2A900E8C2A8002975ED00F1FF3700EB
:108E3000E8C2A900000006006252E2001F003A00EA
:108E400001002000010078007429020000000000E9
:108E50008100E8003322AF00FEFF3700A011880038
:108E6000100120000008E600F6FF37006432EF0032
:108E70002493800003E027000418E1000E00320074
:108E80006412F8002C15F9006A4602000000000088
:108E90002775EF00F246020000000000BE3F02000E
:108EA0000000000004102000239380000480410093
:108EB00020938800EEFF37001F00370014938000D6
:108EC0006124E1001C003A0001002000010078004C
:108ED00094290200000000008100E8003322AF0066
:108EE000FEFF3700A0118800100120000008E600F6
:108EF000F6FF37002C35EF006A4602000000000044
:108F00006432EF002493800003E027000418E1009E
:108F1000070032002775EF00F24602000000000053
:108F2000249380006102420024938800F5FF3700FB
:108F3000BE3F020000000000000006003435EF00D4
:108F40003635EF00F0C1B30033F5B70094A98000C7
:108F50004822DE00F4CFB2000E003200E8C2A900C1
:108F6000E8C2A800E6E2AE00080037004153210045
:108F700033D5BF000160EF0012002000821F78008F
:108F80004F017800DA3C0200000000003375ED006C
:108F9000EEFF3700A0A98000B1A980000000060004
:108FA0005E36EF00F0C0B3005DF6B700E4B28000BB
:108FB0004822DE00F4CFB2000B003200E8C2A90064
:108FC000E8C2A800E6E2AE0005003700E165210036
:108FD0005DD6BF000160EF004220A9001180AD0006
:108FE0005D76ED00F1FF37005E16F8000000F90035
:108FF00000000600851F7800C5002000030009005E
:10900000B51F7800800378008404780004F0A10084
:109010000400E00006003A0009F0A7000200370053
:10902000050020000F003700050020000D0037006C
:10903000E64252000A0039000003200009F0A600B1
:10904000000220003322AF00FEFF3700A01188008D
:109050008502E900FBFF3B005500200001003700BE
:10906000840278006400200005E0A00009F0A70059
:1090700005F0A00008712200110009008883D800C3
:10908000744802000000000081037800883E200040
:10909000110009008883D800744802000000000015
:1090A0008103780048062000110009008883D80059
:1090B000744802000000000081037800A80020002E
:1090C000110009008883D8007448020000000000E5
:1090D0000003200000C040003322AF00FEFF370035
:1090E000A011880017003700060320000000E000F0
:1090F0000E003A0005E0A6000D0037000402E9006A
:109100000524E100020032004200AF00000006002A
:109110000000E00005003A0005E0A600040037006A
:1091200005F0A600060220000100370005E0A100BE
:10913000004043003322AF00FEFF3700A01188003B
:10914000000006002501200003000900CF1278006E
:10915000CF02780000000600E902A80070C0B3004A
:1091600065F2B700249380004822DE00F4CFB200FD
:1091700008003200E8C2A900000000000000000062
:10918000E8C2A80000000000000000006572ED00C9
:10919000F4FF37000060EF0000000600851F780034
:1091A0001E77EF0070C0B3001FF7B700F4B880005F
:1091B0004822DE00F4CFB200170032001DD7BF00F6
:1091C000800078001FD7BF000100A5000200310019
:1091D000E902A90001003700E902A8000000000030
:1091E000E8C2A900E8C2A800E6E2AE000800370025
:1091F000E17121001FD7BF000160EF0012002000C5
:10920000821F78004F017800DA3C02000000000065
:109210001F77ED00E5FF37001ED7BF0000E0B70065
:10922000CF02780000000600851F78001DF7EF00D0
:10923000CE4802000000000014D7BF001DF7B700A1
:10924000CE4802000000000017D7BF00800278005F
:109250000B60EF00054078001DF7B700CE48020014
:109260000000000016D7BF001DF7B700CE4802006F
:109270000000000019D7BF00800278000B60EF00EB
:10928000054078001DF7B700CE480200000000003E
:1092900018D7BF001DF7B700CE480200000000003D
:1092A00015D7BF001DF7B700CE4802000000000030
:1092B0001DF7EF00CE480200000000001DF7EF0090
:1092C000CE480200000000000FEBB7000FCBBF003C
:1092D00000E0B700CF02780000000600851F78008C
:1092E000861F78000001EB000103780064C11000C4
:1092F0004211DD000200DD00800278000C60EC000D
:109300000C60ED000D00320005007800C42ADD007D
:109310004C00DE00F000B2000003B000A203200009
:109320000200E100010039000D40B4003322AF001B
:10933000FEFF3700A0118800F1FF37004F037800CF
:10934000CF027800000006003C2BEF003E2BEF0020
:109350001DF7EF00CE4802000000000065D2BF00FC
:109360001DF7B700CE480200000000001DF7EF0017
:10937000CE480200000000001DF7EF00CE480200BA
:10938000000000001DF7EF00CE48020000000000C2
:109390001DF7EF00CE480200000000001DF7EF00AF
:1093A000CE480200000000001DF7EF00CE4802008A
:1093B000000000001DF7EF00CE4802000000000092
:1093C0001DF7EF00CE4802000000000066F2B70073
:1093D00066D2BF003CEBB7003D6BEF003E2BEF00C9
:1093E0003ECBBF003FEBB7003DCBBF003EEBB7002D
:1093F0003CCBBF003DEBB7003C6BEF001DF7EF002F
:10940000CE4802000000000067F2B70034938000ED
:109410004822DE00E359800004804100E0598800C2
:10942000F3598000E0814900F35988003ECBBF002A
:109430003FEBB7003DCBBF003EEBB7003CCBBF00DE
:109440003DEBB7003C6BEF001DF7EF00CE4802008C
:109450000000000068F2B700449380000960EF004C
:10946000E359800004804100E0598800F3598000EE
:10947000E0814900F35988003ECBBF003FEBB700C5
:109480003DCBBF003EEBB7003CCBBF003DEBB70090
:109490003C6BEF001DF7EF00CE480200000000001B
:1094A00069F2B700449380004822DE00E35980004F
:1094B00004804100E0598800F3598000E0814900B0
:1094C000F3598800E0598000F1598000000006003F
:1094D000851F7800861F7800D49280004822DE0025
:1094E0006524E1001A0039005F76EF0000C2B30086
:1094F00060F6B7000442020000000000082BEF00F5
:10950000F4FF200034588800050020000500780092
:10951000D6230200000000000040B3004220AF004C
:10952000050037008502E80062F6B700BA45020080
:1095300000000000F5FF3700400620008C3B0200D1
:109540000000000020C0B30000E0B70002023700B6
:10955000CA62A900C662A9002D28AE000B00370020
:109560000100200001007800F2230200000000004A
:109570008100E8003322AF00FEFF3700A011880011
:10958000600020000008E600F6FF37005F76EF007D
:1095900000C2B30060F6B700044202000000000001
:1095A000082BEF00F4FF200034588800050020004D
:1095B0000500780006240200000000000040B3000F
:1095C0004220AF00050037008502E80062F6B700D0
:1095D000BA45020000000000F5FF3700200320001C
:1095E0008C3B0200000000005B72EC00CA82A80005
:1095F000C682A900A0C0B3005AF2B700D49280007E
:10960000F4CFB20004003200AC48020000000000B9
:109610005A72ED00F9FF3700CA82A900C682A9007C
:1096200000C4B30014F7B7001637EF001837EF0087
:1096300050C9B30015F7B70014490200000000003C
:109640005CF2B7002D28AE00090037005CD2BF00E5
:109650000160EF00217022006E490200000000004E
:109660003322AF00FEFF370004022000A41188005F
:10967000E49280006124E10006003200CA62A80082
:10968000C662A900A00F20008C3B02000000000071
:1096900091FF370080C4B30014F7B7001637EF000E
:1096A00070C8B30015F7B700A41A2000C4B888002A
:1096B00014490200000000005CF2B7002D28AE0043
:1096C000140037000100200001007800202402006F
:1096D000000000008100E8003322AF00FEFF3700E9
:1096E000A0118800500020000008E600F6FF3700B7
:1096F0005CD2BF000160EF00217022006E490200C1
:10970000000000003322AF00FEFF370004022000FB
:10971000A4118800E49280006124E1002F003A0047
:109720001DF7EF00CE480200000000005CF2B70019
:109730001DF7EF00CE480200000000005CF2B70009
:109740001DF7EF00CE480200000000005EF2B700F7
:109750002D28AE00090037005ED2BF000160EF0087
:10976000217022006E490200000000003322AF0089
:10977000FEFF370004022000A41188001DF7EF004F
:10978000CE480200000000005FF2B7002D28AE00B6
:10979000090037005FD2BF000160EF002170220096
:1097A0006E490200000000003322AF00FEFF3700C8
:1097B00004022000A4118800F49280006124E100DA
:1097C00006003A00F49280004822DE00A4CAB200EB
:1097D00002003A0010C0B3005DF2B7005D52E20033
:1097E00012003A005F76EF0000C2B30060F6B700E7
:1097F000044202000000000005002000050078007F
:1098000036240200000000000040B3004220AF00F8
:10981000050037008502E80062F6B700BA4502008D
:1098200000000000F5FF3700B5003700A0C7B30007
:1098300065F2B700A4490200000000000093880010
:10984000119388002D28AE0017003700010020007A
:109850000100780050240200000000008100E800B0
:109860003322AF00FEFF3700A01188006000200007
:109870000008E600F6FF37001093800041702200D8
:109880006E49020000000000009380004170220039
:109890006E490200000000003322AF00FEFF3700D7
:1098A00004022000A411880000F02F006012B6000E
:1098B0008002780016938000F60FB20004002800A2
:1098C0000520E10003003A00F40F20000620E1002B
:1098D00001003200D5FF370070C7B30014F7B7009E
:1098E0001637EF001837EF0015F7EF0014490200A4
:1098F000000000005EF2B70090C6B30014F7B70096
:109900001837EF0015F7EF0004002400B4B8880002
:1099100014490200000000005FF2B700F4928000DA
:109920006224E100030039005F52E20001003200CE
:10993000E9FF3700A0C7B30065F2B700A4490200F1
:109940000000000000938800119388002D28AE00CD
:109950001700370001002000010078006824020091
:10996000000000008100E8003322AF00FEFF370056
:10997000A0118800600020000008E600F6FF370014
:1099800010938000417022006E4902000000000028
:1099900000938000417022006E4902000000000028
:1099A0003322AF00FEFF370004022000A41188001C
:1099B000846BEF0063C2AF00846BEC0000F02F00FB
:1099C0006012B6008002780016938000F60FB20095
:1099D000040028000520E10003003A00F40F2000F5
:1099E0000620E10001003200D2FF37002D28AE0032
:1099F00014003700010020000100780080240200DC
:109A0000000000008100E8003322AF00FEFF3700B5
:109A1000A0118800500020000008E600F6FF370083
:109A200084CBBF000160EF00217022006E4902006C
:109A3000000000003322AF00FEFF370004022000C8
:109A4000A4118800844BE20018003A00249380009F
:109A500043062000041CE100140039006472EC008D
:109A60005F76EF0000C2B30060F6B7000442020068
:109A70000000000005002000050078009624020088
:109A8000000000000040B3004220AF000500370096
:109A90008502E80062F6B700BA4502000000000047
:109AA000F5FF37008CFF370014003700245C80007E
:109AB0006124E10011003A005F76EF0000C2B300BC
:109AC00060F6B7000442020000000000050020001C
:109AD00005007800B0240200000000000040B30040
:109AE0004220AF00050037008502E80062F6B700AB
:109AF000BA45020000000000F5FF37002B003700D8
:109B0000A0C7B30065F2B700A4490200000000003E
:109B100000938800119388002D28AE0017003700AD
:109B20000100200001007800CA24020000000000AB
:109B30008100E8003322AF00FEFF3700A01188004B
:109B4000600020000008E600F6FF37001093800058
:109B5000417022006E490200000000000093800066
:109B6000417022006E490200000000003322AF0065
:109B7000FEFF370004022000A411880000F02F002F
:109B80006012B6008002780016938000F60FB200D3
:109B9000040028000520E10003003A00F40F200033
:109BA0000620E10001003200D5FF37005F76EF00AC
:109BB00050C0B30060F6B70004420200000000008D
:109BC00070C7B30014F7B7001637EF001837EF006F
:109BD00015F7EF0014490200000000005CF2B70026
:109BE00090C6B30014F7B7001837EF0015F7EF0071
:109BF00004002400B4B888001449020000000000EA
:109C00005CF2B7002D28AE001400370001002000E0
:109C100001007800E2240200000000008100E8005A
:109C20003322AF00FEFF3700A01188007000200033
:109C30000008E600F6FF37005CD2BF000160EF00CD
:109C4000217022006E490200000000003322AF00A4
:109C5000FEFF370004022000A4118800E492800077
:109C60006524E10002003A000600370003003700D7
:109C70005C52E20001003200CCFF37000060EF00D0
:109C8000350037002D28AE000B0037000100200002
:109C900001007800FA240200000000008100E800C2
:109CA0003322AF00FEFF3700A011880080002000A3
:109CB0000008E600F6FF37001DF7EF00CE4802006F
:109CC0000000000010C4B30014F7B7001637EF000F
:109CD0001837EF0015F7EF001449020000000000EC
:109CE0000004E000170032005F76EF0000C2B3000E
:109CF00060F6B700044202000000000005002000EA
:109D00000500780010250200000000000040B300AC
:109D10004220AF00050037008502E80062F6B70078
:109D2000BA45020000000000F5FF37005F76EF0043
:109D300080C2B30060F6B7000442020000000000D9
:109D4000D0FF37001DF7EF00CE48020000000000F2
:109D500010C0B30000E0B7004F037800CF027800D6
:109D600000000600851F780014D7BF001DF7B7005C
:109D7000CE4802000000000017D7BF008002780024
:109D80000B60EF00054078001DF7B700CE480200D9
:109D90000000000016D7BF001DF7B700CE48020034
:109DA0000000000019D7BF00800278000B60EF00B0
:109DB000054078001DF7B700CE4802000000000003
:109DC00018D7BF001DF7B700CE4802000000000002
:109DD00015D7BF001DF7B700CE48020000000000F5
:109DE0001DF7EF00CE48020000000000CF0278000F
:109DF00000000600851F7800844BE20007003A004F
:109E0000940020000402E8000402E900030032008C
:109E10000837D4000AB7D600FBFF37000817F80050
:109E20001217F9000A17F8000817F9000A37EF00AF
:109E30000817F8001017F900CA82A900C682A90005
:109E40001DF7EF00CE4802000000000000C5B3007F
:109E500014F7B7001637EF0015F7EF0004202000C5
:109E6000C4B8880014490200000000000004E000AB
:109E700001003200F2FF37001DF7EF00CE4802006C
:109E8000000000001DF7EF00CE48020000000000B7
:109E9000CA82A800C682A900CA82A900C682A900F7
:109EA00010C5B30014F7B70015F7EF001017F8004E
:109EB0001617F9001217F8001817F900B24E020031
:109EC000000000001DF7EF00CE4802000000000077
:109ED00007F7B7000757E20001003200F9FF37002B
:109EE0001DF7EF00CE48020000000000E40F200044
:109EF0000024E100FAFF3A000E37EF0074B880004A
:109F0000032020000418E1000900360060B880003A
:109F10000C37EC00800278001DF7EF00CE480200FD
:109F200000000000804A78000E37EC00F3FF370095
:109F30001DF7EF00CE48020000000000CA82A80012
:109F4000C682A9000060EF00CF0278000000060082
:109F5000851F7800C500200003000900B51F7800A8
:109F60000202B8000303B8004200A90085024300C2
:109F700060844B00020BB80085024B0008844B0044
:109F8000030BB800080443000780B0008701780085
:109F90000801780085007800040078002501200081
:109FA00003000900CF127800CF02780000000600FD
:109FB000851F7800C500200003000900B51F780048
:109FC000090020004300AF0019002000891F78001D
:109FD0000002EB008002EB000003EB008003EB00CB
:109FE0000304690011003200080220004200A900A9
:109FF0000080D2008180D2000482D2008582D2000B
:10A000000328E10001003A0002A0E100030039004A
:10A010000202520083825A004200A8000683D20046
:10A020008783D2000804E900F0FF3A008700780037
:10A0300006007800CF0478000900E000010032003B
:10A040000400BE002501200003000900CF127800A3
:10A05000CF02780000000600851F78000100200074
:10A060000100780026250200000000008100E800C1
:10A070003322AF00FEFF3700A011880070012000DE
:10A080000008E600F6FF3700CA82A900C682A900D0
:10A090001DF7EF00CE4802000000000000C5B3002D
:10A0A00014F7B7001637EF0015F7EF000420200073
:10A0B000C4B8880014490200000000000004E00059
:10A0C00001003200F2FF37001DF7EF00CE4802001A
:10A0D000000000001DF7EF00CE4802000000000065
:10A0E000CA82A800C682A9000837EF000A37EF002D
:10A0F000E425210064B88800FA4E02000000000048
:10A1000027D4BF005AF2B7005AD2BF0040EBB700C5
:10A11000416BEF00422BEF0042CBBF0043EBB70097
:10A1200041CBBF0042EBB70040CBBF0041EBB700D3
:10A13000406BEF0026D4BF005BF2B700D4928000E2
:10A140004822DE00035A800004804100005A880043
:10A15000135A8000E0814900135A880042CBBF00A7
:10A1600043EBB70041CBBF0042EBB70040CBBF0091
:10A1700041EBB700406BEF0025D4BF005CF2B700A5
:10A18000E49280000960EF00035A800004804100DF
:10A19000005A8800135A8000E0814900135A880051
:10A1A00042CBBF0043EBB70041CBBF0042EBB7004F
:10A1B00040CBBF0041EBB700406BEF0024D4BF00A1
:10A1C0005DF2B700E49280004822DE00035A80006E
:10A1D00004804100005A8800135A8000E081490041
:10A1E000135A88002D48AE001F00370001002000E0
:10A1F000010078004C250200000000008100E8000A
:10A200003322AF00FEFF3700A0118800500020006D
:10A210000008E600F6FF3700105A80004170220067
:10A220006E49020000000000005A800041702200C8
:10A230006E490200000000003322AF00FEFF37002D
:10A2400004022000A41188003322AF00FEFF370073
:10A25000A4002000A41188003322AF00FEFF3700C5
:10A26000D4002000A4118800400BF8000817F90062
:10A27000420BF8000A17F900E425210064B88800B1
:10A28000FA4E0200000000006AD2BF005AF2B70086
:10A290005AD2BF0048EBB700496BEF004A2BEF00E2
:10A2A0004ACBBF004BEBB70049CBBF004AEBB7002E
:10A2B00048CBBF0049EBB700486BEF0069D2BF0045
:10A2C0005BF2B700D49280004822DE00435A80003F
:10A2D00004804100405A8800535A8000E0814900C0
:10A2E000535A88002D28AE001F00370001002000BF
:10A2F0000100780066250200000000008100E800EF
:10A300003322AF00FEFF3700A0118800600020005C
:10A310000008E600F6FF3700505A80004170220026
:10A320006E49020000000000405A80004170220087
:10A330006E490200000000003322AF00FEFF37002C
:10A3400004022000A41188003322AF00FEFF370072
:10A35000A4002000A41188003322AF00FEFF3700C4
:10A36000D4002000A41188006BD2BF0030EBB700EE
:10A37000316BEF002D28AE001B00370001002000DC
:10A380000100780080250200000000008100E80044
:10A390003322AF00FEFF3700A011880080002000AC
:10A3A0000008E600F6FF3700805980004170220067
:10A3B0006E490200000000003322AF00FEFF3700AC
:10A3C00004022000A41188003322AF00FEFF3700F2
:10A3D000A4002000A41188003322AF00FEFF370044
:10A3E000D4002000A41188006DD2BF005AF2B7003B
:10A3F0005AD2BF0036EBB700376BEF0036CBBF0049
:10A4000037EBB700366BEF006CD2BF005BF2B700E2
:10A41000D49280004822DE00B359800004804100BD
:10A42000B05988002D28AE001B0037000100200025
:10A43000010078009C250200000000008100E80077
:10A440003322AF00FEFF3700A0118800500020002B
:10A450000008E600F6FF3700B05980004170220086
:10A460006E490200000000003322AF00FEFF3700FB
:10A4700004022000A41188003322AF00FEFF370041
:10A48000A4002000A41188003322AF00FEFF370093
:10A49000D4002000A41188006ED2BF0032EBB700B8
:10A4A000336BEF002D28AE001B00370001002000A9
:10A4B00001007800B6250200000000008100E800DD
:10A4C0003322AF00FEFF3700A011880050002000AB
:10A4D0000008E600F6FF3700905980004170220026
:10A4E0006E490200000000003322AF00FEFF37007B
:10A4F00004022000A41188003322AF00FEFF3700C1
:10A50000A4002000A41188003322AF00FEFF370012
:10A51000D4002000A4118800005A8000360BB4003B
:10A52000205A8800145A800060024A00345A880079
:10A530002D28AE001F003700010020000100780028
:10A54000D0250200000000008100E8003322AF00A7
:10A55000FEFF3700A0118800800020000008E60000
:10A56000F6FF3700305A8000417022006E49020029
:10A5700000000000205A8000417022006E49020055
:10A58000000000003322AF00FEFF3700040220006D
:10A59000A41188003322AF00FEFF3700A400200082
:10A5A000A41188003322AF00FEFF3700D400200042
:10A5B000A4118800205A8000315A8000425A80003D
:10A5C000535A8000A84F020000000000A05A8800E3
:10A5D000B15A88002D28AE001F003700010020006E
:10A5E00001007800EC250200000000008100E80076
:10A5F0003322AF00FEFF3700A0118800F0002000DA
:10A600000008E600F6FF3700B05A800041702200D3
:10A610006E49020000000000A05A80004170220034
:10A620006E490200000000003322AF00FEFF370039
:10A6300004022000A41188003322AF00FEFF37007F
:10A64000A4002000A41188003322AF00FEFF3700D1
:10A65000D4002000A411880075D2BF005AF2B700C0
:10A660005AD2BF0038EBB700396BEF0038CBBF00D0
:10A6700039EBB700386BEF0074D2BF005BF2B70064
:10A68000D49280004822DE00C3598000048041003B
:10A69000C05988002D28AE001B00370001002000A3
:10A6A0000100780010260200000000008100E80090
:10A6B0003322AF00FEFF3700A011880060002000A9
:10A6C0000008E600F6FF3700C05980004170220004
:10A6D0006E490200000000003322AF00FEFF370089
:10A6E00004022000A41188003322AF00FEFF3700CF
:10A6F000A4002000A41188003322AF00FEFF370021
:10A70000D4002000A411880070D2BF005AF2B70014
:10A710005AD2BF003AEBB7003B6BEF003ACBBF0019
:10A720003BEBB7003A6BEF006FD2BF005BF2B700B4
:10A73000D49280004822DE00D3598000048041007A
:10A74000D05988002D28AE001B00370001002000E2
:10A75000010078002A260200000000008100E800C5
:10A760003322AF00FEFF3700A011880090002000C8
:10A770000008E600F6FF3700D05980004170220043
:10A780006E490200000000003322AF00FEFF3700D8
:10A7900004022000A41188003322AF00FEFF37001E
:10A7A000A4002000A41188003322AF00FEFF370070
:10A7B000D4002000A41188008059800001002000EE
:10A7C000425A8000535A8000A84F02000000000047
:10A7D000E05A8800F15A88003A0BE2006A00320021
:10A7E000380BE20068003200010020000100780010
:10A7F00048260200000000008100E8003322AF007C
:10A80000FEFF3700A0118800700020000008E6005D
:10A81000F6FF3700AE6AA900C45980009359800042
:10A820000320B800245A800004004000205B880008
:10A83000345A80000300200004804900305B880007
:10A840002D28AE001F003700010020000100780015
:10A850005E260200000000008100E8003322AF0005
:10A86000FEFF3700A0118800A00020000008E600CD
:10A87000F6FF3700305B8000417022006E49020015
:10A8800000000000205B8000417022006E49020041
:10A89000000000003322AF00FEFF3700040220005A
:10A8A000A41188003322AF00FEFF3700A40020006F
:10A8B000A41188003322AF00FEFF3700D40020002F
:10A8C000A4118800D5598000C52ADD004300A900E5
:10A8D0000500780001002000425A8000535A800091
:10A8E000D84F020000000000245B800004004000FC
:10A8F000405B8800345B800004804800505B880027
:10A900002D28AE001F003700010020000100780054
:10A910007C260200000000008100E8003322AF0026
:10A92000FEFF3700A0118800D00020000008E600DC
:10A93000F6FF3700505B8000417022006E49020034
:10A9400000000000405B8000417022006E49020060
:10A95000000000003322AF00FEFF37000402200099
:10A96000A41188003322AF00FEFF3700A4002000AE
:10A97000A41188003322AF00FEFF3700D40020006E
:10A98000A411880037013700AE6AA80085D2BF0045
:10A990005AF2B7005AD2BF004CEBB7004D6BEF0034
:10A9A0004E2BEF004ECBBF004FEBB7004DCBBF009F
:10A9B0004EEBB7004CCBBF004DEBB7004C6BEF003C
:10A9C00084D2BF005BF2B700D49280004822DE0040
:10A9D000635A800004804100605A8800735A8000E6
:10A9E000E0814900735A88004ECBBF004FEBB7009F
:10A9F0004DCBBF004EEBB7004CCBBF004DEBB700CB
:10AA00004C6BEF0083D2BF005CF2B700E492800091
:10AA10000960EF00635A800004804100605A88009A
:10AA2000735A8000E0814900735A88004ECBBF0002
:10AA30004FEBB7004DCBBF004EEBB7004CCBBF0088
:10AA40004DEBB7004C6BEF0082D2BF005DF2B70058
:10AA5000E49280004822DE00635A800004804100B6
:10AA6000605A8800735A8000E0814900735A880058
:10AA70002D28AE001F0037000100200001007800E3
:10AA80009E260200000000008100E8003322AF0093
:10AA9000FEFF3700A0118800900020000008E600AB
:10AAA000F6FF3700705A8000417022006E490200A4
:10AAB00000000000605A8000417022006E490200D0
:10AAC000000000003322AF00FEFF37000402200028
:10AAD000A41188003322AF00FEFF3700A40020003D
:10AAE000A41188003322AF00FEFF3700D4002000FD
:10AAF000A41188008DD2BF005AF2B7005AD2BF000D
:10AB000050EBB700516BEF00522BEF0052CBBF0060
:10AB100053EBB70051CBBF0052EBB70050CBBF0097
:10AB200051EBB700506BEF008CD2BF005BF2B70067
:10AB3000D49280004822DE00835A800004804100C5
:10AB4000805A8800935A8000E0814900935A880017
:10AB500052CBBF0053EBB70051CBBF0052EBB70055
:10AB600050CBBF0051EBB700506BEF008BD2BF0052
:10AB70005CF2B700E49280000960EF00835A800025
:10AB800004804100805A8800935A8000E081490087
:10AB9000935A880052CBBF0053EBB70051CBBF0094
:10ABA00052EBB70050CBBF0051EBB700506BEF003A
:10ABB0008AD2BF005DF2B700E49280004822DE0036
:10ABC000835A800004804100805A8800935A800094
:10ABD000E0814900935A88002D28AE001F003700FD
:10ABE0000100200001007800BC26020000000000E7
:10ABF0008100E8003322AF00FEFF3700A01188007B
:10AC0000000120000008E600F6FF3700905A80009F
:10AC1000417022006E49020000000000805A80004E
:10AC2000417022006E490200000000003322AF0094
:10AC3000FEFF370004022000A41188003322AF0079
:10AC4000FEFF3700A4002000A41188003322AF00CB
:10AC5000FEFF3700D4002000A41188009059800026
:10AC6000010020000001780081017800605A800016
:10AC7000715A8000A84F020000000000205B88008D
:10AC8000315B8800205B8000440BB400205B8800AF
:10AC9000345A8000335B800004804900305B8800B8
:10ACA0002D28AE001F0037000100200001007800B1
:10ACB0005E260200000000008100E8003322AF00A1
:10ACC000FEFF3700A0118800A00020000008E60069
:10ACD000F6FF3700305B8000417022006E490200B1
:10ACE00000000000205B8000417022006E490200DD
:10ACF000000000003322AF00FEFF370004022000F6
:10AD0000A41188003322AF00FEFF3700A40020000A
:10AD1000A41188003322AF00FEFF3700D4002000CA
:10AD2000A4118800205B8000315B8000425A8000C3
:10AD3000535A8000A84F020000000000605B8800AA
:10AD4000715B88002D28AE001F0037000100200035
:10AD500001007800E0260200000000008100E80009
:10AD60003322AF00FEFF3700A0118800A0002000B2
:10AD70000008E600F6FF3700705B8000417022009B
:10AD80006E49020000000000605B800041702200FC
:10AD90006E490200000000003322AF00FEFF3700C2
:10ADA00004022000A41188003322AF00FEFF370008
:10ADB000A4002000A41188003322AF00FEFF37005A
:10ADC000D4002000A4118800205B8000300BB40068
:10ADD000405B8800345B800060024A00545B88005E
:10ADE0002D28AE001F003700010020000100780070
:10ADF0007C260200000000008100E8003322AF0042
:10AE0000FEFF3700A0118800D00020000008E600F7
:10AE1000F6FF3700505B8000417022006E4902004F
:10AE200000000000405B8000417022006E4902007B
:10AE3000000000003322AF00FEFF370004022000B4
:10AE4000A41188003322AF00FEFF3700A4002000C9
:10AE5000A41188003322AF00FEFF3700D400200089
:10AE6000A4118800640BF800600BF900660BF80071
:10AE7000620BF900445A800004A0B20002003A00BC
:10AE80004A0BE2000C0032000100200001007800B3
:10AE9000FE260200000000008100E8003322AF001F
:10AEA000FEFF3700A0118800800120000008E600A6
:10AEB000F6FF37000000FE00CF0278000000060019
:10AEC000851F78006072EF00042821002417880095
:10AED000E842A900E862A900E9C2A9000000000058
:10AEE00000000000000000000000000000CCB300E3
:10AEF00081F2B700343C02000000000000000000B6
:10AF00000000000000000000000000008428210074
:10AF1000241788000000000000000000000000006E
:10AF200000000000EC3C02000000000060F2B700EE
:10AF300010C0B30061F2B700049380004822DE0025
:10AF40007024E1000B003200EC3C02000000000025
:10AF500062F2B700049380004822DE0003B12000B3
:10AF60008302420062D2BF00804298006172EC000E
:10AF7000F1FF3700000000000000000000000000AA
:10AF800000000000E9C2A80004282100241788005E
:10AF900060D2BF0000E0B700CF02780000000600DA
:10AFA000851F7800861F7800E10820000000E0007F
:10AFB0001200320000F0A700040037004200A90090
:10AFC0000080D2008100E900FAFF37000180FD0017
:10AFD0004200A9008180D30000F0A1000080FD00A4
:10AFE000814068000040B20007003700014078004F
:10AFF0000170A0000140B200030037000000EB0028
:10B000008000EB00000037004F037800CF0278008B
:10B0100000000600851F7800C5002000030009001D
:10B02000B51F78008004EB00080028004300AF0043
:10B0300083016C00010578008A85690001037800AE
:10B0400083037800030678004220A9004200A9008B
:10B050000683D2000680FD00F60FB2000600E00075
:10B06000960032004220A9004200A9008783D20046
:10B070000780FD00F70FB2000700E00094003200E7
:10B080004220A9004200A9000638E10091003200E8
:10B09000980033000900A1000910A00006845300A5
:10B0A00007037800F10FB2000170A000F30FB200A7
:10B0B0000370A000870220000838E100110033006F
:10B0C0004220A9004200A9008180D3000080D30063
:10B0D0000804E900FAFF3A000D003700870220005B
:10B0E0000838E100090033004220A9004200A9000D
:10B0F0008381D3000281D3000804E900FAFF3A00FB
:10B100000F0037000200780083007800430037000A
:10B110000BF0A600110037000940A7008C0578004D
:10B120000000EA000200320081C0EA00010037009E
:10B130008100EA000940A7002B0037000700370014
:10B140000BF0A600050037000201EA000200320001
:10B1500083C1EA00010037008301EA00F50FB20065
:10B160004220A9004200A9000200400083C048001C
:10B170004200AF000930A0000900A7000900370015
:10B180000910A700010037000B0037000BF0A700E3
:10B19000150037000930A700290037000960A0001A
:10B1A0001E0037000BF0A7000F0037000930A70082
:10B1B00023003700190037000920A1000BF0A70079
:10B1C000040037008A0578000930A7001C0037000A
:10B1D0002B0037000940A00001C8B2000170A70091
:10B1E000CDFF37008A057800F10FB20081037000AF
:10B1F0000A0032000170A700080037004220A900B1
:10B200004200A9000080D2008180D2000603E9003C
:10B210004220AF0026003700F6FF37000900A700E4
:10B220008A0578000910A7008C0578000950A6004F
:10B230000F0037000AF0A7000080A00010003700C0
:10B240004200A80081C0D3000080D3004200AF00BC
:10B250000950A0000603E8000900A7008A0578004D
:10B260000910A7008C0578004220AF0010003700BD
:10B270000960A7008A0578000970A7008C0578008E
:10B2800001017000230032000170A1000680FD0062
:10B290004220A9004200A9000683D30081006B0070
:10B2A00001F0A0000BF0A60001F0A100190037008A
:10B2B0000000200001002000160037000AF0A7005F
:10B2C00083016C00020078008300780011003700D1
:10B2D00010003700F30FB2000370A000F10FB200AE
:10B2E0000170A0000BF0A7000370A1000920A000CE
:10B2F00093FF370007045300F10FB2000170A00064
:10B30000F30FB2000370A0000910A1000900A00013
:10B3100072FF37002501200003000900CF127800DA
:10B32000CF02780000000600851F7800C5002000CD
:10B3300004000900B51F78008004EB0083846800D6
:10B34000010378008002780003047800820378000B
:10B350008180D2000180FD008180FB000100E000BF
:10B360004E0032008381D2000380FD008381FB0008
:10B370000300E000490032000000EB0003C0500071
:10B3800003003900F047B0004400310003003700EB
:10B390001048B100410039004000320085007800BB
:10B3A000060178000270A000F20FB200F80FB200A0
:10B3B0000870A0009A0120008001EB000002EB0061
:10B3C000878050000801590002003300040031005A
:10B3D00004003A008780400008014900010037005E
:10B3E0000400A0000A05E900070032004200A9009D
:10B3F0008180D2000281D2004200A9000482D200E2
:10B400008381D200EEFF37000005EB000380A70028
:10B4100001003700060037004200A9008381D300F5
:10B420000370A1000482D3000A85D2000200370015
:10B430000000E900190032000AF0A70005003900F9
:10B440008180D2000281D20087805000080159001B
:10B45000090039000402E80007003A008301E8000F
:10B4600005003A000000E8000C003200020037003E
:10B470000000E900090032000080FD008080D30058
:10B4800001F0A00009F0A60001F0A1000370A100E6
:10B4900081C069000400780003003700000020002C
:10B4A00001002000000037004501200004000900D1
:10B4B000CF127800CF02780000000600851F7800C8
:10B4C00082017800820278004200A9008381D200C4
:10B4D0000380FD00F30FB2000338B000F207B200A2
:10B4E000360020000002EB004200A9000281D300D8
:10B4F0008180D3000080D3004200AF000402E80046
:10B500000603E900F8FF3A000270A100C419DD004B
:10B5100003F0A10005F0A70003F0A000830169007B
:10B52000010178008000780004007800CF027800E4
:10B5300000000600881F7800280120000400090090
:10B54000B81F78008005EB006066B800030478003F
:10B5500087047800FA7F20004200A9004220A90059
:10B5600044C4DE00080465000800E00070003200FA
:10B570004200A9004220A900C4CCDE008904650075
:10B580000900E0006A0032000884440009B0A70006
:10B5900004003700F83FB100650032006400390054
:10B5A000030037001A40200085424500600031004A
:10B5B000878669004200A9004220A900F300B2007A
:10B5C0000340A000F700B2000740A000881F7800E9
:10B5D0000124B800002DB8000A0544008B854C00FA
:10B5E0000C80B0000224B8008B0544000C864C008F
:10B5F000012CB8008B0544000C864C000034B800C8
:10B600000005EB008B0544000C864C000A80B0005E
:10B610008005EB000324B8000C0644000A854C00AA
:10B620000B80B000022CB8000C0644000A854C00C8
:10B630000B80B0000134B8000C0644000A854C00B1
:10B640000B80B000003CB8000C0644000A854C009A
:10B650000B80B0000C0078000006EB00032CB80053
:10B660000A0544008B854C000C80B0000234B80001
:10B670000A0544008B854C000C80B0000334B800F0
:10B680008B0544000C864C00013CB8000A054400C0
:10B690008B854C000C80B000023CB8008B05440048
:10B6A0000C864C00033CB8000C0644008A0078006D
:10B6B0000B0178008C017800540020004200A900A2
:10B6C0008381D3000281D3008180D3000080D30026
:10B6D0000402E900F9FF3A004F0478000804E8008A
:10B6E0000103700001003200020037000303710003
:10B6F000080032000340A700060037004200A900FE
:10B700000080D2008180D2000281D2008381D200E9
:10B710000804E9004444DD0003F0A1000DF0A70097
:10B7200003F0A0000340A10083016C000300370078
:10B730006000B8006001B80000003700A8012000D8
:10B74000040009004F1478004F0478000000060040
:10B75000881F7800891F78008A1F78008784690015
:10B7600009F0A600060037004200A9004220A90007
:10B7700003F0A600340037004200A8003200370072
:10B78000FA7F2000030478008704780044C4DE00B8
:10B7900008046500C4CCDE008904650008855400F7
:10B7A0000500320003F0A60027003700100020003B
:10B7B00042E0B600240037000304780087047800D4
:10B7C000F301B200F701B2000340A1000740A1005D
:10B7D00003C553000500320008F0A6001A00370028
:10B7E0001000200042E0B6001700370002055300A9
:10B7F0000500320008F0A6001300370010002000FA
:10B8000042E0B6001000370001855200050032000A
:10B8100008F0A6000C0037001000200042E0B6003F
:10B8200009003700000552000500320008F0A600AC
:10B83000050037001000200042E0B600020037008B
:10B840004200A900000037004F057800CF047800BF
:10B850004F04780000000600851F7800C500200016
:10B8600005000900B51F7800030478008203780002
:10B870000103780080027800830478003B472000B1
:10B88000C499DE00FA7F200083016500838555009E
:10B89000F801B2000840A0000000EB008000EB00BF
:10B8A0000001EB008001EB004200A9000884D300F6
:10B8B0008783D3000683D3008582D3008381D3009E
:10B8C0000281D3008180D3000080D3008B05E90082
:10B8D000F5FF3A0009F0A600050037000000EA0075
:10B8E0008180EA000281EA008381EA0000003700DB
:10B8F0006501200005000900CF127800CF02780012
:10B90000000006008C1F78008D1F78000004EB00FB
:10B910008004EB000005EB008005EB000006EB0067
:10B920008006EB00E8002000090020001000FA006B
:10B930000C377C000884E900FDFF3B0005046A0029
:10B9400002003A0007046B002F0032000004EB00F5
:10B950000D0420000D0420004200A9000080D20048
:10B960008180D2000281D2008381D2000884D2007B
:10B970008984D2000A85D2008B85D2000758E10065
:10B9800005003A0006D0E10003003A0005C8E100D6
:10B9900001003A0004C0E10005003900040454002D
:10B9A00085845C0006055D0087855D004200A80077
:10B9B000080F7800190798002A0798003B0798009D
:10B9C0004E049000DE0490006E059000FE0590008D
:10B9D0000884D2008984D2000A85D2008B85D200E7
:10B9E00048079800590798006A0798007B07980055
:10B9F0001E0478009E0490002E059000BE05900065
:10BA00008D06E900D4FF3A004E009000DE00900061
:10BA10006E019000FE0190000080FA0000003700E7
:10BA2000CF0678004F06780000000600851F7800DA
:10BA3000C500200007000900B51F78000900E000DC
:10BA4000130032002800FA00680220000006EB0014
:10BA50000C377C000884E900FDFF3B003917980093
:10BA6000470224000003EB006022B8002917980069
:10BA7000470224000003EB006022B8009A5A02003B
:10BA800000000000AE1490008904E900F7FF3A00BE
:10BA9000D71C240056D62C006022B800000F980056
:10BAA000110F9800220F9800330F980003F0A100A7
:10BAB000A85B0200000000004200AE000E0037004C
:10BAC0000E0890009E0890002E099000BE0990007C
:10BAD000A800200008179800A5B9230004A02C0096
:10BAE0006033B800440F9800550F9800660F980017
:10BAF000770F98000E0037000E0890009E08900007
:10BB00002E099000BE0990004801200008179800F7
:10BB100004002000859E28004630220077AC2800D3
:10BB2000440F9800550F9800660F9800770F980003
:10BB30000005780003F0A7004D0037000A007800E8
:10BB400003F0A1002C5C0200000000009E14900095
:10BB50008004EB00191798004E0A9000DE0A90004E
:10BB60006E0B9000FE0B90009E169000825C02000F
:10BB7000000000009E1690000D00A7002C0037006A
:10BB8000080F9800190F98002A0F9800310F98009D
:10BB90009E1690000D00A2001D1798009E169000A2
:10BBA0000D10A700060037009E1690000000E00070
:10BBB000130032009E1690000D10A0001D17980073
:10BBC0000E129000BE169000800278000D20E10059
:10BBD00005003A003D179800E0C2B30062F6B700D6
:10BBE000BA450200000000003D17980005007800EB
:10BBF0000003B00062F6B700BA4502000000000082
:10BC00008E1690008D06E9001E0032000D17980078
:10BC10004E089000DE0890006E099000FE0990002A
:10BC2000A40020008002EB006033B800CEFF370094
:10BC3000400F9800510F9800620F9800730F980002
:10BC40000002780081027800020378008303780004
:10BC50000E0890009E0890002E099000BE099000EA
:10BC60009E1690000D00A2001D179800BEFF370021
:10BC7000D0C2B30062F6B700BA450200000000006F
:10BC8000AFFF3700000000000080FA00A50120008F
:10BC900007000900CF127800CF02780000000600EC
:10BCA000851F7800861F7800871F7800881F78001E
:10BCB0005D72EF005E32EF002E3D020000000000DA
:10BCC000804278000040EB000AE0AF000000E8008E
:10BCD0000004E00002003A0000000000F6FF370018
:10BCE00040C1B30079F2B7007A72EF007B72EF00C7
:10BCF0007C72EF007D72EF007E72EF007F72EF00CA
:10BD00008072EF00703C0200000000002E3D020037
:10BD100000000000804278000040EB000AE0AF0025
:10BD20000000E8000004E00002003A00000000000B
:10BD3000F6FF370020C2B30079F2B7007A72EF0045
:10BD40007B72EF007C72EF007D72EF007E72EF007D
:10BD50007F72EF008072EF00703C02000000000074
:10BD60006057020000000000804278000040EB00B5
:10BD70000AE0AF000000E8000004E00003003A0021
:10BD8000CE07090000000000F5FF370012CBBF000E
:10BD900024EBB700256BEF0024CBBF0025EBB700E9
:10BDA000246BEF00945880004822DE002359800065
:10BDB000048041002059880020598000D05702009B
:10BDC0000000000080027800010378004300A90011
:10BDD0000500780086007800A2702D0033C2230091
:10BDE0000A58020000000000800378000104780077
:10BDF000070078008800780002002000832C2400CF
:10BE0000945902000000000090428800A14288007E
:10BE10002459800043062000110009000382D80045
:10BE20003059880034598000430620000320B800B0
:10BE300024598000000052004059880010C7B30008
:10BE40005FF6B7006076EF000442020000000000D9
:10BE5000082BEF00F4FF2000345888000000200079
:10BE600091428000A24280005E5A02000000000061
:10BE700019002000165D02000000000000C2B3009F
:10BE800062F6B700BA45020000000000240BF8007B
:10BE90002A0BF90030C2B30079F2B7007A72EF00D2
:10BEA0007B72EF007C72EF007D72EF007E72EF001C
:10BEB0007F72EF008072EF00703C02000000000013
:10BEC0006057020000000000804278000040EB0054
:10BED0000AE0AF000000E8000004E00002003A00C1
:10BEE00000000000F6FF370013EBAE000200370041
:10BEF00010C0B3005DF2B70040C6B3005FF6B700F4
:10BF00006076EF000442020000000000082BEF0002
:10BF1000F4FF200034588800E49280004822DE00BC
:10BF20006124E1000D003A000500200005007800C2
:10BF3000B6230200000000000040B3004220AF0022
:10BF4000050037008502E80062F6B700BA45020036
:10BF500000000000F5FF37000C003700050020004E
:10BF600005007800C6230200000000000040B30076
:10BF70004220AF00050037008502E80062F6B700F6
:10BF8000BA45020000000000F5FF37004F047800BA
:10BF9000CF0378004F037800CF027800000006003E
:10BFA0005F76EF005DD6BF0060F6B7000442020086
:10BFB000000000005E76EF00F4B280007B24E10018
:10BFC0000600320000C2B30062F6B700BA450200B4
:10BFD000000000005E76EC00F7FF3700000006006E
:10BFE0001970EF000570EF001870EF0002002000DC
:10BFF000E101210002007800583402000000000036
:10C00000805878000201E8000004E0004220AE0001
:10C01000F8FF37005172EF001230EF0002002000ED
:10C0200081022100020078006E340200000000004E
:10C03000805878000201E8000004E0004220AE00D1
:10C04000F8FF370002002000C11221000200780032
:10C05000A634020000000000805878000201E800C9
:10C060000004E0004220AE00F8FF3700020020008C
:10C070008116210002007800A634020000000000B2
:10C08000805878000201E8000004E0004220AE0081
:10C09000F8FF370002002000411A2100020078005A
:10C0A000A634020000000000805878000201E80079
:10C0B0000004E0004220AE00F8FF3700020020003C
:10C0C000011E210002007800A634020000000000DA
:10C0D000805878000201E8000004E0004220AE0031
:10C0E000F8FF370002002000A10A210002007800BA
:10C0F0006E34020000000000805878000201E80061
:10C100000004E0004220AE00F8FF370002002000EB
:10C11000A114210002007800A634020000000000F3
:10C12000805878000201E8000004E0004220AE00E0
:10C13000F8FF37000200200061182100020078009B
:10C14000A634020000000000805878000201E800D8
:10C150000004E0004220AE00F8FF3700020020009B
:10C16000211C210002007800A6340200000000001B
:10C17000805878000201E8000004E0004220AE0090
:10C18000F8FF370002002000E11F210002007800C4
:10C19000A634020000000000805878000201E80088
:10C1A0000004E0004220AE00F8FF370040C2B300B8
:10C1B00079F2B70020C0B3007AF2B7007B72EF00CB
:10C1C0007C72EF007D72EF007E72EF007F72EF00F5
:10C1D0008072EF00703C020000000000F96FEF0079
:10C1E0002232EF002432EF001C32EF001E32EF004B
:10C1F000F45580004822DE006124E1003400320062
:10C20000C0C1B3005DF6B700D05F020000000000BF
:10C2100040C2B3005DF6B700D05F0200000000002E
:10C22000A0C2B3005DF6B700D05F020000000000BE
:10C2300020C3B3005DF6B700D05F0200000000002D
:10C24000A0C3B3005DF6B700D05F0200000000009D
:10C2500020C4B3005DF6B700D05F0200000000000C
:10C26000A0C4B3005DF6B700D05F0200000000007C
:10C2700020C5B3005DF6B700D05F020000000000EB
:10C28000A0C5B3005DF6B700D05F0200000000005B
:10C2900020C6B3005DF6B700D05F020000000000CA
:10C2A000A0C6B3005DF6B700D05F0200000000003A
:10C2B00020C7B3005DF6B700D05F020000000000A9
:10C2C000A0C7B3005DF6B700D05F02000000000019
:10C2D00000000600851F7800861F7800871F780001
:10C2E000881F7800856BEF00AE6AAF000C00370046
:10C2F0000100200001007800482602000000000034
:10C300008100E8003322AF00FEFF3700A011880053
:10C31000700020000008E600F6FF37000901370032
:10C32000AE6AAE0007013700700BF800FC16F9008A
:10C33000720BF800FE16F9002D48AE001F00370002
:10C3400001002000010078003029020000000000F8
:10C350008100E8003322AF00FEFF3700A011880003
:10C36000300020000008E600F6FF3700F0B780003C
:10C37000417022006E49020000000000E0B780001A
:10C38000417022006E490200000000003322AF001D
:10C39000FEFF370004022000A41188003322AF0002
:10C3A000FEFF3700A4002000A41188003322AF0054
:10C3B000FEFF3700D4002000A41188007400200084
:10C3C0000960EF00E5B78000F6B780000402E800DE
:10C3D0000402E900030032000603D1008582D30085
:10C3E000FBFF370005007800440BB400C0B788009D
:10C3F000345A800004004B00D0B78800F816F800CB
:10C400000817F900FA16F8000A17F900444F21003E
:10C4100064B88800FA4E020000000000740020009A
:10C420000960EF00E5B78000F6B780000402E8007D
:10C430000402E900030032000603D1008582D30024
:10C44000FBFF3700740020000960EF000500780052
:10C45000860078000402E8000402E90003003200CC
:10C460000000D0008180D200FBFF3700E4B78000DD
:10C4700080035200F4B7800001045A0027B88800F6
:10C4800038B888000437D40006B7D6000437D40083
:10C4900006B7D6000417F800F416F9000617F800DE
:10C4A000F616F900B4B780006020E100A4003E0059
:10C4B00004003900A4B78000C31F20000418E10065
:10C4C0009F003900A4B78000630242008402780014
:10C4D000B4B7800060024A0004037800444F210092
:10C4E0000480420060034B00860078001040780012
:10C4F000EFF4B700EFD4BF0000F7B7000177EF000B
:10C500000237EF0002D7BF0003F7B70001D7BF0023
:10C5100002F7B70000D7BF0001F7B7000077EF00C0
:10C52000A4B780006202420084027800B4B78000A1
:10C5300060024A0004037800444F21000480420056
:10C5400060034B008600780010407800F0F4B700DC
:10C5500084A780000960EF0003B8800004804100D8
:10C5600000B8880013B88000E081490013B8880043
:10C5700002D7BF0003F7B70001D7BF0002F7B7002B
:10C5800000D7BF0001F7B7000077EF00A4B7800025
:10C590006102420084027800B4B7800060024A0061
:10C5A00004037800444F21000480420060034B00E4
:10C5B0008600780010407800F1F4B70084A780006E
:10C5C0004822DE0003B880000480410000B88800E3
:10C5D00013B88000E081490013B8880002D7BF007B
:10C5E00003F7B70001D7BF0002F7B70000D7BF00BD
:10C5F00001F7B7000077EF00444F2100A3B7800098
:10C6000004804100B4B7800060024A0084007800D2
:10C6100010407800F2F4B70094A780000960EF00A2
:10C6200003B880000480410000B8880013B880007F
:10C63000E081490013B8880004B88000F3FF2F00A0
:10C640000418E10006003A0014B88000F3FF20004F
:10C650000418E10002003A000060EF0039003700E2
:10C66000E4B780006102420004007800F4B7800063
:10C6700060024A00840078000017E30003003A00DB
:10C6800014B880000120E1002200320010C0B30085
:10C6900085EBB7002D48AE001B00370001002000DD
:10C6A0000100780048290200000000008100E80035
:10C6B0003322AF00FEFF3700A01188007000200079
:10C6C0000008E600F6FF370085CBBF000160EF00F1
:10C6D000217022006E49020000000000A10020002D
:10C6E0000100780048290200000000008100E800F5
:10C6F0003322AF00FEFF3700A0118800D0002000D9
:10C700000008E600F6FF370010C0B30000E0B700F5
:10C710000C0037000017F800FC16F9000217F800AB
:10C72000FE16F900A4B7800064024200A4B7880096
:10C73000B4B7800060024A00B4B7880059FF3700E0
:10C740001EFF37004F047800CF0378004F037800B6
:10C75000CF02780000000600851F7800F814F8006A
:10C76000FC14F900E0A780001004E0001200320081
:10C77000FA14F800FE14F900F0A780001004E0009D
:10C780000B003200E0A7800090427800F0A7800004
:10C7900010407800002CE10003003A00FC14F8007F
:10C7A0000000F90005003700FE34EC00F2FF37000E
:10C7B000FC34EC00EBFF37000020EF00CF027800E4
:10C7C00000000600851F780002002000214F210094
:10C7D00002007800922A02000000000080587800D1
:10C7E0000201E8000004E0004220AE00F8FF37003C
:10C7F000F014F800F614F900F014F800F814F90039
:10C80000244F2100D4A78800AC6302000000000080
:10C81000A0A78800A0A78000F014E30002003A005F
:10C82000F034EC0022003700F414E20016003A0065
:10C8300080A780001004E00007003200B0A780004D
:10C84000F634EC008002780080A78000F034EC0021
:10C85000904A7800F6FF3700F634ED00B0A780006C
:10C860001042780004C2B20003003A00B5A780006D
:10C87000804AEB0003003700F634EC00B5A78000D7
:10C88000804AEB000A003700A0A78000F014E30004
:10C8900007003200B0A78000F634EC008002780078
:10C8A00080A78000F034EC00904A7800F6FF370053
:10C8B000F414E200D0FF3A00F614F800F014F90086
:10C8C000CF02780000000600851F7800861F7800E0
:10C8D0000001EB000103780064C110004211DD008B
:10C8E0000200DD00800278000C60EC000C60ED00BE
:10C8F0000D00320005007800C42ADD004C00DE0087
:10C90000F000B2000003B000A20320000200E1002A
:10C91000010039000D40B40062F6B700BA450200CC
:10C9200000000000F1FF37004F037800CF027800CD
:10C9300000000600851F780075A78000C82ADE0069
:10C94000C32ADD005F76EF000540780060F6B7008F
:10C950000442020000000000F074EF0084A7800091
:10C960007B24E1000600320000C2B30062F6B7008B
:10C97000BA45020000000000F074EC00F7FF370039
:10C98000CF02780000000600851F78004555E200C0
:10C990001D00320030AA80009042780040AA80003A
:10C9A00010407800002CE1000C00320030AA80001A
:10C9B0009042780040AA800010407800002CE100EE
:10C9C0000200310000C0EB000100370010C0B300CE
:10C9D00000E0B7000D0037000500370030AA8000E6
:10C9E0001004E00002003A000060EF00070037008A
:10C9F00030AA80004635EC0040AA80004835EC00A3
:10CA00004575ED00E1FF37000060EF00CF027800D0
:10CA1000000006000100200001007800D82C020070
:10CA2000000000008100E8003322AF00FEFF370065
:10CA3000A0118800F00020000008E600F6FF370093
:10CA4000AE0AA90002002000014F21000200780078
:10CA5000F62C020000000000805878000201E80077
:10CA60000004E0004220AE00F8FF37000200200082
:10CA7000414F210002007800062D02000000000056
:10CA8000805878000201E8000004E0004220AE0077
:10CA9000F8FF370002002000814F210002007800DB
:10CAA000162D020000000000805878000201E80006
:10CAB0000004E0004220AE00F8FF37000200200032
:10CAC000C14F210002007800262D02000000000066
:10CAD000805878000201E8000004E0004220AE0027
:10CAE000F8FF37000200200001502100020078000A
:10CAF000362D020000000000805878000201E80096
:10CB00000004E0004220AE00F8FF370002002000E1
:10CB10004150210002007800462D02000000000074
:10CB2000805878000201E8000004E0004220AE00D6
:10CB3000F8FF370002002000815021000200780039
:10CB4000562D020000000000805878000201E80025
:10CB50000004E0004220AE00F8FF37000200200091
:10CB6000C150210002007800662D02000000000084
:10CB7000805878000201E8000004E0004220AE0086
:10CB8000F8FF370002002000015121000200780068
:10CB9000762D020000000000805878000201E800B5
:10CBA0000004E0004220AE00F8FF37000200200041
:10CBB0004151210002007800862D02000000000093
:10CBC000805878000201E8000004E0004220AE0036
:10CBD000F8FF370002002000815121000200780098
:10CBE000962D020000000000805878000201E80045
:10CBF0000004E0004220AE00F8FF370002002000F1
:10CC0000C151210002007800A62D020000000000A2
:10CC1000805878000201E8000004E0004220AE00E5
:10CC2000F8FF3700020020000152210002007800C6
:10CC3000B62D020000000000805878000201E800D4
:10CC40000004E0004220AE00F8FF370002002000A0
:10CC50004152210002007800C62D020000000000B1
:10CC6000805878000201E8000004E0004220AE0095
:10CC7000F8FF3700020020008152210002007800F6
:10CC8000D62D020000000000805878000201E80064
:10CC90000004E0004220AE00F8FF37000200200050
:10CCA000C152210002007800E62D020000000000C1
:10CCB000805878000201E8000004E0004220AE0045
:10CCC000F8FF370020C0B30045F5B700E4C72000E7
:10CCD00034AA8800044F210044AA8800C4640200DA
:10CCE00000000000ADEEB70020C0B30045F5B7006E
:10CCF000E4C7200034AA8800444F210044AA8800D9
:10CD0000C464020000000000AEEEB70020C0B30013
:10CD100045F5B700E4C7200034AA8800844F2100FD
:10CD200044AA8800C464020000000000AFEEB7000F
:10CD300020C0B30045F5B700E4C7200034AA88003E
:10CD4000C44F210044AA8800C4640200000000000F
:10CD5000B0EEB70020C0B30045F5B700E4C720002F
:10CD600034AA88000450210044AA8800C464020048
:10CD700000000000B1EEB70020C0B30045F5B700D9
:10CD8000E4C7200034AA88004450210044AA880047
:10CD9000C464020000000000B2EEB70020C0B3007F
:10CDA00045F5B700E4C7200034AA8800845021006C
:10CDB00044AA8800C464020000000000B3EEB7007B
:10CDC00020C0B30045F5B700E4C7200034AA8800AE
:10CDD000C450210044AA8800C4640200000000007E
:10CDE000B4EEB70020C0B30045F5B700E4C720009B
:10CDF00034AA88000451210044AA8800C4640200B7
:10CE000000000000B5EEB70020C0B30045F5B70044
:10CE1000E4C7200034AA88004451210044AA8800B5
:10CE2000C464020000000000B6EEB70020C0B300EA
:10CE300045F5B700E4C7200034AA880084512100DA
:10CE400044AA8800C464020000000000B7EEB700E6
:10CE500020C0B30045F5B700E4C7200034AA88001D
:10CE6000C451210044AA8800C464020000000000EC
:10CE7000B8EEB70020C0B30045F5B700E4C7200006
:10CE800034AA88000452210044AA8800C464020025
:10CE900000000000B9EEB70020C0B30045F5B700B0
:10CEA000E4C7200034AA88004452210044AA880024
:10CEB000C464020000000000BAEEB70020C0B30056
:10CEC00045F5B700E4C7200034AA88008452210049
:10CED00044AA8800C464020000000000BBEEB70052
:10CEE00020C0B30045F5B700E4C7200034AA88008D
:10CEF000C452210044AA8800C4640200000000005B
:10CF0000BCEEB700AD4EE20016003A00447580005A
:10CF10006A24E10013003A00447580004822DE00D4
:10CF20006124E1000F003A00AE0AA800BE2EA8005E
:10CF30000100200001007800F62D02000000000032
:10CF40008100E8003322AF00FEFF3700A011880007
:10CF5000100120000008E600F6FF3700A62EA8000A
:10CF6000AD013700AE4EE20012003A004475800079
:10CF70006624E1000F003A00AE0AA800BE2EA80009
:10CF80000100200001007800162E020000000000C1
:10CF90008100E8003322AF00FEFF3700A0118800B7
:10CFA000100120000008E600F6FF3700A64EA8009A
:10CFB00099013700AE4EE20012003A00447580003D
:10CFC0006624E1000F003A00AE0AA800BE2EA800B9
:10CFD0000100200001007800162E02000000000071
:10CFE0008100E8003322AF00FEFF3700A011880067
:10CFF000100120000008E600F6FF3700A64EA8004A
:10D0000085013700AE4EE20012003A004475800000
:10D010006624E1000F003A00AE0AA800BE2EA80068
:10D020000100200001007800162E02000000000020
:10D030008100E8003322AF00FEFF3700A011880016
:10D04000100120000008E600F6FF3700A64EA800F9
:10D0500071013700AE4EE20012003A0044758000C4
:10D060006624E1000F003A00AE0AA800BE2EA80018
:10D070000100200001007800162E020000000000D0
:10D080008100E8003322AF00FEFF3700A0118800C6
:10D09000100120000008E600F6FF3700A64EA800A9
:10D0A0005D013700AF4EE20016003A004475800083
:10D0B0006C24E10013003A00447580004822DE0031
:10D0C0006124E1000F003A00AE0AA800BE2EA800BD
:10D0D0000100200001007800362E02000000000050
:10D0E0008100E8003322AF00FEFF3700A011880066
:10D0F000F00020000008E600F6FF3700A66EA8004A
:10D1000045013700B04EE20016003A004475800039
:10D110006224E10013003A00447580004822DE00DA
:10D120007924E1000F003A00AE0AA800BE2EA80044
:10D130000100200001007800542E020000000000D1
:10D140008100E8003322AF00FEFF3700A011880005
:10D15000100120000008E600F6FF3700A68EA800A8
:10D160002D013700B14EE20016003A0044758000F0
:10D170006D24E10013003A00447580004822DE006F
:10D180007124E1000F003A00AE0AA800BE2EA800EC
:10D190000100200001007800742E02000000000051
:10D1A0008100E8003322AF00FEFF3700A0118800A5
:10D1B000F00020000008E600F6FF3700A6AEA80049
:10D1C00015013700B24EE20016003A0044758000A7
:10D1D0006924E10013003A00447580004822DE0013
:10D1E0006924E1000F003A00AE0AA800BE2EA80094
:10D1F0000100200001007800922E020000000000D3
:10D200008100E8003322AF00FEFF3700A011880044
:10D21000100120000008E600F6FF3700A6CEA800A7
:10D22000FD003700B34EE20016003A00447580005E
:10D230006624E10013003A00447580004822DE00B5
:10D240007124E1000F003A00AE0AA800BE2EA8002B
:10D250000100200001007800B22E02000000000052
:10D260008100E8003322AF00FEFF3700A0118800E4
:10D27000100120000008E600F6FF3700A6EEA80027
:10D28000E5003700B44EE20012003A004475800019
:10D290006F24E1000F003A00AE0AA800BE2EA800DD
:10D2A0000100200001007800D22E020000000000E2
:10D2B0008100E8003322AF00FEFF3700A011880094
:10D2C000000120000008E600F6FF3700BD0EA800B0
:10D2D000D1003700B54EE20012003A0044758000DC
:10D2E0006D24E1000F003A00AE0AA800BE2EA8008F
:10D2F0000100200001007800F02E02000000000074
:10D300008100E8003322AF00FEFF3700A011880043
:10D31000100120000008E600F6FF3700BD2EA8002F
:10D32000BD003700B64EE20016003A00447580009A
:10D330006524E10013003A00447580004822DE00B5
:10D340006124E1000F003A00AE0AA800BE2EA8003A
:10D350000100200001007800102F020000000000F2
:10D360008100E8003322AF00FEFF3700A0118800E3
:10D37000F00020000008E600F6FF3700BD4EA800D0
:10D38000A5003700B74EE20012003A004475800055
:10D390006824E1000F003A00AE0AA800BE2EA800E3
:10D3A00001002000010078002E2F02000000000084
:10D3B0008100E8003322AF00FEFF3700A011880093
:10D3C000500120000008E600F6FF3700BD6EA800FF
:10D3D00091003700B84EE20016003A004475800014
:10D3E0006F24E10013003A00447580004822DE00FB
:10D3F00014C3B2000F003A00AE0AA800BE2EA80067
:10D400000100200001007800522F020000000000FF
:10D410008100E8003322AF00FEFF3700A011880032
:10D42000000120000008E600F6FF3700BD8EA800CE
:10D4300079003700B94EE20016003A0044758000CA
:10D440006E24E10013003A00447580004822DE009B
:10D450007124E1000F003A00AE0AA800BE2EA80019
:10D460000100200001007800702F02000000000081
:10D470008100E8003322AF00FEFF3700A0118800D2
:10D48000F00020000008E600F6FF3700BDAEA8005F
:10D4900061003700BA4EE20016003A004475800081
:10D4A0006E24E10013003A00447580004822DE003B
:10D4B00014C2B2000F003A00AE0AA800BE2EA800A7
:10D4C00001002000010078008E2F02000000000003
:10D4D0008100E8003322AF00FEFF3700A011880072
:10D4E000000120000008E600F6FF3700BDCEA800CE
:10D4F00049003700BB4EE20016003A004475800038
:10D500006424E10013003A00447580004822DE00E4
:10D510006924E1000F003A00AE0AA800BE2EA80060
:10D520000100200001007800AC2F02000000000084
:10D530008100E8003322AF00FEFF3700A011880011
:10D54000500120000008E600F6FF3700BDEEA800FD
:10D5500031003700BC4EE20016003A0044758000EE
:10D560006C24E10013003A00447580004822DE007C
:10D570006A24E1000F003A00AE0AA800BE2EA800FF
:10D580000100200001007800D02F02000000000000
:10D590008100E8003322AF00FEFF3700A0118800B1
:10D5A000E00020000008E600F6FF3700BE0EA800ED
:10D5B00019003700BC4EE20016003A0044758000A6
:10D5C0006C24E10013003A00447580004822DE001C
:10D5D0006724E1000F003A00AE0AA800BE2EA800A2
:10D5E0000100200001007800EC2F02000000000084
:10D5F0008100E8003322AF00FEFF3700A011880051
:10D60000C00020000008E600F6FF3700BE0EA800AC
:10D6100001003700AE0AA90000000600861F78004E
:10D62000871F7800881F7800891F78000002EB00B0
:10D630008002EB000003EB008003EB0003046900B1
:10D6400011003200080220004200A9000080D20030
:10D650008180D2000482D2008582D2000328E100BA
:10D6600001003A0002A0E10003003900020252006A
:10D6700083825A004200A8000683D2008783D2002A
:10D680000804E900F0FF3A008700780006007800FF
:10D69000CF0478004F047800CF0378004F03780060
:10D6A00000000600851F7800C50020000300090067
:10D6B000B51F780000037800810378000406780025
:10D6C00004F0A1000400E00006003A0009F0A70001
:10D6D000020037000500200013003700050020007D
:10D6E00011003700EB4252000E0039000003200009
:10D6F00009F0A600000220003322AF00FEFF370031
:10D70000A011880041E0AF00FBFF370080108800C7
:10D710001162EF008502E900F7FF3B005500200091
:10D720000100370084027800E80020000900200092
:10D730001000FA000C377C000884E900FDFF3B0074
:10D74000A400200005E0A0000CF0A70005F0A00058
:10D75000040F78001507980006007800870078000D
:10D7600002A02C00A3B92300087122000DF0A10033
:10D770000DF0A2000E6B0200000000000DF0A700EB
:10D780000700370040079800510798000001780013
:10D79000810178002E009000BE009000F4FF370059
:10D7A000420798005307980024079800350798000F
:10D7B0001E0278009E029000060320000000E00098
:10D7C00012003A0005E0A600120037000402E9004A
:10D7D000040F78000400E0000E0032000524E10090
:10D7E000020032004200AF000E00370006032000A6
:10D7F0000000E00005003A0005E0A6000500370043
:10D8000005F0A600060220000200370005E0A10096
:10D8100015079800004043003322AF00FEFF370099
:10D82000A01188004E009000DE009000A2002000B1
:10D830008001EB006100E10001003200CCFF370005
:10D840000080FA002501200003000900CF127800B3
:10D85000CF02780000000600851F7800861F780040
:10D86000871F7800881F78002D48AE000B00370016
:10D8700001002000010078002427020000000000C1
:10D880008100E8003322AF00FEFF3700A0118800BE
:10D89000400020000008E600F6FF370001002000ED
:10D8A0000100780036270200000000008100E80037
:10D8B0003322AF00FEFF3700A01188006000200077
:10D8C0000008E600F6FF37008874EF006428EF00D8
:10D8D0006628EF005168EF005A68EF007234EF00DD
:10D8E0007434EF005E68EF00149380006124E1005F
:10D8F00016003A005F76EF0000C7B30060F6B7008D
:10D90000044202000000000005002000050078002D
:10D910004A270200000000000040B3004220AF0090
:10D92000050037008502E80062F6B700BA4502003C
:10D9300000000000F5FF37005F76EF0080C7B300FE
:10D9400060F6B70004420200000000002D48AE005F
:10D950000B00370001002000010078006227020060
:10D96000000000008100E8003322AF00FEFF370016
:10D97000A0118800400020000008E600F6FF3700F4
:10D98000AE6AAE0008003700440BF8006E14F900D0
:10D99000460BF8007014F900500BF8007614F900EB
:10D9A000520BF8007814F900640BF8008414F900A5
:10D9B000660BF8008614F9007E34EF008034EF0027
:10D9C000AE6AAE000700370020A48000300BB40020
:10D9D00070A4880034A4800060024A0084A48800F7
:10D9E00011003700AE6AAF000F003700D559800034
:10D9F000C52ADD004300A9000500780001002000D1
:10DA0000425A8000535A8000D84F020000000000A4
:10DA100024A480000400400070A4880034A4800086
:10DA20000480480080A488008414F8006A14F90077
:10DA30008614F8006C14F90050A380008E14E300E3
:10DA400003003A0060A380009014E3009E063200B9
:10DA50002D48AE006700370001002000010078006B
:10DA600074270200000000008100E8003322AF00AC
:10DA7000FEFF3700A0118800900020000008E6009B
:10DA8000F6FF370060A38000417022006E4902005B
:10DA90000000000050A38000417022006E49020087
:10DAA000000000003322AF00FEFF37000402200018
:10DAB000A4118800010020000100780090270200D6
:10DAC000000000008100E8003322AF00FEFF3700B5
:10DAD000A0118800700020000008E600F6FF370063
:10DAE000E0A38000417022006E49020000000000A7
:10DAF000D0A38000417022006E49020000000000A7
:10DB00003322AF00FEFF370004022000A41188007A
:10DB10000100200001007800AA2702000000000098
:10DB20008100E8003322AF00FEFF3700A01188001B
:10DB3000800020000008E600F6FF370000A4800007
:10DB4000417022006E49020000000000F0A3800036
:10DB5000417022006E490200000000003322AF0035
:10DB6000FEFF370004022000A411880088D4BF0003
:10DB70000160EF004200DD00044A21000400400083
:10DB8000900278001003900001002000010078004E
:10DB9000C4270200000000008100E8003322AF002B
:10DBA000FEFF3700A0118800800020000008E6007A
:10DBB000F6FF370006007800417022006E4902002F
:10DBC0000000000005007800417022006E4902004C
:10DBD000000000003322AF00FEFF3700A400200049
:10DBE000A41188003322AF00FEFF3700D4002000CC
:10DBF000A4118800D4A3800004A0B20004003A005D
:10DC00007C14E20002003A007E34EF008034EF0022
:10DC10006A14F8000817F9006C14F8000A17F900E4
:10DC2000A426210064B88800FA4E0200000000001B
:10DC30007E14F8007A14F9008014F8007C14F900BE
:10DC4000D4A3800004A0B20002003A007C14E200D9
:10DC500019063200A4262100D3A3800004804100CD
:10DC6000E4A3800060024A008400780004082000D9
:10DC70001024E10011003E002D48AE000D003700D9
:10DC80000500200005007800E027020000000000E9
:10DC90000040B3004220AF00060037008502E800D4
:10DCA0003322AF00FEFF370034E2B7003562EF00E9
:10DCB000F4FF3700F8053700D5023700D4A3800001
:10DCC0006B02420084027800E4A3800060024A00F4
:10DCD00004037800A42621000480420060034B0066
:10DCE00086007800104078006C4060006C04E10011
:10DCF00011003A002D48AE000D003700050020004D
:10DD000005007800F2270200000000000040B30088
:10DD10004220AF00060037008502E8003322AF0042
:10DD2000FEFF370034E2B7003562EF00F4FF370042
:10DD3000D9053700B6023700D4A380006B02420039
:10DD400084027800E4A3800060024A0004037800A3
:10DD5000A42621000480420060034B008600780066
:10DD6000104078007C4060007004E1004E023A00F0
:10DD7000A4262100D3A3800004804100E4A38000F6
:10DD800060024A008400780010427800E4C2B200C9
:10DD900001003A00C00537006252E20002003A007A
:10DDA0005F68EC0011003700149380006224E100EA
:10DDB0000E003A005E68EC005DC8BF005E48E300FC
:10DDC0000A003A0024438000610242004443880074
:10DDD0003443800060024A00544388002DA8A90003
:10DDE00010C0B30062F2B700B7FE370088D4BF009E
:10DDF0000160EF004200DD00044A2100840240007F
:10DE00007A94BF00800298007C94BF009002980032
:10DE100088D4BF000160EF004200DD00844C210087
:10DE2000840240006A94BF00800298006C94BF0096
:10DE3000900298008874EC005168EC0084428000E5
:10DE40004822DE00C3BA20008302420088D4BF000B
:10DE5000804298005A68EF0002002000214921000A
:10DE600002007800042802000000000080587800BA
:10DE70000201E8000004E0004220AE00F8FF370095
:10DE80006872EF00449380006824E10012003200C1
:10DE9000449380000960EF0023492100830242007F
:10DEA000449380000960EF00D3A380000483410005
:10DEB000E3A38000E081490083037800A4262100C9
:10DEC00004004300E0834B0087007800904A78000C
:10DED0006872EC00EBFF37004E6EEF00E1C72000E8
:10DEE00022492100B24878003104E0004220AE000F
:10DEF000FCFF3700E4C7200084A78800E26302002B
:10DF0000000000000100200001007800122802003B
:10DF1000000000008100E8003322AF00FEFF370060
:10DF2000A0118800400020000008E600F6FF37003E
:10DF3000E1C720001104E000070032003322AF00E7
:10DF4000FEFF37001140780034E2B7003562EF0081
:10DF50008100E800F7FF3700710020000100780021
:10DF600012280200000000008100E8003322AF0008
:10DF7000FEFF3700A0118800D00020000008E60056
:10DF8000F6FF370044A480006124E1000A00390054
:10DF900088D4BF0089F4B7008954E200060032003B
:10DFA0003322AF00FEFF3700E4022000A4118800F6
:10DFB0008974ED00F8FF37003322AF00FEFF370011
:10DFC000C4052000A4118800214921001104E000AB
:10DFD000070032003322AF00FEFF37001140780007
:10DFE00034E2B7003562EF008100E800F7FF370048
:10DFF0003322AF00FEFF370004022000A411880086
:10E000003322AF00FEFF3700A4002000A4118800D7
:10E010003322AF00FEFF3700D4002000A411880097
:10E02000149380006324E100EB003A005D48E200B5
:10E0300002003A0010C0B3005DE8B7005E68EC0073
:10E040005DC8BF00F44280000024E1009A0039005E
:10E0500044A480006124E100200039000200200077
:10E06000214921000200780004280200000000007D
:10E07000805878000201E8000004E0004220AE0071
:10E08000F8FF37006872EF00449380006824E100D5
:10E0900012003200449380000960EF002349210000
:10E0A00083024200449380000960EF00D3A3800004
:10E0B00004834100E3A38000E081490083037800EA
:10E0C000A426210004004300E0834B008700780071
:10E0D000904A78006872EC00EBFF37002D48AE00E4
:10E0E0001800370001002000010078002E280200EF
:10E0F000000000008100E8003322AF00FEFF37007F
:10E10000A0118800500020000008E600F6FF37004C
:10E110006CC8BF000160EF0004002000FA47020055
:10E12000000000003322AF00FEFF37000402200091
:10E13000A41188003322AF00FEFF37000402200044
:10E14000A41188002D48AE001A0037003322AF001A
:10E15000FEFF3700C4052000A411880021492100DA
:10E160001104E000070032003322AF00FEFF370049
:10E170001140780034E2B7003562EF008100E8001A
:10E18000F7FF37003322AF00FEFF37000402200004
:10E19000A41188003322AF00FEFF3700A400200046
:10E1A000A41188003322AF00FEFF3700D400200006
:10E1B000A411880065438000C32ADD005F76EF006C
:10E1C0000540780060F6B70004420200000000003D
:10E1D0006C48E20003003A00F4FF20004458880035
:10E1E000062BEF002D48AE000B0037000100200089
:10E1F0000100780046280200000000008100E800CD
:10E200003322AF00FEFF3700A0118800500020002D
:10E210000008E600F6FF37005DC8BF006C48B40098
:10E220000080FB0064B82000040040001043780028
:10E23000064078000160EF00217022006464020053
:10E240000000000088D4BF0089F4B7008954E200C0
:10E2500006003200E0C2B30062F6B700BA45020021
:10E26000000000008974ED00F8FF3700C0C5B3005E
:10E2700062F6B700BA450200000000002149210003
:10E280001104E00008003200811F7800114078007E
:10E2900062F6B700BA45020000000000CF00780027
:10E2A0008100E800F6FF3700082BEF00F4FF2000A4
:10E2B000345888006C68EC00E44280004822DE009C
:10E2C000634242000440780000E0B7005E48E3008B
:10E2D000030032005EC8BF005F48E3003E003A0022
:10E2E0002D48AE000B00370001002000010078002F
:10E2F0005A280200000000008100E8003322AF002D
:10E30000FEFF3700A0118800500020000008E60042
:10E31000F6FF37005F76EF0000C4B30060F6B70089
:10E320000442020000000000050020000500780003
:10E330006E280200000000000040B3004220AF0041
:10E34000050037008502E80062F6B700BA45020012
:10E3500000000000F5FF37002D48AE000B0037002D
:10E360000100200001007800802802000000000069
:10E370008100E8003322AF00FEFF3700A0118800C3
:10E38000500020000008E600F6FF370086CBBF00F3
:10E390000160EF00217022006464020000000000B0
:10E3A0002D48AE000B00370001002000010078006E
:10E3B00094280200000000008100E8003322AF0032
:10E3C000FEFF3700A0118800500020000008E60082
:10E3D000F6FF37003C063700149380006124E1000B
:10E3E00002003A0051C8BF005DE8B7002D48AE00FA
:10E3F0000B0037000100200001007800A82802006F
:10E40000000000008100E8003322AF00FEFF37006B
:10E41000A0118800400020000008E600F6FF370049
:10E42000D4A380007502420084027800E4A3800037
:10E4300060024A0004037800A42621000480420000
:10E4400060034B00860078001040780063F2B7004C
:10E4500063D2BF008AF4B7008B74EF008C34EF00F6
:10E460008CD4BF008DF4B7008BD4BF008CF4B70000
:10E470008AD4BF008BF4B7008A74EF00D4A3800065
:10E480007402420084027800E4A3800060024A0023
:10E4900004037800A42621000480420060034B009E
:10E4A000860078001040780064F2B7002493800062
:10E4B0000960EF0053A480000480410050A488004C
:10E4C00063A48000E081490063A488008CD4BF006D
:10E4D0008DF4B7008BD4BF008CF4B7008AD4BF0092
:10E4E0008BF4B7008A74EF00D4A380007B02420053
:10E4F00084027800E4A3800060024A0004037800EC
:10E50000A42621000480420060034B0086007800AE
:10E510001040780065F2B700249380004822DE00A6
:10E5200053A480000480410050A4880063A48000AC
:10E53000E081490063A488008CD4BF008DF4B7004B
:10E540008BD4BF008CF4B7008AD4BF008BF4B70023
:10E550008A74EF00D4A380007A024200840278001B
:10E56000E4A3800060024A0004037800A42621008E
:10E570000480420060034B00860078001040780061
:10E5800066F2B700349380000960EF0053A4800066
:10E590000480410050A4880063A48000E081490009
:10E5A00063A4880054A480006200520050A4880034
:10E5B00064A4800060005A0060A48800010020006C
:10E5C00001007800BA280200000000008100E80085
:10E5D0003322AF00FEFF3700A0118800700020003A
:10E5E0000008E600F6FF370060A4800041702200BA
:10E5F0006E4902000000000050A48000417022001B
:10E600006E490200000000003322AF00FEFF370019
:10E6100004022000A41188003322AF00FEFF37005F
:10E62000A4002000A41188003322AF00FEFF3700B1
:10E63000D4002000A411880050A4800061A48000B0
:10E640008259800003002000A84F02000000000053
:10E6500020A4880031A4880020A48000680BB400A6
:10E6600020A48800545B800033A48000048049000B
:10E6700030A48800AE6AAE000700370024A48000F2
:10E68000835980000300520020A4880034A4800035
:10E6900060005A0030A488007E34EF008034EF0020
:10E6A000C7FC37005A003700A4262100D3A38000FE
:10E6B00004804100E4A3800060024A0084007800E6
:10E6C0001004E00052003A0044A480006124E100FC
:10E6D000390039002D48AE000D003700050020003C
:10E6E00005007800D6280200000000000040B300BA
:10E6F0004220AF00060037008502E8003322AF0059
:10E70000FEFF370034E2B7003562EF00F4FF370058
:10E710008874ED00D44280006142420004407800D9
:10E720005AE8B70088D4BF000160EF004200DD0066
:10E73000044A210004004000901F78007E14F90074
:10E740001000900080B4B70088D4BF000160EF00D3
:10E750004200DD00844C210004004000901F78003E
:10E760008414F9001000900086B4B7000402200061
:10E77000F3A3800004804100F0A3880004A480007B
:10E7800060024A0004A48800F4A3800004A0B20040
:10E7900007003A008014E20005003A008434EC00DF
:10E7A0004220AF008634EC007E34EF008034EF006E
:10E7B00083FC3700160037008854E20014003A004A
:10E7C0002D28AE000D003700050020000500780060
:10E7D000E8280200000000000040B3004220AF0023
:10E7E000060037008502E8003322AF00FEFF370045
:10E7F00034E2B7003562EF00F4FF370000C2B30027
:10E80000EFF4B7009A640200000000002E05370004
:10E81000D4A380006802420084027800E4A3800050
:10E8200060024A0004037800A4262100048042000C
:10E8300060034B00860078001040780069F2B70052
:10E84000D4A380006902420084027800E4A380001F
:10E8500060024A0004037800A426210004804200DC
:10E8600060034B00860078001040780082F4B70007
:10E87000D4A380006A02420084027800E4A38000EE
:10E8800060024A0004037800A426210004804200AC
:10E8900060034B00860078001040780083F4B700D6
:10E8A000449380004822DE00A4C6B2000C0032006F
:10E8B000449380004822DE00A4C4B2000800320065
:10E8C000449380004822DE0044C6B20004003200B7
:10E8D000449380004822DE0044C4B200EE023A00B5
:10E8E00014A4800004C7B2000900320014A4800000
:10E8F00004C5B2000600320014A4800014C6B200A1
:10E900000300320014A4800014C4B200E2023A00F2
:10E9100014A480004822DE0074C6B2000C0032004D
:10E9200014A480004822DE0074C4B2000800320043
:10E9300014A480004822DE0044C7B2000400320064
:10E9400014A480004822DE0044C5B200D2023A007E
:10E950006252E200D4013A006028EC004220AF008D
:10E960006228EC008854E2001A0032005A48E200A3
:10E970000D003200844280004822DE00D342800035
:10E98000034052000080FB00C4BA20000400400095
:10E990001040780044A480000024E100020031000F
:10E9A0005A68EC00F3FF3700844280004822DE0002
:10E9B000D3428000034052000080FB0064B8200076
:10E9C000040340001642780061424200044398006C
:10E9D000060037008854E20004003A00345C8000EE
:10E9E000614242000440780086EBB7000A650200ED
:10E9F000000000000043800011438000040020005C
:10EA0000526B0200000000003322AF00FEFF37000F
:10EA100004022000A4118800A4262100D3A38000B2
:10EA200004804100E4A3800060024A008400780072
:10EA3000904278003322AF00FEFF37000540780097
:10EA400034E2B7003562EF00D4A3800061024200D7
:10EA500084027800E4A3800060024A000403780086
:10EA6000A42621000480420060034B008600780049
:10EA7000904378003322AF00FEFF37000740780054
:10EA800034E2B7003562EF00D4A380006202420096
:10EA900084027800E4A3800060024A000403780046
:10EAA000A42621000480420060034B008600780009
:10EAB000904378003322AF00FEFF37000740780014
:10EAC00034E2B7003562EF00D4A380006302420055
:10EAD00084027800E4A3800060024A000403780006
:10EAE000A42621000480420060034B0086007800C9
:10EAF000904378003322AF00FEFF370007407800D4
:10EB000034E2B7003562EF00D4A380006402420013
:10EB100084027800E4A3800060024A0004037800C5
:10EB2000A42621000480420060034B008600780088
:10EB3000904378003322AF00FEFF37000740780093
:10EB400034E2B7003562EF00D4A3800065024200D2
:10EB500084027800E4A3800060024A000403780085
:10EB6000A42621000480420060034B008600780048
:10EB7000904378003322AF00FEFF37000740780053
:10EB800034E2B7003562EF00D4A380006602420091
:10EB900084027800E4A3800060024A000403780045
:10EBA000A42621000480420060034B008600780008
:10EBB000904378003322AF00FEFF37000740780013
:10EBC00034E2B7003562EF00D4A380006702420050
:10EBD00084027800E4A3800060024A000403780005
:10EBE000A42621000480420060034B0086007800C8
:10EBF000904378003322AF00FEFF370007407800D3
:10EC000034E2B7003562EF003322AF00FEFF370079
:10EC100004022000A41188003322AF00FEFF370059
:10EC2000A4002000A41188003322AF00FEFF3700AB
:10EC3000D4002000A4118800AE0AAE0019013700EC
:10EC4000D4A380007502420084027800E4A380000F
:10EC500060024A0004037800A426210004804200D8
:10EC600060034B00860078001040780063F2B70024
:10EC700063D2BF0042EEB700436EEF00442EEF00B8
:10EC800044CEBF0045EEB70043CEBF0044EEB70010
:10EC900042CEBF0043EEB700426EEF00D4A3800027
:10ECA0007402420084027800E4A3800060024A00FB
:10ECB00004037800A42621000480420060034B0076
:10ECC000860078001040780064F2B700249380003A
:10ECD0000960EF0013728000048041001072880008
:10ECE00023728000E08149002372880044CEBF0077
:10ECF00045EEB70043CEBF0044EEB70042CEBF00A2
:10ED000043EEB700426EEF00D4A380007B024200C6
:10ED100084027800E4A3800060024A0004037800C3
:10ED2000A42621000480420060034B008600780086
:10ED30001040780065F2B700249380004822DE007E
:10ED400013728000048041001072880023728000DA
:10ED5000E08149002372880044CEBF0045EEB70031
:10ED600043CEBF0044EEB70042CEBF0043EEB70033
:10ED7000426EEF00D4A380007A0242008402780041
:10ED8000E4A3800060024A0004037800A426210066
:10ED90000480420060034B00860078001040780039
:10EDA00066F2B700349380000960EF0013728000B0
:10EDB000048041001072880023728000E0814900C5
:10EDC000237288004ECEBF000160EF004200DD00DC
:10EDD00024C9200084024000428EBF0080029800B7
:10EDE000448EBF00900298004ECEBF000160EF003D
:10EDF0004200DD0024C9200004004000901F78007C
:10EE00004A0EF900100090004CAEB700547280001A
:10EE1000E20252006472800060035A00050078002C
:10EE2000860078008259800003002000A84F02006D
:10EE3000000000003072880041728800307280004B
:10EE4000680BB40030728800545B8000437280000D
:10EE50000480490040728800AE6AAE0007003700A7
:10EE600034728000835980000300520030728800A1
:10EE70004472800060005A00407288004ECEBF008D
:10EE80000160EF004200DD00E4CF2000840240007A
:10EE9000468EBF0080029800488EBF009002980006
:10EEA000D4A380007F02420084027800E4A38000A3
:10EEB00060024A0004037800A42621000480420076
:10EEC00060034B00860078001040780063F2B700C2
:10EED00063D2BF0042EEB700436EEF00442EEF0056
:10EEE00044CEBF0045EEB70043CEBF0044EEB700AE
:10EEF00042CEBF0043EEB700426EEF00D4A38000C5
:10EF00007E02420084027800E4A3800060024A008E
:10EF100004037800A42621000480420060034B0013
:10EF2000860078001040780064F2B70024938000D7
:10EF30000960EF00137280000480410010728800A5
:10EF400023728000E08149002372880044CEBF0014
:10EF500045EEB70043CEBF0044EEB70042CEBF003F
:10EF600043EEB700426EEF00D4A380007D02420062
:10EF700084027800E4A3800060024A000403780061
:10EF8000A42621000480420060034B008600780024
:10EF90001040780065F2B700249380004822DE001C
:10EFA0001372800004804100107288002372800078
:10EFB000E08149002372880044CEBF0045EEB700CF
:10EFC00043CEBF0044EEB70042CEBF0043EEB700D1
:10EFD000426EEF00D4A380007C02420084027800DD
:10EFE000E4A3800060024A0004037800A426210004
:10EFF0000480420060034B008600780010407800D7
:10F0000066F2B700349380000960EF00137280004D
:10F01000048041001072880023728000E081490062
:10F02000237288004ECEBF000160EF004200DD0079
:10F03000A4D6200084024000428EBF0080029800C7
:10F04000448EBF00900298004ECEBF000160EF00DA
:10F050004200DD0024C9200004004000901F780019
:10F06000700BF9001000900072ABB7006A610200EB
:10F07000000000004ECEBF000160EF004200DD0046
:10F0800064DD20008402400085CBBF00804A780008
:10F0900000C0B30080429800040020009402980051
:10F0A0004E6EEC00FC003700149380006124E100F8
:10F0B000F3003A006428EC004220AF006628EC0020
:10F0C000404380006408E300EC003A0050438000B5
:10F0D0006608E300E9003A0080C2B300EFF4B7002D
:10F0E0009A64020000000000D4A380007502420070
:10F0F00084027800E4A3800060024A0004037800E0
:10F10000A42621000480420060034B0086007800A2
:10F110001040780063F2B70063D2BF0070EBB70015
:10F12000716BEF00722BEF0072CBBF0073EBB70077
:10F1300071CBBF0072EBB70070CBBF0071EBB700B3
:10F14000706BEF00D4A38000740242008402780048
:10F15000E4A3800060024A0004037800A426210092
:10F160000480420060034B00860078001040780065
:10F1700064F2B700249380000960EF00835B800095
:10F1800004804100805B8800935B8000E08149003F
:10F19000935B880072CBBF0073EBB70071CBBF00ED
:10F1A00072EBB70070CBBF0071EBB700706BEF0074
:10F1B000D4A380007B02420084027800E4A3800094
:10F1C00060024A0004037800A42621000480420063
:10F1D00060034B00860078001040780065F2B700AD
:10F1E000249380004822DE00835B8000048041007D
:10F1F000805B8800935B8000E0814900935B88001E
:10F2000072CBBF0073EBB70071CBBF0072EBB700DE
:10F2100070CBBF0071EBB700706BEF00D4A3800020
:10F220007A02420084027800E4A3800060024A006F
:10F2300004037800A42621000480420060034B00F0
:10F24000860078001040780066F2B70034938000A2
:10F250000960EF00835B800004804100805B8800D0
:10F26000935B8000E0814900935B8800845B8000B1
:10F27000E2025200945B800060035A0080598000D3
:10F28000010020000001780081017800050078006D
:10F2900086007800A84F020000000000905E880001
:10F2A000A15E8800905E8000680BB400905E8800CC
:10F2B000545B8000A35E800004804900A05E88004B
:10F2C000AE6AAE0007003700945E8000835980006C
:10F2D00003005200905E8800A45E800060005A0027
:10F2E000A05E8800D4A380007F02420084027800E0
:10F2F000E4A3800060024A0004037800A4262100F1
:10F300000480420060034B008600780010407800C3
:10F3100063F2B70063D2BF0078EBB700796BEF0000
:10F320007A2BEF007ACBBF007BEBB70079CBBF0025
:10F330007AEBB70078CBBF0079EBB700786BEF00C2
:10F34000D4A380007E02420084027800E4A38000FF
:10F3500060024A0004037800A426210004804200D1
:10F3600060034B00860078001040780064F2B7001C
:10F37000249380000960EF00C35B8000048041009B
:10F38000C05B8800D35B8000E0814900D35B8800CC
:10F390007ACBBF007BEBB70079CBBF007AEBB7002D
:10F3A00078CBBF0079EBB700786BEF00D4A3800077
:10F3B0007D02420084027800E4A3800060024A00DB
:10F3C00004037800A42621000480420060034B005F
:10F3D000860078001040780065F2B7002493800022
:10F3E0004822DE00C35B800004804100C05B8800CF
:10F3F000D35B8000E0814900D35B88007ACBBF00FB
:10F400007BEBB70079CBBF007AEBB70078CBBF00BE
:10F4100079EBB700786BEF00D4A380007C02420048
:10F4200084027800E4A3800060024A0004037800AC
:10F43000A42621000480420060034B00860078006F
:10F440001040780066F2B700349380000960EF0046
:10F45000C35B800004804100C05B8800D35B8000F8
:10F46000E0814900D35B880000C2B300EFF4B7002D
:10F470009A64020000000000130237000600370003
:10F48000149380006224E10003003A006428EC0039
:10F490004220AF006628EC0004022000D3A38000C5
:10F4A00004804100D0A38800E4A3800060024A00E9
:10F4B000E4A38800E2F937006A34EC004220AF0090
:10F4C0006C34EC005CF9370024A48000035B8000FE
:10F4D0008302520034A48000135B800003035A00AF
:10F4E0008059800001002000140020000960EF0016
:10F4F0000402E8000402E900030032000000D0002A
:10F500008180D200FBFF370085034000068448005D
:10F5100080598000010020004300A900000178000C
:10F52000810178000700780088007800D84F020039
:10F5300000000000B0A38800C1A38800AE6AAF003D
:10F540001A003700140020000960EF00405A8000C4
:10F55000515A80000402E8000402E900030032006E
:10F560008100D1000080D300FBFF37004300A900D9
:10F570000001780081017800B0A38000C1A3800061
:10F58000D84F0200000000008002780001037800DC
:10F5900005007800440BB40070A38800345A800042
:10F5A00004004B0080A388001B003700AE6AAE0049
:10F5B00019003700240020000960EF00405A800045
:10F5C000515A80000402E8000402E90003003200FE
:10F5D0008100D1000080D300FBFF37004300A90069
:10F5E0000001780081017800B0A38000C1A38000F1
:10F5F000D84F02000000000080027800010378006C
:10F6000005007800440BB40070A38800345A8000D1
:10F6100004004B0080A38800AE6AAF00B50037003D
:10F6200001002000010078004826020000000000D0
:10F630008100E8003322AF00FEFF3700A0118800F0
:10F64000700020000008E600F6FF37006E14F80096
:10F650000817F9007014F8000A17F900A426210011
:10F6600064B88800FA4E02000000000077D4BF00A2
:10F670008002780078D4BF000BE0B70079D4BF00D7
:10F68000000378000D60EF000640780003E0B7004B
:10F690000BE0B700804078000540780001E0B7003B
:10F6A0000040EB00B4A3800080035200C4A380009C
:10F6B00001045A00D7A38800E8A388007A34D40054
:10F6C0007CB4D600D4A3800061024200840278009A
:10F6D000E4A3800060024A0004037800A42621000D
:10F6E0000480420060034B008600780010407800E0
:10F6F00063F2B70063D2BF0072F4B7007374EF0017
:10F700007434EF0074D4BF0075F4B70073D4BF0035
:10F7100074F4B70072D4BF0073F4B7007274EF00D2
:10F72000A4262100D3A3800004804100E4A380002C
:10F7300060024A00840078001040780064F2B7004C
:10F74000249380000960EF0093A3800004804100AF
:10F7500090A38800A3A38000E0814900A3A38800B0
:10F76000A4A380006020E1006200390004003E0094
:10F7700094A3800003FF2F000418E1005D003E0009
:10F780002D48AE001F003700010020000100780066
:10F79000FA280200000000008100E8003322AF00D8
:10F7A000FEFF3700A0118800B00020000008E6002E
:10F7B000F6FF3700A0A38000417022006E490200CE
:10F7C0000000000090A38000417022006E490200FA
:10F7D000000000003322AF00FEFF370004022000CB
:10F7E000A41188003322AF00FEFF3700A4002000E0
:10F7F000A41188003322AF00FEFF3700D4002000A0
:10F80000A4118800140020000960EF00405A800015
:10F81000515A80000402E8000402E90003003200AB
:10F820008100D1000080D300FBFF37004300A90016
:10F83000000178008101780090A38000A1A38000DE
:10F84000D84F020000000000800278000103780019
:10F8500005007800440BB40070A38800345A80007F
:10F8600004004B0080A388007214F8007614F9009D
:10F870007414F8007814F900805980000100200009
:10F880000001780081017800B0A38000C1A380004E
:10F89000A84F0200000000008002780001037800F9
:10F8A00005007800600BB400800378000600780043
:10F8B000628BB400000478008059800001002000B1
:10F8C000140020000960EF000402E8000402E900CF
:10F8D000030032000000D0008180D200FBFF37001F
:10F8E0000080530020A4880001005C0030A4880040
:10F8F00033F83700AE6AAE00F30037000100200095
:10F90000010078001A290200000000008100E800D0
:10F910003322AF00FEFF3700A011880070002000E6
:10F920000008E600F6FF37006E14F8000817F9002B
:10F930007014F8000A17F900A426210064B88800A2
:10F94000FA4E020000000000740020000960EF0081
:10F95000B5A38000C6A380000402E8000402E90009
:10F96000030032000603D1008582D300FBFF37007D
:10F97000740020000960EF00050078008600780020
:10F980000402E8000402E900030032000000D00095
:10F990008180D200FBFF3700B4A3800080035200B7
:10F9A000C4A3800001045A00D7A38800E8A38800FC
:10F9B0007A34D4007CB4D6007A34D4007CB4D60037
:10F9C000D4A380006302420084027800E4A3800094
:10F9D00060024A0004037800A4262100048042004B
:10F9E00060034B00860078001040780063F2B70097
:10F9F00063D2BF0072F4B7007374EF007434EF0089
:10FA000074D4BF0075F4B70073D4BF0074F4B700AA
:10FA100072D4BF0073F4B7007274EF00D4A38000F7
:10FA20006202420084027800E4A3800060024A007F
:10FA300004037800A42621000480420060034B00E8
:10FA4000860078001040780064F2B70024938000AC
:10FA50000960EF0093A380000480410090A3880018
:10FA6000A3A38000E0814900A3A3880074D4BF0051
:10FA700075F4B70073D4BF0074F4B70072D4BF003C
:10FA800073F4B7007274EF00D4A3800061024200E7
:10FA900084027800E4A3800060024A000403780036
:10FAA000A42621000480420060034B0086007800F9
:10FAB0001040780065F2B700249380004822DE00F1
:10FAC00093A380000480410090A38800A3A380003A
:10FAD000E0814900A3A3880074D4BF0075F4B70087
:10FAE00073D4BF0074F4B70072D4BF0073F4B700CE
:10FAF0007274EF00A4262100D3A38000048041008B
:10FB0000E4A3800060024A0084007800104078007E
:10FB100066F2B700349380000960EF0093A3800081
:10FB20000480410090A38800A3A38000E0814900E5
:10FB3000A3A3880094A38000F3FF2F000418E10022
:10FB400004003A00A4A38000F3FF20000418E100A1
:10FB50005D0032002D48AE001F003700010020007C
:10FB600001007800FA280200000000008100E8008F
:10FB70003322AF00FEFF3700A0118800B000200044
:10FB80000008E600F6FF3700A0A3800041702200C5
:10FB90006E4902000000000090A380004170220026
:10FBA0006E490200000000003322AF00FEFF370064
:10FBB00004022000A41188003322AF00FEFF3700AA
:10FBC000A4002000A41188003322AF00FEFF3700FC
:10FBD000D4002000A4118800240020000960EF0058
:10FBE000405A8000515A80000402E8000402E900F3
:10FBF000030032008100D1000080D300FBFF3700FA
:10FC00004300A900000178008101780090A38000E2
:10FC1000A1A38000D84F02000000000080027800FD
:10FC20000103780005007800440BB40070A388003D
:10FC3000345A800004004B0080A388007214F8003E
:10FC40007614F9007414F8007814F90080598000D3
:10FC5000010020000001780081017800B0A380003D
:10FC6000C1A38000A84F02000000000080027800BD
:10FC70000103780005007800600BB4008003780071
:10FC800006007800628BB400000478008059800080
:10FC900001002000140020000960EF000402E800C9
:10FCA0000402E900030032000000D0008180D2008D
:10FCB000FBFF37000080530020A4880001005C0097
:10FCC00030A488003EF737004F047800CF03780057
:10FCD0004F037800CF02780000000600851F7800EF
:10FCE000861F7800A62EA900A64EA900A66EA90020
:10FCF000A68EA900A6AEA900A6CEA900A6EEA900D0
:10FD0000BD0EA900BD2EA900BD4EA900BD6EA90063
:10FD1000BD8EA900BDAEA900BDCEA900BDEEA90053
:10FD2000BE0EA90001002000010078008C2B02000B
:10FD3000000000008100E8003322AF00FEFF370022
:10FD4000A0118800B00020000008E600F6FF370090
:10FD500010C0B30062F2B7001C47020000000000B0
:10FD600064E0270014B38800423F02000000000056
:10FD7000903F020000000000ABEEB700BE3F020063
:10FD800000000000547580004822DE00F4CFB2006D
:10FD900002003A00A86EEF0002003700ABCEBF00B1
:10FDA000A8EEB70074E0270014B38800423F0200B9
:10FDB00000000000903F020000000000ACEEB70021
:10FDC000BE3F02000000000064758000F4CFB20066
:10FDD00002003A00A96EEF0002003700ACCEBF006F
:10FDE000A9EEB7000100200001007800A62B020058
:10FDF000000000008100E8003322AF00FEFF370062
:10FE0000A0118800F00020000008E600F6FF37008F
:10FE1000A8CEBF000160EF00217022006E490200F1
:10FE2000000000002101200001007800A62B020044
:10FE3000000000008100E8003322AF00FEFF370021
:10FE4000A0118800600120000008E600F6FF3700DE
:10FE5000A9CEBF000160EF00217022006E490200B0
:10FE6000000000003322AF00FEFF37000402200034
:10FE7000A41188003322AF00FEFF3700A400200049
:10FE8000A41188003322AF00FEFF3700D400200009
:10FE9000A41188006A610200000000006272EF0095
:10FEA0002C6C0200000000002D28AE001C00370062
:10FEB0000100200001007800D02B020000000000AB
:10FEC0008100E8003322AF00FEFF3700A011880058
:10FED000C00020000008E600F6FF37000043800065
:10FEE0001143800044002000526B0200000000001B
:10FEF0003322AF00FEFF370004022000A411880067
:10FF00003322AF00FEFF3700A4002000A4118800B8
:10FF10003322AF00FEFF3700D4002000A411880078
:10FF20003322AF00FEFF370004022000A411880036
:10FF30003322AF00FEFF3700A4002000A411880088
:10FF40003322AF00FEFF3700D4002000A411880048
:10FF50005C68EF005CC8BF00844280004822DE007D
:10FF60000024E10032003900010020000100780087
:10FF7000F22B0200000000008100E8003322AF00F5
:10FF8000FEFF3700A0118800A00020000008E60056
:10FF9000F6FF37005CC8BF000160EF00217022004F
:10FFA0006E490200000000003322AF00FEFF370060
:10FFB000D4032000A41188003322AF00FEFF3700D5
:10FFC00004022000A4118800E44280000960EF00D0
:10FFD00063B8200003004200904278000B60EF00FD
:10FFE000060020000500780086007800440020000C
:10FFF000526B0200000000003322AF00FEFF37000A
:020000040001F9
:1000000004022000A41188003322AF00FEFF370055
:10001000A4002000A41188003322AF00FEFF3700A7
:10002000D4002000A41188005C68EC00C9FF3700F0
:100030000100200001007800102C020000000000E8
:100040008100E8003322AF00FEFF3700A0118800D6
:10005000A00020000008E600F6FF37005FC8BF00E0
:100060000160EF00217022006E49020000000000D4
:100070003322AF00FEFF370004022000A4118800E5
:100080003322AF00FEFF3700A4002000A411880037
:100090003322AF00FEFF3700D4002000A4118800F7
:1000A0004F037800CF02780000000600851F78001B
:1000B000C500200003000900B51F780000F0A6006D
:1000C000020037000000EA000480A0008002EB007C
:1000D000800378008404780004F0A1000404E000A8
:1000E00006003A0009F0A7000200370005002000D2
:1000F0000F003700050020000D003700E6425200D7
:100100000A0039000003200009F0A60000022000C8
:100110003322AF00FEFF3700A01188008502E900FE
:10012000FBFF3B00550020000100370084027800EF
:100130006400200005E0A00009F0A70005F0A00081
:1001400008712200110009008883D800EA800200AB
:100150000000000081037800883E200011000900A3
:100160008883D800EA800200000000008103780044
:1001700048062000110009008883D800EA800200A8
:100180000000000081037800A80020001100090091
:100190008883D800EA800200000000000980A600E1
:1001A00005003700D00220003322AF00FEFF3700E9
:1001B000A01188000980A1000003200000C04000B9
:1001C000500188003322AF00FEFF3700A0118800E5
:1001D00020003700060320000000E0000E003A0077
:1001E00005E0A600160037000402E9000524E1003E
:1001F000020032004200AF00000006000000E000F4
:1002000005003A0005E0A6000D00370005F0A60045
:10021000060220000A00370005E0A1000980A600C0
:100220000700370000057800D00220003322AF001D
:10023000FEFF3700A01188000980A1000A007800A5
:10024000004043003322AF00FEFF3700A0118800BA
:10025000000006002501200003000900CF127800ED
:10026000CF02780000000600811F780041808000E6
:10027000805878008048EB00CF0078000830EC0010
:1002800000000600851F7800C5002000030009005B
:10029000B51F780000F0A600020037000000EA0059
:1002A0000480A0008002EB008003780084047800C2
:1002B00004F0A1000404E00006003A0009F0A700E1
:1002C0000200370005002000100037000500200064
:1002D0000E003700E64252000B00390000032000F8
:1002E00009F0A60000022000801F78004F0078006F
:1002F00034810200000000008502E900FAFF3B00A3
:1003000055002000010037008402780064002000BE
:1003100005E0A00009F0A70005F0A0000871220088
:10032000110009008883D800DC8102000000000071
:1003300081037800883E2000110009008883D800DE
:10034000DC810200000000008103780048062000E4
:10035000110009008883D800DC8102000000000041
:1003600081037800A8002000110009008883D800CC
:10037000DC810200000000000980A60006003700B2
:10038000D0022000801F78004F00780034810200E6
:10039000000000000980A1000003200000C0400010
:1003A00050018800801F78004F00780034810200DF
:1003B0000000000022003700060320000000E000DB
:1003C0000E003A0005E0A600170037000402E9001D
:1003D0000524E100020032004200AF0000000600E8
:1003E0000000E00005003A0005E0A6000E0037001E
:1003F00005F0A600060220000B00370005E0A10072
:100400000980A6000800370000057800D00220000F
:10041000801F78004F007800348102000000000047
:100420000980A1000A00780000404300801F780086
:100430004F00780034810200000000000000060038
:100440002501200003000900CF127800CF027800B8
:1004500000000600851F78003E15F8004415F900DD
:100460004015F8003E15F9004035EF003E15F80044
:100470004215F900CA82A900C682A9001DF7EF0043
:10048000CE4802000000000000C5B30014F7B7001A
:100490001637EF0014002000C4B8880015F7EF00ED
:1004A00014490200000000000004E00001003200D6
:1004B000F2FF37001DF7EF00CE48020000000000F9
:1004C0001DF7EF00CE48020000000000CA82A8001D
:1004D000C682A900CA82A900C682A90010C5B300BD
:1004E00014F7B70015F7EF004215F8001617F900DA
:1004F0004415F8001817F900B24E02000000000081
:100500001DF7EF00CE4802000000000046F5B700DE
:100510004655E20001003200F9FF37001DF7EF00F9
:10052000CE48020000000000E40F20000024E1009B
:1005300001003200F9FF37001DF7EF00CE4802003E
:10054000000000003DF5B7001DF7EF00CE480200A7
:1005500000000000CA82A800C682A9003DD5BF00E5
:100560000160EF0001002000CF02780000000600CB
:10057000851F7800861F7800AE8AA900AE6AAF009A
:1005800011003700140020000960EF00E05B8000DC
:10059000F15B80000402E8000402E900030032007D
:1005A0000000D0008180D200FBFF3700A45A8000F9
:1005B0000400400080A98800B45A800004804800EC
:1005C00090A9880012003700AE6AAE001000370014
:1005D000240020000960EF00E05B8000F15B8000F8
:1005E0000402E8000402E900030032000000D00029
:1005F0008180D200FBFF3700A45A80000400400035
:1006000080A98800B45A80000480480090A988001E
:10061000245C80004822DE006124E100C5003A002D
:10062000AE6AAF004700370084A980006102420033
:100630008402780094A9800060024A0004037800D4
:10064000F5A9880006AA88002A820200000000009E
:1006500034F5B70034D5BF0080EBB700816BEF00F5
:10066000822BEF0082CBBF0083EBB70081CBBF00B2
:1006700082EBB70080CBBF0081EBB700806BEF004F
:100680003015F8003E15F9003215F8004015F90054
:100690002A8202000000000035F5B700A4A98000FE
:1006A0004822DE00035C800004804100005C88007A
:1006B000135C8000E0814900135C8800822BEF000E
:1006C000145C80006020E10019003E000400390045
:1006D000045C800003FF2F000418E10014003600C2
:1006E000140020000960EF00005C8000115C8000B5
:1006F0000402E8000402E900030032000000D00018
:100700008180D200FBFF3700A45A80000400400023
:1007100080A98800B45A80000480480090A988000D
:10072000D62BEC004220AF00D82BEC0004003700A1
:10073000AE8AA80010C0B30000E0B70090003700F8
:100740007B003700AE6AAE007900370084A98000D4
:10075000630242008402780094A9800060024A008B
:1007600004037800F5A9880006AA88002A820200FE
:100770000000000034F5B70034D5BF0080EBB700AF
:10078000816BEF00822BEF0082CBBF0083EBB700C1
:1007900081CBBF0082EBB70080CBBF0081EBB700FD
:1007A000806BEF0084A9800062024200840278001E
:1007B00094A9800060024A0004037800F5A988002B
:1007C00006AA88002A8202000000000035F5B70062
:1007D000A4A980004822DE00035C80000480410060
:1007E000005C8800135C8000E0814900135C880095
:1007F00082CBBF0083EBB70081CBBF0082EBB70099
:1008000080CBBF0081EBB700806BEF0084A9800034
:10081000610242008402780094A9800060024A00CC
:1008200004037800F5A9880006AA88002A8202003D
:100830000000000036F5B700B4A980000960EF00A1
:10084000035C800004804100005C8800135C800031
:10085000E0814900135C880082CBBF0083EBB700C6
:1008600081CBBF0082EBB70080CBBF0081EBB7002C
:10087000806BEF003015F8003E15F9003215F800D6
:100880004015F9002A8202000000000037F5B70089
:10089000B4A980004822DE00035C8000048041008F
:1008A000005C8800135C8000E0814900135C8800D4
:1008B000045C8000F3FF2F000418E10004003A00FC
:1008C000145C8000F3FF20000418E10014003200E3
:1008D000240020000960EF00005C8000115C8000B3
:1008E0000402E8000402E900030032000000D00026
:1008F0008180D200FBFF3700A45A80000400400032
:1009000080A98800B45A80000480480090A988001B
:10091000D62BEC004220AF00D82BEC0004003700AF
:10092000AE8AA80010C0B30000E0B7001400370082
:1009300012003700854BE20010003A00E45B8000B3
:1009400061024200045C8800F45B800060024A009F
:10095000145C8800D62BEC004220AF00D82BEC00B2
:10096000B05E8000720CE30004003A00C05E8000BC
:10097000740CE30001003A00AE8AA8000060EF00AA
:100980004F037800CF02780000000600851F780032
:10099000C500200003000900B51F78000202B8005E
:1009A00003F0A600020037000383B90001003700FE
:1009B0000303B8004200A9008502430060844B0095
:1009C00001F0A60002003700028BB90001003700D9
:1009D000020BB80085024B0008844B000980B00070
:1009E000038BB90008044B0087834C008701780013
:1009F00008017800850078000400780025012000B7
:100A000003000900CF127800CF0278000000060032
:100A1000851F7800861F7800871F78005A35EF0001
:100A20005635EF00A4002000C4AA88005235EF001C
:100A30005435EF005015E20003003A00000020009A
:100A400001002000D9003700D0AA80005A35EC0000
:100A500080027800050078005015B400104078003E
:100A60005CF5B700E4AA8000D4C2B2000A003A00E4
:100A700014002000B4AA8800D0AA80005A35EC00E7
:100A800080027800050078005015B400104078000E
:100A90005CF5B7000A003700E4AA8000B4C2B200D7
:100AA00007003A00D0AA80005A35EC008002780096
:100AB000050078005015B400104078005CF5B700D0
:100AC000E4AA800003032000041CE100A7003E000C
:100AD000E4AA800093032000041CE100A300390075
:100AE000E4AA800004C3B20014003A00D0AA800037
:100AF0005015B4001042780084C7B20005003200DF
:100B0000D0AA80005015B4001042780084C5B2000D
:100B10000A003A0004012000C4AA88005A35EC00FB
:100B2000D0AA80005A35EC008002780005007800D9
:100B30005015B400104078005CF5B700C4AA8000DE
:100B40006A20E10023003A00E4AA800003032000A9
:100B5000041CE1001E003E00E4AA80009303200074
:100B6000041CE1001A003900A00020000100200050
:100B700092AA8000A3AA8000C684020000000000A0
:100B80008002780001037800E4AA80000443B100E9
:100B90000440780000E0B7000080FB000500400042
:100BA00090AA88000400200006004A00A0AA88003D
:100BB000D0AA80005A35EC00800278000500780049
:100BC0005015B400104078005CF5B700DEFF370028
:100BD00066003700C4AA80007020E10063003A007C
:100BE000E4AA800013062000041CE10007003E0078
:100BF000E4AA8000A3072000041CE10003003900E0
:100C00005CD5BF00F04DB200010037005CD5BF00DD
:100C10005CF5B700E4AA800003032000041CE10097
:100C200005003E00E4AA800093032000041CE100BC
:100C30000100390008003700E4AA800013042000F6
:100C4000041CE10049003E00E4AA80006304200087
:100C5000041CE10045003900E4AA800003032000E1
:100C6000041CE10018003E00E4AA80009303200069
:100C7000041CE100140039004400200095AA800003
:100C8000A6AA80000402E8000402E9000300320082
:100C90008502D0000683D200FBFF3700E4AA800063
:100CA0000443B1000440780000E0B7000080FB007E
:100CB000050040000400200086004A0090AA880039
:100CC000A1AA8800140037004400200095AA8000E3
:100CD000A6AA80000402E8000402E9000300320032
:100CE0008502D0000683D200FBFF3700E4AA800013
:100CF0001444B1000440780000E0B7006A404000AE
:100D00000080FB00050040000400200086004A002F
:100D100090AA8800A1AA8800D0AA80005A35EC00C9
:100D200080027800050078005015B400104078006B
:100D30005CF5B700E4AA800013062000041CE10063
:100D400007003E00E4AA8000A3072000041CE10085
:100D5000030039005CD5BF00F04DB2000100370040
:100D60005CD5BF005CF5B700AAFF3700C4AA8000BD
:100D70006A20E1000B003A00B4AA80006120E10083
:100D800008003A000400200093AA800003005200EB
:100D900090AA880004002000A3AA800003005A0043
:100DA000A0AA880090AA8000A1AA8000CF037800A2
:100DB0004F037800CF02780000000600851F7800FE
:100DC000861F780040D5BF0043F5B70014AA800005
:100DD0004822DE006A24E10008003A00C06EEF00FD
:100DE000C36EEF00A0C0B300BFEEB7009C6FEF0072
:100DF0000060EF00AD00370033003700F47580006D
:100E00004822DE006A24E10011003A0014AA8000A2
:100E10004822DE00B4C3B2000D003A00C36EEC00FD
:100E2000F47580004822DE006A24E10005003A00E3
:100E3000C3CEBF004155E30002003A0010C0B3002A
:100E4000BFEEB7000060EF00980037001E003700CB
:100E5000F47580004822DE006A24E10005003A00B3
:100E60004155E20003003A0010C0B300BFEEB700E6
:100E700015003700F47580004822DE006124E1008F
:100E800007003A0014AA80004822DE00B4C3B20072
:100E900003003A0020C0B300BFEEB7000A003700DD
:100EA000F47580004822DE006324E10006003A0069
:100EB00014AA80004822DE006D24E10002003A00FE
:100EC00040C0B300BFEEB700F47580004822DE00DA
:100ED0006124E10018003A00047680000960EF0008
:100EE000C3FE20008302420043D5BF00804A780041
:100EF00014AA80006124E1000D003A00047680000D
:100F00000960EF00C3FE2000030042009042780019
:100F1000047680000960EF00C3EF20000300420068
:100F200010407800002CE10001003200BF6EEF009D
:100F3000C06EEC005C003700F47580004822DE00D3
:100F40006224E1002E003A00047680000960EF0080
:100F5000C3FE200083024200804AEB00C06EEF0017
:100F600014AA80006524E10014003A00C4FE2000A9
:100F700084AA8800088502000000000060768800CE
:100F800060768000747680000020E1000200360068
:100F9000BE6EA90004003700BE6EA80030C0B300CA
:100FA00000E0B70041003700BF6EEF00C16EEF00F8
:100FB00020C0B30000E0B7003C00370050C0B300D1
:100FC00045F5B700C4EF200034AA8800C4FE200015
:100FD00044AA8800C46402000000000044F5B70081
:100FE0004455E20004003A0030C0B300BFEEB70041
:100FF000C16EEF0001003700BF6EEF002A0037001E
:10100000F47580004822DE006324E10008003A0005
:10101000047680004822DE00C3F9200083024200EB
:1010200043D5BF00804A7800C16EEC001E00370037
:10103000F47580004822DE006424E1001A003A00C2
:10104000047680004822DE00614052000080FB00F0
:10105000C4F920000400400010427800B4C3B2007C
:1010600007003A00047680004822DE00614052000A
:101070000080FB00C4F9200004034000004BEB009B
:10108000047680004822DE00C3F92000830242007B
:10109000804AEB00BF6EEF00C16EEF0010C0B300DE
:1010A00000E0B700010037000060EF004F03780058
:1010B000CF02780000000600851F780040D5BF00F1
:1010C00042F5B70014AA80006A24E10008003A0043
:1010D000C16EEF00C36EEF00BFEEEF00D46EEF0005
:1010E000DE6EEF000060EF001A0137005900370094
:1010F00014AA8000A4C3B20001003A0055003700D2
:10110000F47580004822DE00F4CFB20010003A00EF
:1011100014AA8000B4C3B2000D003A00C36EEC0004
:10112000F47580004822DE00F4CFB20005003A00DA
:10113000C3CEBF004155E30002003A0010C0B30027
:10114000BFEEB7000060EF0002013700410037003A
:10115000F47580004822DE00F4CFB20005003A00AA
:101160004155E20003003A0010C0B300BFEEB700E3
:1011700038003700F47580004822DE006124E10069
:1011800006003A0014AA8000B4C3B20003003A007B
:1011900020C0B300BFEEB7002E003700F47580000A
:1011A0004822DE006324E10006003A0014AA800011
:1011B000B4C3B20003003A0040C0B300BFEEB700B2
:1011C00024003700F47580004822DE006624E10028
:1011D00006003A0014AA8000B4C3B20003003A002B
:1011E00070C0B300BFEEB7001A003700F47580007E
:1011F0004822DE006724E10003003A0080C0B3000B
:10120000BFEEB70013003700F47580004822DE00FF
:101210006924E10006003A0014AA8000B4C3B200B9
:1012200003003A00B0C0B300BFEEB70009003700BA
:10123000F47580004822DE006B24E10005003A00CE
:1012400014AA8000B4C3B20002003A00C0C0B300C8
:10125000BFEEB700F47580004822DE006124E10093
:1012600008003A00047680004822DE0043ED2000AA
:101270008302420042D5BF0080429800C16EEC005C
:10128000B3003700F47580004822DE006224E100DC
:1012900009003A00047680004822DE0043ED200079
:1012A00083024200804AEB00C16EEF0030C0B30001
:1012B000BFEEB700A6003700F47580004822DE00BC
:1012C0006324E10008003A00047680004822DE0032
:1012D000E3ED20008302420042D5BF008042980027
:1012E000C16EEC009A003700F47580004822DE00E1
:1012F0006424E10009003A00047680004822DE0000
:10130000E3ED200083024200804AEB00C16EEF0053
:1013100050C0B300BFEEB7008D003700F4758000F9
:101320004822DE006524E10016003A0014AA80007D
:1013300014C3B20003003A0010C0B300C2EAB70001
:101340000D00370014AA800024C3B20003003A0045
:1013500020C0B300C2EAB7000700370014AA80001B
:1013600054C3B20003003A0050C0B300C2EAB70051
:1013700001003700C26AEF0060C0B300BFEEB700E3
:1013800073003700F47580004822DE006824E10015
:1013900009003A0014AA800014C3B20002003A0007
:1013A000AE4AA80001003700AE4AA90090C0B300C1
:1013B000BFEEB70066003700F47580004822DE00FB
:1013C0006B24E1000B003A0014AA8000B4C3B20001
:1013D00007003200047680004822DE0083EE200001
:1013E0008302420042D5BF0080429800C16EEC00EB
:1013F00057003700F47580004822DE006C24E100BD
:1014000009003A00047680004822DE0083EE2000C6
:1014100083024200804AEB00C16EEF00D0C0B300EF
:10142000BFEEB7004A003700F47580004822DE00A6
:101430006D24E10015003A0014AA8000B4C3B20084
:101440000A003A00047680004822DE0023FF2000D4
:1014500083024200804AEB00C16EEF00E0C0B3009F
:10146000BFEEB7000060EF003A003700047680005E
:101470004822DE0023FF20008302420042D5BF0045
:1014800080429800C16EEC0031003700F475800096
:101490004822DE006E24E10015003A0014AA800004
:1014A000B4C3B2000A003A00047680004822DE008D
:1014B000A3FF200083024200804AEB00C16EEF00D0
:1014C000F0C0B300BFEEB7000060EF0021003700AE
:1014D000047680004822DE00A3FF20008302420041
:1014E00042D5BF0080429800C16EEC001800370062
:1014F000F47580004822DE006F24E10014003A00F9
:1015000014AA8000B4C3B2000A003A000476800036
:101510004822DE002300210083024200804AEB00C3
:10152000C16EEF00BF6EEF0010C0B30000E0B70067
:1015300008003700047680004822DE0023002100E6
:101540008302420042D5BF0080429800C16EEC0089
:101550000060EF00CF02780000000600851F7800D1
:10156000C500200003000900B51F78000900200015
:101570004300AF0019002000891F780083846800B1
:1015800001F0A600050037000000EA00010032006B
:1015900001003A008100EA008180EA0003F0A60021
:1015A000050037000201EA000100320001003A00A4
:1015B0008301EA008381EA0003026900150032001A
:1015C0000002EB008002EB000003EB008003EB0065
:1015D000080220004200A9000080D2008180D200D1
:1015E0000482D2008582D2000328E10001003A0083
:1015F00002A0E100030039000202520083825A0077
:101600004200A8000683D2008783D2000804E900C4
:10161000F0FF3A0009F0A600060037000600EA00D5
:101620000100320001003A008700EA008780EA00EA
:1016300003003700870078000600780000003700BC
:10164000CF0478000900E000010032000400BE0071
:101650002501200003000900CF127800CF02780096
:1016600000000600851F78006B55E2000400320080
:1016700074AB8000F3072000041CE100010031007E
:10168000230037006BD5BF005FF6B7006ED5BF00F3
:1016900060F6B700044202000000000060AB80006A
:1016A000EF02600085AB88007035D4007035D4003F
:1016B00060AB80004400DE0060AB880060AB80005F
:1016C000EF02600095AB88007235D4007235D4000B
:1016D00060AB80004400DE0060AB880060AB80003F
:1016E000EF026000A5AB88007435D4007435D400D7
:1016F00070D5BF006CF6B70072D5BF006DF6B700AD
:1017000074D5BF006EF6B700F44002000000000080
:10171000CF02780000000600851F7800D0C2B30019
:1017200051F5B700E4AA8000D3AA8000030052005C
:10173000F0AA8800C4AA8000B3AA80000300520067
:1017400000AB8800F4AA80006020E10006003D00A4
:1017500004002000F3AA800003005200F0AA8800D1
:1017600064B5EF00020037001400200024AB8800AD
:1017700004AB80006020E10006003D000400200072
:1017800003AB80000300520000AB880062B5EF009D
:10179000020037001400200014AB8800F0AA80007B
:1017A0004100DD00F0AA880000AB80004100DD00B0
:1017B00000AB880056D5BF006BF5B7005AD5BF0007
:1017C0006EF5B7005215F8006C15F900328B020067
:1017D00000000000F0AA800004AB80000020E100BF
:1017E000CD00340084AA80006124E1003700340079
:1017F000C0AA8000B4AA80000020E10015003600D5
:10180000D4AA8000E102520056D5BF006BF5B700A4
:10181000054078006EF5B7005415F8006C15F90016
:10182000328B020000000000D4AA8000E2025200C5
:1018300056D5BF006BF5B700054078006EF5B700D0
:101840005415F8006C15F900328B020000000000FE
:101850001E003700B0AA8000C4AA80000020E1006A
:1018600017003600D4AA800061024200840278008A
:1018700056D5BF006BF5B700054078006EF5B70090
:101880005415F8006C15F900328B020000000000BE
:10189000D4AA8000620242008402780056D5BF00BC
:1018A0006BF5B700054078006EF5B7005415F800E9
:1018B0006C15F900328B02000000000003003700B5
:1018C000C0AA80005615E30000003A0000AB80007B
:1018D0004100DE00F4AA80000000520030AB880016
:1018E000B0AA80005815E3008A00320034AB8000B3
:1018F0006020E10007003500D0AA80006415B40024
:10190000D0AA880034AB800003AB800003005200F3
:1019100030AB8800B0AA80006215B400B0AA88007D
:1019200030AB80005E15B40030AB880056D5BF00E8
:101930006BF5B7005AD5BF006EF5B7005215F80029
:101940006C15F900328B02000000000084AA8000B0
:101950006124E1006E003400C0AA8000B4AA8000B7
:101960000020E1001700360010C6B30051F5B700A3
:10197000D4AA8000E102520056D5BF006BF5B70033
:10198000054078006EF5B7005415F8006C15F900A5
:10199000328B020000000000D4AA8000E202520054
:1019A00056D5BF006BF5B700054078006EF5B7005F
:1019B0005415F8006C15F900328B0200000000008D
:1019C00053003700B0AA8000C4AA80000020E100C4
:1019D0001900360020C6B30051F5B700D4AA800024
:1019E000610242008402780056D5BF006BF5B70053
:1019F000054078006EF5B7005415F8006C15F90035
:101A0000328B020000000000D4AA80006202420073
:101A10008402780056D5BF006BF5B700054078000A
:101A20006EF5B7005415F8006C15F900328B020002
:101A30000000000036003700C0AA80005615E30001
:101A400033003A0084AA80004822DE0014C6B200A7
:101A500015003A00D4AA8000E102520056D5BF001A
:101A60006BF5B700054078006EF5B7005415F80027
:101A70006C15F900328B020000000000D4AA80002F
:101A8000E202520056D5BF006BF5B7000540780062
:101A90006EF5B7005415F8006C15F900328B020092
:101AA000000000001A00370084AA80004822DE00EF
:101AB00024C6B20016003A00D4AA80006102420097
:101AC0008402780056D5BF006BF5B700054078005A
:101AD0006EF5B7005415F8006C15F900328B020052
:101AE00000000000D4AA8000620242008402780054
:101AF00056D5BF006BF5B700054078006EF5B7000E
:101B00005415F8006C15F900328B0200000000003B
:101B100073FF3700CC00370084AA80006124E10005
:101B200037003400E0AA8000D4AA80000020E10041
:101B300017003600B4AA80006102420084027800D7
:101B4000054078006BF5B7005AD5BF006EF5B700B9
:101B50005415F8006C15F900328B020000000000EB
:101B6000B4AA800062024200840278000540780036
:101B70006BF5B7005AD5BF006EF5B7005415F800E5
:101B80006C15F900328B0200000000001C003700C9
:101B9000D0AA8000E4AA80000020E10015003600F1
:101BA000B4AA8000E1025200054078006BF5B7004E
:101BB0005AD5BF006EF5B7005415F8006C15F90042
:101BC000328B020000000000B4AA8000E202520042
:101BD000054078006BF5B7005AD5BF006EF5B70029
:101BE0005415F8006C15F900328B0200000000005B
:101BF00003003700E0AA80005A15E30000003A0015
:101C0000F0AA80004100DE0004AB8000000052001A
:101C100030AB8800D0AA80005C15E3008A00320057
:101C200034AB80006020E10007003500B0AA8000DE
:101C30006215B400B0AA880034AB8000F3AA80001B
:101C40000300520030AB8800D0AA80006415B400B5
:101C5000D0AA880030AB80006015B40030AB88009B
:101C600056D5BF006BF5B7005AD5BF006EF5B7006B
:101C70005215F8006C15F900328B020000000000CC
:101C800084AA80006124E1006E003400E0AA800094
:101C9000D4AA80000020E1001900360040C6B3003D
:101CA00051F5B700B4AA80006102420084027800B6
:101CB000054078006BF5B7005AD5BF006EF5B70048
:101CC0005415F8006C15F900328B0200000000007A
:101CD000B4AA8000620242008402780005407800C5
:101CE0006BF5B7005AD5BF006EF5B7005415F80074
:101CF0006C15F900328B0200000000005100370023
:101D0000D0AA8000E4AA80000020E100170036007D
:101D100050C6B30051F5B700B4AA8000E1025200EA
:101D2000054078006BF5B7005AD5BF006EF5B700D7
:101D30005415F8006C15F900328B02000000000009
:101D4000B4AA8000E2025200054078006BF5B700AB
:101D50005AD5BF006EF5B7005415F8006C15F900A0
:101D6000328B02000000000036003700E0AA80003D
:101D70005A15E30033003A0084AA80004822DE00AE
:101D800044C6B20017003A00B4AA800061024200C3
:101D900084027800054078006BF5B7005AD5BF0083
:101DA0006EF5B7005415F8006C15F900328B02007F
:101DB00000000000B4AA80006202420084027800A1
:101DC000054078006BF5B7005AD5BF006EF5B70037
:101DD0005415F8006C15F900328B02000000000069
:101DE0001800370084AA80004822DE0054C6B200E2
:101DF00014003A00B4AA8000E102520005407800C5
:101E00006BF5B7005AD5BF006EF5B7005415F80052
:101E10006C15F900328B020000000000B4AA8000AB
:101E2000E2025200054078006BF5B7005AD5BF00BA
:101E30006EF5B7005415F8006C15F900328B0200EE
:101E40000000000073FF3700CF027800000006009A
:101E5000851F7800861F780070C1B30068F6B70050
:101E600002CBBF0069F6B700C63F020000000000C9
:101E7000545880000960EF006620B8000080FB0025
:101E80001458800084024000801F780080C1B30095
:101E900068F6B7004F007800801F78000540780092
:101EA00069F6B7004F007800C63F0200000000004E
:101EB00090C1B30068F6B70004CBBF0069F6B70065
:101EC000C63F020000000000245880008307200065
:101ED0000418E1000D0039000BCBBF004300DD000A
:101EE0000080FB002458800084024000618352007F
:101EF000A0C1B30068F6B7000640780069F6B700E5
:101F0000C63F0200000000000C0037000BCBBF00F2
:101F10004300DD000080FB00245880008402400064
:101F200068835200A0C1B30068F6B700064078008D
:101F300069F6B700C63F02000000000000C2B3000F
:101F400068F6B70002CBBF0069F6B700C63F0200D3
:101F5000000000000BCBBF004300DD000080FB0051
:101F600024588000840240006183520010C2B300F4
:101F700068F6B7000640780069F6B700C63F020071
:101F8000000000000470200094168800E822A900D8
:101F9000CB62A900C762A900CB82A800C782A900B2
:101FA000CBA2A900C7A2A90024822000B4168800F1
:101FB000CBA2A800C7A2A900CB62A800C762A90053
:101FC000E822A8005375EF0094AA80004822DE00A2
:101FD00084C2B2004900320094AA80006124E1006A
:101FE00007003A0053D5BF000160EF004100DD005B
:101FF0001822020000000000A0AA88001D0037007F
:1020000094AA80006224E10007003A0053D5BF0083
:102010000160EF004100DD006E22020000000000C0
:10202000A0AA88001300370094AA80006324E1006E
:1020300007003A0053D5BF000160EF004100DD000A
:10204000C422020000000000A0AA88000900370096
:1020500094AA80006424E10006003A0053D5BF0032
:102060000160EF004100DD001A23020000000000C3
:10207000A0AA8800A0AA8000EF026000D5AA88006C
:102080005A35D4005A35D400A0AA80004400DE009E
:10209000A0AA8800A0AA8000EF026000C5AA88005C
:1020A0005835D4005835D400A0AA80004400DE0082
:1020B000A0AA8800A0AA8000EF026000B5AA88004C
:1020C0005635D4005635D400A0AA80004400DE0066
:1020D000A0AA880056D5BF006CF6B70058D5BF003F
:1020E0006DF6B7005AD5BF006EF6B700F440020097
:1020F000000000005375EC00B3FF37005458800017
:102100000960EF006620B8000080FB00022BB400DD
:102110004F037800CF02780000000600851F78008A
:10212000861F78005835EF005435EF00A4002000DA
:10213000B4AA88005235EF005015E20002003A00C0
:102140000020EF00B9003700C0AA80005835EC002D
:1021500080027800050078005015B4001040780027
:102160005AF5B700D4AA8000D4C2B2000A003A00DF
:1021700014002000A4AA8800C0AA80005835EC00F2
:1021800080027800050078005015B40010407800F7
:102190005AF5B7000A003700D4AA8000B4C2B200D2
:1021A00007003A00C0AA80005835EC008002780091
:1021B000050078005015B400104078005AF5B700BB
:1021C000D4AA800003032000041CE1008B003E0021
:1021D000D4AA800093032000041CE100870039008A
:1021E000D4AA800004C3B20014003A00C0AA800040
:1021F0005015B4001042780084C7B20005003200C8
:10220000C0AA80005015B4001042780084C5B20006
:102210000A003A0004012000B4AA88005835EC00F6
:10222000C0AA80005835EC008002780005007800D4
:102230005015B400104078005AF5B700B4AA8000D9
:102240006A20E1001B003A00D4AA800003032000AA
:10225000041CE10016003E00D4AA80009303200075
:10226000041CE1001200390094AA80006A20B80022
:1022700080027800D4AA80000443B10004407800B2
:1022800000E0B7000080FB000500400090AA880035
:10229000C0AA80005835EC00800278000500780064
:1022A0005015B400104078005AF5B700E6FF37002B
:1022B00052003700B4AA80007020E1004F003A00BD
:1022C000D4AA800013062000041CE10007003E0091
:1022D000D4AA8000A3072000041CE10003003900F9
:1022E0005AD5BF00F04DB200010037005AD5BF00EB
:1022F0005AF5B700D4AA800003032000041CE100B3
:1023000005003E00D4AA800093032000041CE100D5
:102310000100390008003700D4AA8000130420000F
:10232000041CE10035003E00D4AA800063042000B4
:10233000041CE10031003900D4AA8000030320000E
:10234000041CE1000E003E00D4AA8000930320008C
:10235000041CE1000A00390095AA8000C42ADD00AF
:10236000D4AA80000443B1000440780000E0B70024
:102370000080FB000500400090AA88000A0037009A
:1023800095AA8000C42ADD00D4AA80001444B100BC
:102390000440780000E0B7006A4040000080FB0085
:1023A0000500400090AA8800C0AA80005835EC00C3
:1023B00080027800050078005015B40010407800C5
:1023C0005AF5B700D4AA800013062000041CE100CF
:1023D00007003E00D4AA8000A3072000041CE100EF
:1023E000030039005AD5BF00F04DB200010037009C
:1023F0005AD5BF005AF5B700BEFF3700A4AA800027
:102400006120E10007003A00B4AA80006A20E100E0
:1024100004003A000400200093AA80000300520048
:1024200090AA88005215F8000000F9004F037800C8
:10243000CF02780000000600851F7800861F780014
:10244000871F7800881F7800C34AE20003003A0023
:10245000A4AA200074AA88002C003700145680001B
:102460004822DE006124E10003003A00040F20004E
:1024700074AA880025003700145680004822DE0028
:102480006224E10003003A00F40F200074AA8800DF
:102490001E003700145680004822DE006324E1004D
:1024A00003003A00F400200074AA880017003700E7
:1024B000145680004822DE006624E10003003A0042
:1024C000040F200074AA8800100037001456800002
:1024D0004822DE006724E10003003A00F40F2000E8
:1024E00074AA880009003700145680004822DE00D4
:1024F0006824E10003003A00F400200074AA880078
:1025000002003700F40F200074AA88004435EF0061
:1025100040568000E45680000020E10020003C008E
:102520000400350030568000D45680000020E100C1
:102530001B003E0060578000445680000020E100F0
:1025400017003C00040035005057800034568000CE
:102550000020E10012003E008056800004578000F9
:102560000020E1000E003C000400350070568000A1
:10257000F45680000020E10009003E0080578000F2
:10258000845680000020E1000800350004003C0073
:1025900070578000745680000020E1000300360070
:1025A00024AA80006202420024AA880060568000AB
:1025B000E45680000020E10020003C0004003500CB
:1025C00050568000D45680000020E1001B003E00E1
:1025D00060578000645680000020E10017003C0036
:1025E0000400350050578000545680000020E10060
:1025F00012003E00A0568000045780000020E10039
:102600000E003C000400350090568000F456800017
:102610000020E10009003E0080578000A4568000A1
:102620000020E1000800350004003C0070578000E5
:10263000945680000020E1000300360024AA8000A8
:102640006102420024AA88004415E20001003A0019
:102650000400370024AA80006320E1000100390053
:10266000130237004255E20004003A004355E200ED
:1026700002003A000E0237000C0037004255E2001B
:102680000A003A0014AA80004822DE006124E1001A
:1026900006003A0024AA80006120E10002003E000A
:1026A000D7003700010037000102370024AA80005C
:1026B0006220E100D2003E00A400200024AA88008D
:1026C00040568000E45680000020E10006003500FE
:1026D0000E003C0030568000D45680000020E100FF
:1026E000010039000900370060578000445680001F
:1026F0000020E1000800350004003C005057800035
:10270000345680000020E1000300390024AA800034
:102710006102420024AA880080568000045780008D
:102720000020E100060035000E003C0070568000DD
:10273000F45680000020E100010039000900370054
:1027400080578000845680000020E100080035009A
:1027500004003C0070578000745680000020E100A7
:102760000300390024AA80006102420024AA8800E4
:1027700060568000E45680000020E100060035002D
:102780000E003C0050568000D45680000020E1002E
:10279000010039000900370060578000645680004E
:1027A0000020E1000800350004003C005057800084
:1027B000545680000020E1000300390024AA800064
:1027C0006102420024AA8800A056800004578000BD
:1027D0000020E100060035000E003C00905680000D
:1027E000F45680000020E1000100390009003700A4
:1027F00080578000A45680000020E10008003500CA
:1028000004003C0070578000945680000020E100D6
:102810000300390024AA80006102420024AA880033
:1028200024AA80006B20E100010039004375EF000D
:1028300024AA80006B20E1006D003E00405680001D
:10284000E45680000020E1000A00350004003C004E
:1028500030568000D45680000020E1000500390089
:10286000DA0AF800C60AF900DC0AF800C80AF9001A
:102870000D00370060578000445680000020E100C2
:102880000900350004003C00505780003456800099
:102890000020E10004003600EA0AF800C60AF90048
:1028A000EC0AF800C80AF90080568000045780003E
:1028B0000020E1000A00350004003C007056800052
:1028C000F45680000020E10005003900DE0AF8001F
:1028D000CE0AF900E00AF800D00AF9000D0037002E
:1028E00080578000845680000020E10009003500F8
:1028F00004003C0070578000745680000020E10006
:1029000004003600EE0AF800CE0AF900F00AF800DA
:10291000D00AF90060568000E45680000020E100F3
:102920000A00350004003C0050568000D456800058
:102930000020E10005003900DA0AF800CA0AF900AF
:10294000DC0AF800CC0AF9000D003700605780005F
:10295000645680000020E1000900350004003C00BE
:1029600050578000545680000020E10004003600DB
:10297000EA0AF800CA0AF900EC0AF800CC0AF900E1
:10298000A0568000045780000020E1000A003500B6
:1029900004003C0090568000F45680000020E100C6
:1029A00005003900DE0AF800D20AF900E00AF80052
:1029B000D40AF9000D00370080578000A45680002B
:1029C0000020E1000900350004003C007057800041
:1029D000945680000020E10004003600EE0AF80062
:1029E000D20AF900F00AF800D40AF900040037000E
:1029F00024AA80006B20E100010036002C01370082
:102A000034568000D3568000830252004456800022
:102A1000E356800003035A00B0568000C156800080
:102A200002FA200003002000A84F0200000000006E
:102A300080037800010478004300A90007007800B3
:102A400088007800020A200003002000D84F02000E
:102A5000000000004300A900000178008101780017
:102A60000500780086007800AE8A020000000000B1
:102A700030AA880054568000D3568000830252004A
:102A800064568000E356800003035A00B05680006D
:102A9000C156800002FA200003002000A84F020067
:102AA0000000000080037800010478004300A900C2
:102AB0000700780088007800020A20000300200048
:102AC000D84F0200000000004300A9000001780078
:102AD000810178000500780086007800AE8A020047
:102AE0000000000040AA880074568000F356800061
:102AF00083025200845680000357800003035A006B
:102B0000B0568000C15680000278200003002000EB
:102B1000A84F020000000000800378000104780044
:102B2000740020000960EF0007007800880078003A
:102B30000402E8000402E900030032008100D10031
:102B40000080D300FBFF37004300A900000178009C
:102B5000810178000500780086007800AE8A0200C6
:102B60000000000050AA880094568000F3568000B0
:102B700083025200A45680000357800003035A00CA
:102B8000B0568000C156800002782000030020006B
:102B9000A84F0200000000008003780001047800C4
:102BA000740020000960EF000700780088007800BA
:102BB0000402E8000402E900030032008100D100B1
:102BC0000080D300FBFF37004300A900000178001C
:102BD000810178000500780086007800AE8A020046
:102BE0000000000060AA88004AB5EE0054AA8000E8
:102BF000030820000418E10003003E0054AA8000EE
:102C00000408B10054AA88004CB5EE0064AA800004
:102C1000030820000418E10003003E0064AA8000BD
:102C20000408B10064AA880014AA80006124E100AD
:102C300010003A0010C0B30050F5B7005435EF0053
:102C4000F4FF200094AA88004615F8005615F900F4
:102C50004815F8005815F9004A15F8005A15F900FA
:102C60004C15F8005C15F9008C8B02000000000088
:102C70005400370014AA80006224E10010003A00DA
:102C800010C0B30050F5B7005435EF0004F0200039
:102C900094AA88004615F8005615F9004815F80062
:102CA0005815F9004A15F8005A15F9004C15F800A6
:102CB0005C15F9008C8B0200000000004100370019
:102CC00014AA80006324E10011003A0020C0B30080
:102CD00050F5B700F4FF200094AA88004E15F800C4
:102CE0005415F9004615F8005615F9004815F80076
:102CF0005815F9004A15F8005A15F9004C15F80056
:102D00005C15F9008C8B0200000000002D003700DC
:102D100014AA80006424E10018003A0046D5BF00E0
:102D20005FF6B7004AD5BF0060F6B7000442020064
:102D300000000000145680004822DE006424E100F8
:102D400008003600145680004822DE00E44252009B
:102D50000540780052F5B700288F020000000000FF
:102D600004003700C3CABF0052F5B700288F020025
:102D7000000000004375EF001200370014AA800025
:102D80006524E1000F003A0010C0B30050F5B70011
:102D90005435EF00D4D0200094AA88004615F800DE
:102DA0005615F9004815F8005815F9004A15F800AD
:102DB0005A15F9004C15F8005C15F9008C8B0200CF
:102DC0000000000014AA80004822DE006124E10017
:102DD00037003A000250E20001003A000C003700D0
:102DE0002400210084AA88008E90020000000000C8
:102DF000C45680000120E1000500350003003C00BE
:102E0000B45680000020E1000100360028003700A1
:102E100054AA800083F72F000418E10001003E004F
:102E20002300370046D5BF005FF6B7004AD5BF0084
:102E300060F6B7000442020000000000F24FE2001A
:102E400002003A0004F020003458880024FF2000DB
:102E500084AA88000885020000000000305888001D
:102E6000FA4FE20002003A00F40F200044588800B4
:102E7000A4FF200084AA880008850200000000004A
:102E80004058880081EE20001104E0000800320064
:102E9000811F78001140780062F6B700BA45020041
:102EA00000000000CF0078008100E800F6FF370046
:102EB000C60AF800CA0AF900C80AF800CC0AF900E4
:102EC000CE0AF800D20AF900D00AF800D40AF900B4
:102ED0004F047800CF0378004F037800CF027800CA
:102EE00000000600851F78006E08F8003215F90012
:102EF0007008F8003415F9003215F8003815F9009B
:102F00003415F8003215F9003435EF003215F800A9
:102F10003615F9003F75EF00545D80004822DE0051
:102F20006124E1000400320084A980004822DE0010
:102F30006524E1004C003A00CA82A900C682A900BB
:102F40001DF7EF00CE4802000000000010C5B300DE
:102F500014F7B70015F7EF003615F8001617F9004B
:102F60003815F8001817F900B24E020000000000F2
:102F70001DF7EF00CE480200000000003DF5B7004D
:102F80003D55E200170032003F75EC00F4A98000C7
:102F90004822DE007424E100120039000100200004
:102FA0000100780034340200000000008100E800D5
:102FB0003322AF00FEFF3700A01188004000200040
:102FC0000008E600F6FF37003F75EF00CA82A80050
:102FD000C682A900400620008C3B020000000000D1
:102FE000D5FF37001DF7EF00CE48020000000000BB
:102FF000E40F20000024E100190032003F75EC00CE
:10300000F4A980004822DE0023032000041CE10014
:1030100012003E000100200001007800463402004A
:10302000000000008100E8003322AF00FEFF3700FF
:10303000A0118800300020000008E600F6FF3700ED
:103040003F75EF00CA82A800C682A9004006200092
:103050008C3B020000000000B7FF3700E1FF3700A3
:10306000E8C2A800E902A8003A35EF00D4A9800020
:1030700004A0B200700032003E75EF00AE8AAE00D0
:1030800007003700DA0BE20002003A00DC0BE20036
:1030900003003200DA2BED004200AE00DC2BED0025
:1030A00070C0B3003CF5B700E4A98000F4CFB200D3
:1030B0000E003200E8C2A900E8C2A800E6E2AE00B5
:1030C00008003700E15321003CD5BF000160EF004C
:1030D00012002000821F78004F017800DA3C0200C5
:1030E000000000003C75ED00EFFF3700AE8AAE0037
:1030F00005003700DA0BE20003003A00DC0BE200C7
:1031000001003A004A003700BE4EAE000100370011
:1031100047003700147680006124E10001003A0086
:103120004300370084A980004822DE006124E100CA
:103130000D003A003ED5BF0040F5B70030D5BF00C6
:1031400041F5B70010C0B30042F5B700DE860200BB
:10315000000000006104E10002003A0010C0B3006A
:10316000C2EEB7003200370084A980004822DE009A
:103170006524E1000D003A003ED5BF0040F5B700E0
:1031800030D5BF0041F5B70050C0B30042F5B700DD
:10319000DE860200000000006204E1000200390047
:1031A000BE4EA800220037002100370084A980000D
:1031B0004822DE006924E1001D003A003ED5BF0030
:1031C00040F5B70010C0B30041F5B7005C880200BD
:1031D000000000006104E10015003A0044ED200009
:1031E00084AA88000885020000000000305688008C
:1031F00041568800E4ED200084AA8800088502007A
:103200000000000070568800815688008042EB0064
:10321000AE4AAF008502E800C2CABF0042F5B7005F
:103220000540780043F5B7001C9202000000000042
:103230003A35EC008DFF37001DF7EF00CE48020055
:10324000000000001DF7EF00CE4802000000000063
:10325000AB4BE2000F003A0084A980004822DE0058
:103260006124E1000400320084A980004822DE00CD
:103270006924E10007003A001DF7EF00CE48020084
:1032800000000000E40F20000024E10001003200F3
:10329000F9FF3700545D80004822DE006124E10020
:1032A0000400320084A980004822DE006524E10089
:1032B00002003A00CA82A800C682A90014768000E3
:1032C0006124E10003003A0010C0B30000E0B70041
:1032D00011003700DA0BE20005003A00DC0BE200D7
:1032E00003003A0010C0B30000E0B7000A00370046
:1032F00084A980004822DE006524E10004003A0031
:1033000010C0B30000E0B700030037000200370030
:103310000060EF0000003700CF02780000000600D8
:10332000851F7800861F7800871F7800881F780027
:1033300027D5BF004EEEB70044A980004822DE002A
:103340006524E1000400320044A980004822DE0028
:103350006924E10004003A00C42EEF00C62EEF00FD
:10336000C82EEF00CA2EEF0044A980004822DE00DC
:103370006124E10015003A00347680006020E1000D
:103380001200390003003E00247680007020E10026
:103390000E003900247680007000520020768800EC
:1033A0003476800060005A003076880080598000B2
:1033B0004400DD0044768000000052004076880022
:1033C0005476800060005A00507688004ECEBF00D0
:1033D0000160EF004200DD0024C92000040040002D
:1033E000900278001003900005007800C40EB4002D
:1033F000805B88003476800004004B00905B88007E
:103400004ECEBF000160EF004200DD00E4CF20009F
:10341000040040009002780010039000050078003E
:10342000C80EB400905E88005476800004004B0003
:10343000A05E88004ECEBF000160EF004200DD00BC
:10344000A4D6200004004000901F7800780BF900FB
:10345000100090007AABB7004ECEBF000160EF00C5
:103460004200DD0064DD20000400400010407800D0
:10347000ABEBB7002B75EF001400200094638800BD
:10348000742CEF0085598000C92ADD000500780002
:103490000100200092638000A3638000A84F020017
:1034A00000000000D45B80000120E100080039002A
:1034B00003003E00C45B80000020E10004003600F1
:1034C000722CEC004220AF00742CEC00EDFF3700B2
:1034D00044A980004822DE006524E10008003A008B
:1034E000A46380006020E10005003E000300390075
:1034F000946380007020E100010031006B0137000F
:1035000094638000E1025200A463800060035A00CB
:1035100005007800860078008259800003002000B2
:10352000A84F02000000000080037800010478002A
:103530009400200007007800880078000402E8006A
:103540000402E900030032000000D0008180D200B4
:10355000FBFF3700C45B800000005200D05E880093
:10356000D45B800001005A00E05E8800D62BEF009B
:10357000D82BEF00700BF8007C0BF900720BF800F1
:103580007E0BF900D20BF8008A08F900D40BF80082
:103590008C08F900BF6EEF00C06EEF00C26EEF0046
:1035A000AB4BE2005D003A0044A980004822DE00F7
:1035B0006124E1000400320044A980004822DE00BA
:1035C0006924E10055003A00940020008A08F800C0
:1035D0006E08F9008C08F8007008F9000402E80091
:1035E0000402E900030032006E28D40070A8D6005F
:1035F000FBFF37006E08F8002E15F9007008F80080
:103600006E08F9007028EF006E08F8002C15F9001C
:10361000CA82A900C682A9001DF7EF00CE480200A9
:103620000000000020C5B30014F7B70010C0B300BD
:1036300015F7B7002C15F8001617F9002E15F8002D
:103640001817F900B24E0200000000001DF7EF004D
:10365000CE480200000000002AF5B7002A55E2001B
:103660000E0032002D28AE000B00370001002000B4
:1036700001007800E4330200000000008100E8004F
:103680003322AF00FEFF3700A01188005000200059
:103690000008E600F6FF3700ECFF37001DF7EF00EB
:1036A000CE48020000000000E40F20000024E100EA
:1036B000180032002B75EC0054A980004822DE006F
:1036C00023032000041CE10011003E000100200043
:1036D00001007800F8330200000000008100E800DB
:1036E0003322AF00FEFF3700A01188003000200019
:1036F0000008E600F6FF3700CA82A800C682A900CB
:10370000A00020008C3B020000000000C0FF37003A
:10371000E2FF3700E8C2A800E902A800C42EEF00CB
:10372000C62EEF00C82EEF00CA2EEF00BE6EA90015
:10373000C05E8000A46380000020E100B200390078
:1037400004003E00B05E8000946380000020E10031
:10375000AD003900BE4EA900ABCBBF0085EBB70072
:10376000B88202000000000044A980004822DE0068
:103770006524E1001C003A00C45E80006020E10086
:103780001000390003003E00B45E80006120E100BB
:103790000C00360024768000610242002476880006
:1037A0003476800060024A003476880040768000DB
:1037B000300BB400407688005476800060024A00E6
:1037C00054768800B05E8000EF0260000000EB00DD
:1037D0006128E10002003A000600E0000200320029
:1037E000BE4EA90076003700545D80004822DE00FE
:1037F0006124E1000400320044A980004822DE0078
:103800006524E1004C003A00CA82A900C682A900E2
:103810001DF7EF00CE4802000000000000C5B30015
:1038200014F7B7001637EF0015F7EF00042020005B
:10383000C4B8880014490200000000000004E00041
:103840000E0032002D28AE000B00370001002000D2
:10385000010078000A340200000000008100E80046
:103860003322AF00FEFF3700A01188006000200067
:103870000008E600F6FF3700E5FF37001DF7EF0010
:10388000CE480200000000001DF7EF00CE48020005
:1038900000000000CA82A800C682A900E45B800084
:1038A000E2025200F45B800060035A0005007800D9
:1038B000860078008259800003002000A84F020093
:1038C000000000005044880061448800504480009B
:1038D000680BB40050448800545B8000634480004F
:1038E0000480490060448800AE6AAE0007003700DB
:1038F00054448000835980000300520050448800E3
:103900006444800060005A006044880094002000F5
:103910008A08F8008208F9008C08F8008408F90089
:103920000402E8000402E900030032008228D40007
:1039300084A8D600FBFF37008208F8006E08F90063
:103940008408F8007008F900104480005C0BB40093
:10395000F45A800023448000848049006E08E3000C
:1039600003003A00844380000120E100140032008B
:1039700028D5BF0030F5B70029D5BF0031F5B70015
:1039800072970200000000006104E10001003A00AB
:103990000B003700BE4EAE000100370008003700B4
:1039A000042020007343800004804100704388009D
:1039B0008443800060024A0084438800E2FF3700AD
:1039C000147680006124E10001003A000E00370007
:1039D000BE6EAE00010037000B003700AE8AAF00AC
:1039E00005003700800BF8007C0BF900820BF80013
:1039F0007E0BF90003003700AE8AAE0001003700ED
:103A0000010037004AFF3700AB4BE20027003A00C5
:103A100044A980004822DE006124E1000400320055
:103A200044A980004822DE006924E1001F003A001A
:103A3000CA82A900C682A900C0C4B30014F7B700A7
:103A40001637EF001837EF0015F7EF0014490200A2
:103A5000000000000004E0000C0032000100200023
:103A6000010078001E340200000000008100E80020
:103A70003322AF00FEFF3700A01188007000200045
:103A80000008E600F6FF3700EBFF37001DF7EF00F8
:103A9000CE480200000000001DF7EF00CE480200F3
:103AA00000000000CA82A800C682A9004F04780066
:103AB000CF0378004F037800CF02780000000600A3
:103AC000851F78002C15F8003015F9002B55E20001
:103AD0000B00320070A980001004E00008003200E2
:103AE00080A980003035EC008002780070A9800049
:103AF0002E35EC00904A78002B75ED00F3FF37006F
:103B00002B55E2000600320080A980003035EC0021
:103B100080027800804AEB002B75ED00F8FF37003B
:103B20002C15F8000000F900CF0278000000060014
:103B3000851F78006016F8006216F90010B3800047
:103B40001004E000020032006236EC00FBFF370098
:103B500014B3800003B380000300520000E0B700FC
:103B6000CF02780000000600851F7800861F7800CD
:103B7000C36EEF002455E20009003A00A0C0B30074
:103B80002BF5B700C4EF200064A98800C4F9200019
:103B900074A98800609D0200000000002800370022
:103BA0002575EF0024A980004822DE00B4C4B200CD
:103BB0001600320024A980004822DE00C3F920004C
:103BC0000300420010427800B4C3B2000700320084
:103BD00024A980004822DE00C3F92000030042002F
:103BE00010427800C4C2B20006003A00C36EEC0076
:103BF000C3CEBF002455E30001003A0003003700A4
:103C0000000037002575EC00E6FF370024A980008E
:103C10004822DE00C3F9200084824100E182420094
:103C200005037800D0C0B3002BF5B700C4EF200027
:103C300064A9880076A98800609D02000000000049
:103C40002575EF0024A980004822DE006D24E100E4
:103C50001500320024A980004822DE00C3EF2000B6
:103C60000300420010427800B4C3B20007003200E3
:103C700024A980004822DE00C3EF20000300420098
:103C800010427800C4C2B20005003A0024A98000A6
:103C90004822DE00C3EF200083024200804AEB008E
:103CA0002575EC00E7FF3700C4EF200004B388005F
:103CB000989D0200000000000004E00003003A00AC
:103CC0000060EF00040037000300370010C0B300AD
:103CD00000E0B700000037004F037800CF02780003
:103CE00000000600851F7800C500200003000900C1
:103CF000B51F78000003780081037800040678007F
:103D000004F0A1000400E00006003A0009F0A7005A
:103D100002003700050020001300370005002000D6
:103D200011003700EB4252000E0039000003200062
:103D300009F0A6000002200062F6B700BA450200B2
:103D40000000000041E0AF00FBFF3700801088005A
:103D50001162EF008502E900F7FF3B0055002000EB
:103D60000100370084027800E800200009002000EC
:103D70001000FA000C377C000884E900FDFF3B00CE
:103D8000A400200005E0A0000CF0A70005F0A000B2
:103D9000040F780015079800060078008700780067
:103DA00002A02C00A3B92300087122000DF0A1008D
:103DB0000DF0A2000E6B0200000000000DF0A70045
:103DC000070037004007980051079800000178006D
:103DD000810178002E009000BE009000F4FF3700B3
:103DE0004207980053079800240798003507980069
:103DF0001E0278009E029000060320000000E000F2
:103E000012003A0005E0A600120037000402E900A3
:103E1000040F78000400E0000E0032000524E100E9
:103E2000020032004200AF000E00370006032000FF
:103E30000000E00005003A0005E0A600050037009C
:103E400005F0A600060220000200370005E0A100F0
:103E5000150798000040430062F6B700BA4502001B
:103E6000000000004E009000DE009000A200200044
:103E70008001EB006100E10001003200CCFF37005F
:103E80000080FA002501200003000900CF1278000D
:103E9000CF02780000000600670160004300DE00EA
:103EA00001004000104078000010A5000000EB0069
:103EB0004200AF000000E800000006002415F800F2
:103EC0002815F9002615F8002A15F900F0C1B300ED
:103ED0002CF5B70064A98000F4CFB2000E003200C8
:103EE000815221002CD5BF000160EF004C9F0200E1
:103EF000000000000000A30002003100E902A90058
:103F000001003700E902A800E8C2A900E8C2A80041
:103F10002C75ED00EFFF3700E8C2A9000000060095
:103F2000851F7800861F7800871F7800881F78001B
:103F30002CB5EF002E35EF0074A980008487B20005
:103F4000200032002ED5BF000BE0B7008042EB000E
:103F500015B38800423F020000000000903F0200BD
:103F6000000000004FEEB70034A980004822DE00B8
:103F70006124E10006003A00747280004822DE00ED
:103F80006124E10001003A002C35EC000300370009
:103F90002755E20001003A002C35EC0060A98000B2
:103FA0002815E30003003A00BE3F020000000000B5
:103FB00004003700BE3F0200000000002E35EC0078
:103FC000DDFF37002CD5BF000BE0B7008042EB00CF
:103FD000440B20000483420016B38800423F0200D5
:103FE00000000000903F020000000000C3EAB7009C
:103FF000BE3F0200000000002CD5BF000BE0B70060
:104000008042EB00540B20000483420016B388006A
:10401000423F0200000000002A75EF0054A9800012
:104020006824E100140032002AD5BF000160EF00CF
:104030004200DD0084E52000840240009E4702002B
:1040400000000000800A7800910298002AD5BF0085
:104050000160EF004200DD00C4E720008402400060
:104060009E47020000000000800A7800910298003C
:104070002A75EC00E9FF3700BE3F02000000000097
:104080002CD5BF000BE0B7008042EB00E482420079
:104090000503780016B38800423F020000000000CC
:1040A000903F020000000000C4EAB700BE3F0200DB
